:020000040800F2
:10000000F0FF0010A9B70508E37E0308F9F800081F
:1000100049B8050849B8050849B8050800000000B6
:10002000000000000000000000000000E17E030866
:10003000DF7E030800000000DD7E03085DF9000894
:1000400049B8050849B8050849B8050849B8050878
:1000500049B8050849B80508C1F80308EDF90308CF
:10006000B1F9030875F9030839F903083D3D05089E
:100070002D3D05081D3D05080D3D0508F93C050809
:10008000E53C0508D13C050849B8050849B805080C
:1000900049B8050849B8050849B80508FDF8030836
:1000A00081A200081DA80008B1A10008F9A8000855
:1000B0005DA700089DA60008D1A50008B553050856
:1000C000BD530508A5530508AD53050849B80508F3
:1000D00049B8050861FB000849B80508A9FA0008F5
:1000E00085F8030849B8050899C30308E1A000088A
:1000F00051A3000811A0000831A40008BD3C050868
:1001000049B8050849B8050801A5000849B8050817
:1001100049B8050849B805084929030835290308DD
:10012000A93C0508953C0508813C05086D3C05087F
:10013000593C050849B8050849B8050849B80508F3
:1001400049B8050849B8050849B80508999503084C
:10015000453C0508313C05081D3C0508F1F900083F
:10016000955305089D53050849B8050849B8050881
:1001700049B8050849B8050849B8050849B8050847
:0801800049B8050849B805085B
:0801880050B305000100000066
:100190001A0201003C00000068190020D41D002054
:1001A00000000000E17F02082700010004000000B9
:1001B000501C0020101E002000000000E008000875
:1001C0003810010001000000E8170020141E002074
:1001D00000000000E4080008220201001C010000E9
:1001E00034360020B838002000000000CD8302081B
:1001F0000C200600CC0000008C340020D4390020F4
:1002000000000000C5E10208010201000500000035
:1002100054340020A03A002000000000BD0D010869
:1002200000020100050000004C340020A83A002024
:1002300000000000000000001B0201001000000090
:1002400020340020B03A0020000000002D78020881
:100250001B1001000C00000078200020C03A002094
:10026000000000006F25010821020100F0000000DD
:10027000F81E0020CC3A002000000000CD24010828
:1002800023120100100000009C350020BC3B002020
:1002900000000000E808000805100100060000004A
:1002A00094350020CC3B002000000000F808000836
:1002B000371001002E00000090330020D43B0020B6
:1002C00000000000FE0800080E020100020000000D
:1002D00090350020043C0020000000002C0900089C
:1002E00016100100060000001C1E0020083C002023
:1002F000000000002E0900082F100100220000005D
:1003000094380020103C0020000000003409000850
:100310001E0001000700000084300020343C002053
:100320000000000056090008231001000E00000024
:10033000E43000203C3C0020000000004D86010815
:10034000F5610100CC000000241E00204C3C002080
:1003500000000000255801081C0202001C000000DB
:10036000C44400206849002000000000B180020859
:1003700028100100160000005C480020844900207D
:10038000000000003DA70108140001000300000068
:10039000544800209C490020000000005E0900082D
:1003A000012001000C00000034400020A049002082
:1003B00000000000620900080A7001002800000027
:1003C000983F0020AC49002000000000F1850108A2
:1003D0000ED0030092010000043E0020D44900200A
:1003E000000000004538040801010100040000007D
:1003F000583D0020684B0020000000000000000075
:100400000001010004000000503D00206C4B002062
:10041000000000006E090008020101000300000056
:100420004C3D0020704B00200000000001E202085B
:100430001F02080010000000F4560020E4560020BF
:1004400000000000C1780208081203000F0000003D
:1004500038810020948100200000000051780208BB
:1004600007020100020000007C810020A48100201E
:100470000000000074090008F62101000C000000D3
:1004800064810020A8810020000000007809000895
:10049000020001000C00000058810020B4810020FF
:1004A0000000000000000000060203000C00000035
:1004B0004C810020C081002000000000398102082A
:1004C0001D0201000200000030810020CC810020CC
:1004D00000000000840900080A0201001400000066
:1004E000087E0020508600200000000049E6020837
:1004F00003000100010000001C7900206486002038
:100500000000000000000000031201003D00000098
:10051000DC800020688600200000000086090008BA
:1005200025201E002C010000447E0020A88600200B
:100530000000000000000000101001000200000098
:1005400084780020D487002000000000C40900083F
:10055000261001000E0000008C9900207C990020DC
:1005600000000000A96A03080B3001001A00000017
:1005700088930020C899002000000000C8090008E6
:100580001F30010024000000D48A0020E4990020DC
:1005900000000000E409000805020100040000005A
:1005A00058960020089A002000000000080A000861
:1005B000030101000A000000209300200C9A002093
:1005C0000000000039660308130201000400000067
:1005D000FC870020189A0020000000000C0A000888
:1005E0002802040004000000B09A0020B49A002001
:1005F000000000004D7802082702040004000000FB
:10060000AC9A0020B89A002000000000417802084F
:10061000190001000500000044A300206CA4002084
:1006200000000000100A00081A0001000E0000007F
:10063000CCA2002074A4002000000000160A0008CC
:10064000F82101000600000094A1002084A40020ED
:1006500000000000240A0008203201000A00000007
:100660009CA100208CA40020000000002538040874
:100670001500100070000000A49F002098A4002026
:1006800000000000000000002A00080060000000D8
:10069000ACA3002008A5002000000000FD370408DE
:1006A0002C0004001000000078A5002068A50020A0
:1006B00000000000ED3604082B00120024000000AA
:1006C000ACA5002088A5002000000000BD3604086D
:1006D0002920140078000000509D0020D0A50020A3
:1006E00000000000000000001002010001000000F6
:1006F00048BA002044BA0020000000002A0A00087E
:100700000D00010034000000C8D9002018E30020CB
:10071000000000001520020809020100010000008D
:1007200030D900204CE30020000000002C0A000813
:100730000400080080000000ACD8002050E3002036
:100740000000000000000000130001000400000091
:100750008CD80020D0E3002000000000300A000800
:10076000FD010100240000004CD80020D4E300204B
:10077000000000001BC50308182001003000000025
:1007800018D80020F8E3002000000000E1820208F1
:10079000061001001C00000078BA002028E40020A8
:1007A000000000004D820208FB0101000100000072
:1007B000DCD7002044E4002000000000B5820208DD
:1007C000FC01010009000000A8D6002048E4002038
:1007D00000000000C5820208F701010006000000C9
:1007E000A0D6002054E4002000000000340A0008D5
:1007F000F9010100040000009CD600205CE4002008
:1008000000000000C9C50308160215003F000000E3
:1008100094BA002060E40020000000005D8302081C
:100820003400010010000000CCD50020A0E400201E
:1008300000000000794104081102010008000000D6
:10084000A4D50020B0E40020000000003A0A00080F
:1008500012120100040000009CD50020B8E4002022
:1008600000000000420A00081220010010000000F1
:100870008CD50020BCE4002000000000460A0008DF
:10088000FA01010003000000C0CB0020CCE40020EE
:1008900000000000E97902080202010003000000E4
:1008A00070BA0020D0E4002000000000000000002A
:1008B0000C020100040000005CBA0020D4E4002017
:1008C00000000000A9780208FE01010014000000E9
:1008D000C8C50020D8E4002000000000E17802082C
:1008E00020030000000000000000000000000000E5
:1008F00000000000000000002000010100002000B6
:100900003200C800D00796001400320028004C04C2
:1009100040060005500014000F00080064000100AC
:10092000010005000A000000F40196000000C4095F
:10093000000019000000000000000000000000009E
:1009400000000000000000000000000000000000A7
:100950000000000000000000010000000000030093
:100960000000E8036400040A000114001E00900166
:1009700000000000013C0000000000000100000039
:100980000202000000000000000000000000000063
:100990000000000000000000000000000000000057
:1009A0000000000000000000000000000000000047
:1009B0000000000000000000000000000000000037
:1009C0000000010000050000AE014A015E012C019B
:1009D00064010200000001000A019A01001E0A00E1
:1009E0000000000000000000000100000005000001
:1009F00001020300000000000000000000000000F1
:100A00000000000000800700000000000000013529
:100A10000000280100007E05EA05B4053200E80365
:100A2000D00700000401F4011400000039000000A8
:100A3000080044301801000000000000000001011F
:100A40000101FFFFFFFF00000001000005465934CF
:060A50004F000008000247
:100A5600685E0C0002010000A00F0000B80B000049
:100A66000102FFFF0100000000000100E001018219
:100A7600FFFFFFFF080101FFFF000000FFFFFFFF70
:100A860001000000C57C01080000000024E90508FB
:100A9600FFFFFFFF4442002098420020D6010101DB
:100AA6000000000000000000F8FE0508000000003D
:100AB60000000000A4FE05080001010100FF2D2032
:100AC6002D2D202D2D2D2D202D2D2D2D000000001E
:100AD600000000000000000000000000002D202D96
:100AE6002D202D2D2D2D202D2D2D00000000000058
:100AF60000000000000000000000000000000000F0
:100B06000000000034FE050801000000FA000000A5
:100B1600010000000100000001010000304000203B
:100B26000000F401010000002E4000200000F40146
:100B3600010000002C4000200000F401010000002C
:100B46002A4000200000F401010000002840002097
:100B56000000F40101000000264000200000F4011E
:100B660001000000244000200000F4010100000004
:100B7600AD84010871840108E0EA050814400020EC
:100B860005320100224000206400F401010000004B
:100B9600204000206400C40901000000124000202B
:100BA600E803D0070100000010400020E803D0074A
:100BB600010000000E400020E803D00701000000FD
:100BC6000C4000201E00B80B010000001A40002057
:100BD60005000F00010000001C40002003000A0071
:100BE600010000000A4000201E00F4010100000080
:100BF6001E400020020000006CEB050808400020A3
:100C06001400640001000000164000203200E803D2
:100C160001000000064000200000C800010000009E
:100C2600DF3F002000C80100DE3F00200050010029
:100C3600DD3F0020005A0100DB3F002002000000DB
:100C460078EB0508F46B0608FC6B06084EDA002004
:100C56000100C409000000004CDA00200100C409AC
:100C6600000000004ADA00200100C409000000006C
:100C760048DA00200100C4090000000044DA002020
:100C86000100C4090000000046DA00200100C40982
:100C96000000000042DA00200100C4090000000044
:100CA60040DA00200100C40900000000753D002064
:100CB60000C80100743D002000C80100723D0020FC
:100CC6000100C80001000000703D002032003075B0
:100CD600320000006E3D0020058205006C3D0020BC
:100CE60005002C01050000006A3D0020055A05009C
:100CF600673D002000FF0100693D00200200000062
:100D06007C030020653D002003000000F0E5050897
:100D1600663D002000FF0100683D00200200000043
:100D26007C030020643D002003000000F0E5050878
:100D3600018401089183010884EB050844400020E2
:100D4600EE02CA08010000004240002000C801006F
:100D5600640000004140002000C80100640000005B
:100D6600404000200200000090EC05085E3D002097
:100D76000000803E050000005C3D002080C1803EF2
:100D860005000000563D00200083007D05000000A0
:100D9600543D002080C1803E050000004F3D0020EC
:100DA60000FF01004A3D00206400F401010000003C
:100DB600483D0020040000009CEC0508473D00204B
:100DC60002000000B0EC0508F53D00200D00000013
:100DD600BCEC0508F23D002000640100F03D002057
:100DE600320010270A000000EE3D00200D00000032
:100DF600BCEC0508ED3D00200D000000BCEC05082C
:100E0600EC3D002002000000F4EC0508AD100108DE
:100E16000000000000ED0508049600209CFF2C0150
:100E260000000000EC430020E0150C170000000055
:100E3600EE4300200200000038ED0508484000207F
:100E46000100FF7F01000000474000200200000073
:100E560044ED0508F73D00200300000054ED0508A9
:100E6600F63D00200300000054ED0508CC3F0020AD
:100E76000000E80301000000CA3F00200000E8036C
:100E860001000000C83F00200000E8030100000048
:100E9600C63F00200000E80301000000C43F002018
:100EA6000000E80301000000C23F00200000E80344
:100EB60001000000C13F002000140100C03F0020D7
:100EC6000300000064ED0508DA3F00200200000080
:100ED60074ED0508D83F00200000F4010100000071
:100EE600D63F00200000F40101000000D43F00209E
:100EF6000000F40101000000D23F00200000F401D0
:100F060001000000D03F00200000A00F01000000FB
:100F1600CE3F00200000A00F01000000F33F00209C
:100F260019640100F23F00200200000080ED050870
:100F3600F03F0020E803D0070A000000EE3F002043
:100F4600006401000A000000E33F00200064010085
:100F5600E23F002000640100EA3F00200064010037
:100F66000A000000E93F0020006401000A000000BA
:100F7600E83F0020006401000A000000ED3F002069
:100F8600006401000A000000EC3F0020006401003C
:100F96000A000000EB3F0020006401000A00000088
:100FA600E73F002001FF01000A000000E63F0020A5
:100FB60001FF01000A000000E53F002001FF0100DB
:100FC6000A000000003E00200000F40101000000BD
:100FD600FE3D00200000A00F01000000FC3D0020A7
:100FE6000000A00F01000000FA3D00200000A00F45
:100FF60001000000F83D00200000A00F01000000E5
:101006000B44002000C801000A44002000640100CF
:101016000944002000640100084400200064010027
:10102600074400200064010006440020FF08010078
:101036000544002001640100F9820108BD8201080F
:101046008CED05080E440020016401000D440020CB
:1010560001000000FCED05080C440020040000001F
:1010660004EE050804440020006401000244002048
:101076001400E8030100000000440020E803307576
:101086000A000000FE43002000C80100FD430020C6
:1010960000C80100FC43002000C80100FB430020FB
:1010A60000320100FA430020006401000A0000003B
:1010B6001C4400200000D007010000001744002057
:1010C60000C801001644002000C801001544002095
:1010D60000C801001A4400200000D00701000000EB
:1010E6001444002000C801001344002000C8010079
:1010F6001244002000C80100184400200000D00758
:10110600010000001144002000C801001044002026
:1011160000C801000F44002000C8010000000000C4
:10112600A180010818EE0508E93D0020005A0100DB
:10113600EA3D00203B000000B4EE0508E83D002033
:1011460000C80100E63D0020E803D00701000000CA
:101156004655525946344F5344000000633D002023
:1011660000030100623D002000030100C57F010865
:10117600797F0108A4EF0508357F0108E97E01089B
:1011860030F00508118001085DA00108B0F00508DF
:10119600603D00200103010015850108E98401086E
:1011A600DCF30508797E0108397E01084CF4050850
:1011B600B780010879A00108E8F40508C1B4010860
:1011C6000000000090F5050835A5010841850108D5
:1011D6002CF605080981010800000000ACF6050898
:1011E600E18101088D81010810F70508798201085F
:1011F60035820108ACF705081D1B02083583010876
:1012060038F8050805400020010601005181010853
:101216001D81010834F90508631A020839A101087D
:10122600A4F90508651B0208F1A10108D8FA05080A
:10123600044000200103010065800108298001089F
:10124600ACFB0508BD1B0208000000001CFC0508DD
:10125600B97E01082DA0010880FC050800000000E9
:10126600000000000CFD05086983010869A2010859
:101276008CFD0508423D002088136F170100000011
:10128600443D002088136F170000000092DA00200A
:10129600000000000000000090DA002000000000BE
:1012A600000000008EDA00200000000000000000B0
:1012B6008CDA002000000000000000008ADA00201E
:1012C600000000000000000088DA00200000000096
:1012D60000000000FC0D00200000000000000000DF
:1012E600183D00200300000040FF0508403D002097
:1012F60088136F17010000004E96002088136F17A1
:10130600000000007D7D01080000000050FF050878
:10131600F943002001000000A4FF050850960020B4
:1013260001000000B0FF05084696002002000000FC
:10133600B8FF05080000000000000000C4FF050813
:10134600697D01080000000060000608000000003A
:1013560000000000B40006080000000000000000C5
:1013660024010608463D0020020000005C01060834
:101376004A960020E0150C1700000000000000004F
:10138600B44C00200800000000000000A44C00201F
:1013960008000000F58C030823630308898C030802
:1013A600000000001D60030881820308CD8B03083E
:1013B600058203080000000000000000DD5F03084E
:1013C600A95F03089B5F0308B57F0308D17F030865
:1013D600997F03087D7F0308637F0308AD8C0308AC
:1013E60001630308CF8B030800000000F55F0308C4
:1013F60007820308A18B030873810308000000001D
:1014060000000000E95F03081A0300000000000066
:1014160000000000000000000000000000000000C6
:10142600000000000403090412010002000000404D
:1014360083042057000201020301000015840208FC
:1014460045790208417902083D7902082584020897
:1014560039790208357902086C0B06086188030899
:10146600E16203084D890308000000000000000047
:10147600798B0308898A0308000000000000000039
:1014860000000000D15F0308DD790208D179020867
:101496005589020871890208897902083989020882
:1014A6001D8902081F0000001C0000001F0000002C
:1014B6001E0000001F0000001E0000001F000000AC
:1014C6001F0000001E0000001F0000001E0000009C
:1014D6001F0000000068214CFF01FF000000803F54
:1014E6000000000000000000000000005547020850
:1014F600000000000000000000000000FFFFFFFFEA
:10150600FF000000401B0608040309041201000244
:10151600EF0201408304563200020102030100007B
:101526001201000202020040830440570002010239
:101536000301000009022000010104C03209040071
:101546000002080650050705810240000007050154
:101556000240000009026400030100C032090400D1
:1015660000010300000009211101000122260007E5
:1015760005830308000A080B0102020201000904A0
:1015860001000102020100052400100105240100EA
:10159600020424020205240601020705820308004C
:1015A600FF09040200020A000000070501024000CC
:1015B600000705810240000009024300020100C045
:1015C6003209040000010202010005240010010591
:1015D60024010001042402020524060001070582F5
:1015E600030800FF09040100020A000000070501C4
:1015F600024000000705810240000000FF000000D5
:1016060000FF0000000000000000AA5507010000CE
:1016160001AA550501000000681C0608FF1FFF1FF0
:1016260005010905A101A1000501093009310932A9
:10163600093309350934094009381581257F7508AC
:1016460095088102C0C0000009022200010100E0E5
:101656003209040000010301020009211101000101
:101666002226000705830308000A00000000000088
:10167600010203040102030406070809ED8D0308AD
:10168600118D03089183030853600308ED63030873
:10169600636003087F6003082D6003081F6003086A
:1016A6000000000000000000AA550B010000AA552A
:1016B60005010000AA550902000000AA5503009F73
:1016C60001000000C01200009C99002000000000EC
:1016D600C099002000000000FFFF0000FFFFFFFF91
:1016E6003CCE0608000008020503030000000000C7
:1016F60044CE0608010008020504030000000000AD
:10170600448C06080200FE010110030000000000E0
:1017160084700608030014020003000000000000A5
:101726004CCE060804001F0202000800000000005C
:1017360054CE060805001F02020108000000000042
:10174600006002401060024000000000000000003F
:10175600000B000000000000000000000000000078
:101766000060024028600240010000000000000006
:10177600060C000000000000000000000000000051
:1017860000600240406002400200000000000000CD
:10179600100D000000000000000000000000000026
:1017A6000060024058600240030000000000000094
:1017B600160E0000000000000000000000000000FF
:1017C600006002407060024004000000000000005B
:1017D600200F0000000000000000000000000000D4
:1017E6000060024088600240050000000000000022
:1017F60026100000000000000000000000000000AD
:1018060000600240A06002400600000000000000E8
:101816003011000000000000000000000000000081
:1018260000600240B86002400700000000000000AF
:10183600362F00000000000000000000000000003D
:101846000064024010640240000000000000000036
:10185600003800000000000000000000000000004A
:1018660000640240286402400100000000000000FD
:101876000639000000000000000000000000000023
:1018860000640240406402400200000000000000C4
:10189600103A0000000000000000000000000000F8
:1018A600006402405864024003000000000000008B
:1018B600163B0000000000000000000000000000D1
:1018C6000064024070640240040000000000000052
:1018D600203C0000000000000000000000000000A6
:1018E6000064024088640240050000000000000019
:1018F6002644000000000000000000000000000078
:1019060000640240A06402400600000000000000DF
:10191600304500000000000000000000000000004C
:1019260000640240B86402400700000000000000A6
:101936003646000000000000000000000000000025
:1019460001000000FFFFFFFF0000803F00000000D5
:1019560000000000000000000000803F00000000C2
:101966000000000000000000000000000000000071
:101976000000000000000000000000000000000061
:101986000000803F00000000000000000000000092
:10199600010000000000803F080000000000040174
:1019A6000000000000000002100000000700000018
:1019B6007D000000995F0308975F0308955F0308A1
:1019C6008F5F03088D5F0308935F0308915F030829
:1019D60001000000D8CE0608586A0608000000007C
:1019E600B11C0208A08601000400000000000000EF
:1019F60000000000000000000000000000000000E1
:101A060000000000000000000000000000000000D0
:101A160000000000D8CE060868D3060800000000C3
:101A260045800008E80300000400000000000000F4
:101A360000000000000000000000000000000000A0
:101A46000000000000000000000000000000000090
:101A560000000000687406087C6E0608000000009E
:101A6600E5F402087D00000006000000000000000A
:101A76000000000000000000000000000000000060
:101A86000000000000000000000000000000000050
:101A96000000000030CE0608000000000000000034
:101AA6003DF10008E803000003000000000000000C
:101AB6000000000000000000000000000000000020
:101AC6000000000000000000000000000000000010
:101AD6000000000070D306080000000000000000AF
:101AE60069C704081027000003000000000000007A
:101AF60000000000000000000000000000000000E0
:101B060000000000000000000000000000000000CF
:101B16000000000048CE0608000000002D3404082E
:101B2600F98400085F760000050000000000000050
:101B3600000000000000000000000000000000009F
:101B4600000000000000000000000000000000008F
:101B560000000000ECD106080000000000000000B4
:101B660019FC00081027000001000000000000001A
:101B7600000000000000000000000000000000005F
:101B8600000000000000000000000000000000004F
:101B9600000000007CD306080000000000000000E2
:101BA60049800008E803000005000000000000006E
:101BB600000000000000000000000000000000001F
:101BC600000000000000000000000000000000000F
:101BD6000000000088D30608000000000000000096
:101BE600E91E0208204E000003000000000000006D
:101BF60000000000000000000000000000000000DF
:101C060000000000000000000000000000000000CE
:101C16000000000098D30608000000000000000045
:101C2600ED1C0208204E000003000000000000002A
:101C3600000000000000000000000000000000009E
:101C4600000000000000000000000000000000008E
:101C560000000000A8D306080000000000000000F5
:101C6600E9950008400D0300030000000000000095
:101C7600000000000000000000000000000000005E
:101C8600000000000000000000000000000000004E
:101C9600000000008C7F0608000000000000000025
:101CA6004D4502081027000001000000000000005A
:101CB600000000000000000000000000000000001E
:101CC600000000000000000000000000000000000E
:101CD6000000000048670608000000000000000041
:101CE600B5300108102700000300000000000000C6
:101CF60000000000000000000000000000000000DE
:101D060000000000000000000000000000000000CD
:101D160000000000B8D30608000000000000000024
:101D2600F9130208A086010001000000000000006F
:101D3600000000000000000000000000000000009D
:101D4600000000000000000000000000000000008D
:101D560000000000E471060800000000000000001A
:101D66008583000850C30000010000000000000049
:101D7600000000000000000000000000000000005D
:101D8600000000000000000000000000000000004D
:101D960000000000906F0608000000000000000030
:101DA60081800008A861000001000000000000001A
:101DB600000000000000000000000000000000001D
:101DC600000000000000000000000000000000000D
:101DD60000000000C0D3060800000000000000005C
:101DE6004D790108A08601000100000000000000F6
:101DF60000000000000000000000000000000000DD
:101E060000000000000000000000000000000000CC
:101E160000000000AC7F0608000000000000000083
:101E260061BD0008A00F00000100000000000000D6
:101E3600000000000000000000000000000000009C
:101E4600000000000000000000000000000000008C
:101E560000000000CCD306080000000000000000CF
:101E66004D7401081027000001000000000000006A
:101E7600000000000000000000000000000000005C
:101E8600000000000000000000000000000000004C
:101E960000000000147C060800000000000000009E
:101EA6003D5101081A410000010000000000000039
:101EB600000000000000000000000000000000001C
:101EC600000000000000000000000000000000000C
:101ED60000000000506F060800000000000000002F
:101EE6006D660308102700000100000000000000D6
:101EF60000000000000000000000000000000000DC
:101F060000000000000000000000000000000000CB
:101F1600000000006C6A06080000000000000000D7
:101F2600F1BC01081A410000010000000000000099
:101F3600000000000000000000000000000000009B
:101F4600000000000000000000000000000000008B
:101F560000000000D8D306080000000000000000C2
:101F6600E16D0308400D03000000000000000000C2
:101F7600000000000000000000000000000000005B
:101F8600000000000000000000000000000000004B
:101F960000000000E0D3060800000000000000007A
:101FA60001800008400D0300000000000000000052
:101FB600000000000000000000000000000000001B
:101FC600000000000000000000000000000000000B
:101FD60000000000E8D30608000000000000000032
:101FE600395F010850C30000030000000000000034
:101FF60000000000000000000000000000000000DB
:1020060000000000000000000000000000000000CA
:1020160000000000F4D306080000000000000000E5
:102026000124020840420F000000000000000000EA
:10203600000000000000000000000000000000009A
:10204600000000000000000000000000000000008A
:102056000000000000D40608000000000000000098
:102066008521020850C300000000000000000000A7
:10207600000000000000000000000000000000005A
:10208600000000000000000000000000000000004A
:08209600000000000000803F83
:082800000000000000000000D0
:108000000C4B1B78DB0700D570470B4A1368002B1D
:10801000FAD04FF47A7101FB03F39842F4D3074B83
:108020001B781BB9064B99681B690B600023136012
:10803000704700BF309300201C7E0020087E002087
:1080400064780020704700BF70B50C4C23689BB16A
:108050005A68821A002A0FDB0546002603E05A6898
:10806000AA1A002A08DB9A681E73226018461A684A
:1080700090472368002BF2D170BD00BFF07800203C
:108080002DE9F047A94D2C682DED028B041B46F21B
:10809000A7139C4282B004D802B0BDEC028BBDE8AD
:1080A000F087A34B28601E6816F0040140F08D8015
:1080B0000F4616F0200344D19FED9E8A9C46184639
:1080C0009D4E9E4A367892F8008016F0010671D1D6
:1080D000B8F1000F00D016706A6901922A69BF1AC0
:1080E000019AA0EB0208002B3ED151B12B7E012B4F
:1080F00007D8934B214638461F6045F0F9FF914B56
:108100001880914B1B780E2BC6D1DFED907A8D4BEA
:108110008F49188828EE278A0022BDEEC88A1346A8
:1081200018EE104A68F30F0364F30F0267F31F425F
:1081300060F31F43C1E9002302B0BDEC028BBDE830
:10814000F087844B1B7813F0020300F08E80824A84
:10815000824E538A9068B6F900C0002B40F0CB8065
:108160009FED748A0123ABE72B7E002972D0002B90
:1081700040F0BD80002E00F0D680F7EE007A37EE9A
:10818000C87A07EE907AF8EEE77A67EE877A07EE1C
:10819000108AB8EEC77AE7EE087AFDEEE77A17EEB6
:1081A000903A674A21463846136045F0A1FF654B77
:1081B0001880A6E7B8F1000F8ED14FF0010EC5E987
:1081C000047082F800E047468DE7DFF8ACA1DFF8E5
:1081D000AC819AF80630B8F800906F68013BB7FBA5
:1081E000F3F7B9F1000F45D05D4A9FED5E0A1368C1
:1081F000002B1946B8BFD91DA3EBE1031F44002F84
:108200003B46B8BFFB1DDB1007EE903AF8EEE77A6D
:10821000176027EE800A23F09FF8DFED537A20EEF7
:10822000270A23F0DFF8F7EE007A77EEC07A9FEDA9
:108230004F0AEB6867EE807A9F42FDEEE77AC5ED64
:10824000027A6AD009F1FF390021EF60A8F80090A6
:108250000F462EE713F0FD0F7FF453AF384A394B2A
:10826000C2F80080A3F800C04BE79FED328A9C461D
:10827000184625E707EE907A9FED3A0ADFF800816D
:10828000F8EE677AB7EE008A27EE800A23F064F8EA
:10829000DFED357A20EE270A23F0A4F8DFED337AFC
:1082A00038EE400A20EE270A53F02CFCBAF80830CA
:1082B000DFED2F6A07EE103AAB68C01AB8EEC77A46
:1082C00007EE900AA7EE668AB8EEE70AD8ED0D7AB7
:1082D000F8EEE77A20EE080A67EEA67AA7EE270AFC
:1082E00053F010FC01210746C8F83400E1E6022BE8
:1082F0007FF4FDAEB2E707EE903ADFED146A9FED32
:108300001D7AF8EEE77A86EEA78AB4EEC78AF1EE18
:1083100010FA88BFB0EE478A24E700231946A8F870
:1083200000301F46C5E643463BE700BFD01700209C
:108330000C8900209A99993E30930020C433002084
:10834000AC960020BA93002061BA00200000C84219
:1083500064BA00206C930020B0D900205C3100206A
:10836000880100200894253741D3423ED048874AEF
:108370006F12833A6666663F8C9900207E780020F3
:1083800058CB0020534B1B685B0700D470472DE986
:10839000F04F514D514C2A782379372A08BF504A63
:1083A00083B008BF1380042B76D8DFE803F06D6339
:1083B0005B4F03004B4FFB6A38469847002849D073
:1083C000494E3B6B06F11C0106F120009847474BD4
:1083D000D6F804809879D6E909A2D6E9073B0AF1D4
:1083E0000109511C814508BF4FF000090329C7F856
:1083F0003CB0BB635DD03E48B16296F82C1040F8AB
:1084000022B000295DD1584606EB8A0A06EB8902A4
:10841000CAF83000397CD2F830C02A78C6F82490E7
:108420000029A8EB0C080CBF052102214044372A83
:108430007060217104D12A4A5380A2F804B0D08020
:108440007B8A002B42D103B0BDE8F08F2548836AB8
:10845000984748BB4FF47A73264A1268136103B0F9
:10846000BDE8F08F1F4D6B6A284698470322AB8A00
:108470002271E6E71B48036A98470028EAD00223E6
:1084800023714FF47A73E7E71648C36998470028C9
:10849000E0D001232371DDE7124DAB6928469847F0
:1084A00000226B8A2271CCE7042323714FF47A7384
:1084B000D2E70F4A0121C2F808B0002286F82C103A
:1084C000B262019350F052FD019B9DE70A2BB8BFA9
:1084D0000A23C1E70C89002061BA0020880100202E
:1084E00064BA002058CB0020D01700208C990020BF
:1084F000A0D80020701200102DE9F04FE04D2DEDB6
:10850000068B2B7893B0044643B1DFF8BCA3DAF8AE
:1085100010305046984780F001002870D94B1A78E7
:10852000002A00F0FE81D84ED84896F8F050D6F8D0
:10853000F41004F5EC425F32026000221A70002D44
:1085400000F0F4818C4202D9013D86F8F0502046BB
:108550002AF03EFA002800F0E481D6F88031C6F80F
:108560008041E41A47F230539C42A8BF1C46C84DD4
:10857000C84A2F78C84BDFF85483B4F57A7FB8BF68
:108580004FF47A741480012217401A7000F062824E
:10859000C24AB8F906301268D1898B4280F21F8234
:1085A000BF4A4FF07E511160BE4ADFF824C392F9F2
:1085B0000410BCF81250B8F90090107892F801E05D
:1085C000B94CA9EB0502002914BF01214FF0FF317E
:1085D000002AB8BF5242B2F5FA7FA8BF4FF4FA7230
:1085E0008242C5BF121A07EE902ADFEDB07AF8EE8C
:1085F000E77A4D45B8F90290C4ED007AA9EB05027F
:10860000C4BFF1EE677AC4ED007A002AB8BF5242C7
:10861000B2F5FA7FA8BF4FF4FA729042BABF121AAD
:1086200007EE902ADFEDA17AB8F90400B8BFF8EEA2
:10863000E77A4D45A0EB0502C4ED017AC4BFF1EE27
:10864000677AC4ED017A002AB8BF5242B2F5FA7FC8
:10865000A8BF4FF4FA72964580F2D981A2EB0E0EB4
:1086600001FB0EFE07EE90EAF8EEE77A904AC4EDC1
:10867000027A85421168C4BFF1EE677AC4ED027ACE
:1086800011F4805100F09781B3F5FA6FA8BF4FF451
:10869000FA63B3F57A7FB8BF4FF47A73A3F57A70B3
:1086A000844B1A78002A40F09081DFF82882DFF8A6
:1086B00028C288FB0023C217C2EB631303F1010E2B
:1086C0006FF063023CF91EE03CF913C002FB0303A8
:1086D000AEEB0C0003FB00F388FB0302DB17C3EBDC
:1086E000621363441BB207EE903AB8EEE78A84ED5A
:1086F000038A002940F083826F4B1B885A0640F1A1
:108700000C8140F603026D49D4ED011A91ED010A86
:10871000D1ED033AD1ED028AD1ED005A94ED002A51
:108720001340674A08BFD4ED022A92ED019A92EDF8
:10873000026AD2ED030A92ED004A18BFDFED5B2A10
:10874000604A30EE635A39EE461A74EE207A25EE0E
:10875000011A75EEE86A35EEA8AA74EE609A66EE24
:10876000A76AB0EE413AAAEE293AB0EE665A30EE68
:10877000237A79EE067AAAEE295AA7EE273AA7EECF
:10878000675AF0EE414AD7EE274A33EE263AB6EE64
:10879000008A75EE80AA28EE433A35EE415A34EE4F
:1087A000091AB0EE647AEAEE694AAAEE813A77EEE7
:1087B000667A36EE601A73EEE8AA25EE085AEAEEFB
:1087C000297AAAEE815A74EEA64A63EE036A34EE61
:1087D000494A73EEA83A64EE884A75EEC05A36EEFE
:1087E000206A67EE887AB0EE667AE3EE844A95EE08
:1087F000057AE5EE056AE5EE867AB1EE648AF0EE7A
:10880000665AF0EE476AB1EE674AE8EE246A63EE14
:10881000270A67EEA43AE4EE275AB1EE450AB0EE15
:10882000609AB0EE631AA4EE277A23EE244AE7EEAC
:10883000A76AA5EE249AA0EE031AE8EE245AB0EE39
:10884000448A31EEA16AE0EE240AA5EE278A66EE9C
:10885000A16A72EE028AE5EE033A61EE211A26EE73
:10886000096AA4EEA47AA0EE274AA2EE256AE8EEF1
:10887000A06AE2EE081A73EEA33A27EE227A2DE000
:10888000149B00201C9B0020D0170020189B002068
:108890003093002044A1002028A40020C09600208E
:1088A0009CA0002044A3002078930020000000003A
:1088B0008CD80020CC4B0020B0930020140C00205A
:1088C00080100020B810002070D8002040DA00206E
:1088D00018D800201F85EB5110A4002034EE044A64
:1088E000F0EE005AE2EEA36AA2EE846AA1EEA57A47
:1088F000C6ED626AC4ED016A86ED616A84ED006AC4
:1089000086ED637A82ED005A82ED013AC2ED027A79
:10891000C2ED034A002B00F09A80002F7AD125F097
:10892000B1FE13B0BDEC068BBDE8F08F8C427FF634
:108930000EAECC4B1B78002B00F0B681DFF85CA3A9
:10894000DFF85C83DFF85C93574606F1F80B28E00C
:1089500018F805109847032D03462ADCC8B109EB27
:10896000850339F825105A88401A4FF47A7303FBAF
:1089700000F0521A40F6CA0390FBF2F000F57A704C
:108980009842A8BF184640F2EE239842B8BF184656
:1089900000B2B44B2BF8020B1B7801359D4280F2DC
:1089A0008381072D3846DAF80830D1DDE9B29847DF
:1089B000034618B2EDE7BCF81420934237DAAA4B0D
:1089C0001A780846002A3FF470AE5B78A74A00FB8D
:1089D00003F382FB0320DB17C3EB601065E6B3F5FE
:1089E000FA6F127B9FEDA27ABFBF581A4243C1F5BE
:1089F000FA6192FBF1F2C2F1640207EE902AF8EEFE
:108A0000E77A9C4A67EE877AC2ED007ACCE5DFED23
:108A10009A7A2BE6994A9A4B1178186801F001016D
:108A200036F0F2FE13B0BDEC068BBDE8F08FB3F567
:108A3000FA6FD4BFC2EB0303C2F5FA634FF47A7046
:108A4000C2F5FA6200FB03F3B3FBF2F028E684ED13
:108A5000027A62E7B8F90090B8F902E0B8F90CC000
:108A6000B8F90440B8F90800B8F90610B8F90E20B2
:108A7000B8F90A30DFF820A2B9F5FA6FA8BF4FF4B1
:108A8000FA69BEF5FA6FA8BF4FF4FA6EBCF5FA6F3B
:108A9000A8BF4FF4FA6CB4F5FA6FA8BF4FF4FA64AC
:108AA000B0F5FA6FA8BF4FF4FA60B9F57A7FB8BF96
:108AB0004FF47A79BEF57A7FB8BF4FF47A7EBCF571
:108AC0007A7FB8BF4FF47A7CB4F57A7FB8BF4FF4A1
:108AD0007A74B0F57A7FB8BF4FF47A70B1F5FA6F57
:108AE000A8BF4FF4FA61B1F57A7FB8BF4FF47A713D
:108AF000B2F5FA6FA8BF4FF4FA62B2F57A7FB8BF49
:108B00004FF47A72B3F5FA6FA8BF4FF4FA63B3F576
:108B10007A7FA0F57A70B8BF4FF47A73C0EBC010BB
:108B2000A9F57A79AEF57A7EACF57A7CA4F57A74FB
:108B3000A1F57A71A2F57A724000A3F57A73AAFBC7
:108B400000B0C9EBC919CEEBCE1ECCEBCC1CC4EBEC
:108B5000C414C1EBC111C2EBC212C3EBC3135B005F
:108B600080094FEA49094FEA4E0E4FEA4C0C640067
:108B700049005200AAFB09B9AAFB0EBEAAFB0CBC15
:108B8000AAFB04B4AAFB01B1AAFB02B2AAFB033AF6
:108B9000A0F17F033B488DF8443090F812314FEA42
:108BA00099194FEA9E1E4FEA9C1CA4098909920953
:108BB0004FEA9A1AA9F17F09CEF17F0EACF17F0C32
:108BC0007F3C7F397F3AAAF17F0A032B8DF84090D2
:108BD0008DF841E08DF842C08DF843408DF8451086
:108BE0008DF846208DF847A07FF4D2AC082310AA58
:108BF00083212FF09BFA2F7807F00107C8E4224B5E
:108C0000DB78002B7FF478AD204B214893F80C8063
:108C1000152121F0F3FAB8F1000F40F03981002856
:108C20003FF46AADDFED1B7A1B4978EE677AC5F534
:108C3000FA63FDEEE77A1AB217EE903A1BB21B0305
:108C400081FB0301DB17C3EBA11302FB03F343F327
:108C50000F332B4407EE903AF8EEE77AC4ED037A2F
:108C60004AE500BF7C9E0020CC4B00201F85EB51C5
:108C70000AD7233C9CA00020000000003FC5002034
:108C800040C5002000CC002034930020CCA200205E
:108C90006C46002000007A44D34D621070D800204A
:108CA00018D8002078A50020BB4A1178BB4AD2F81A
:108CB0000090002940F0E7800A46B9480078039008
:108CC000282804D1B74DB8482D7845800180B74990
:108CD00001270F70002B00F0AF81B54905910D7889
:108CE0000495B44DDFF8E4E2E98B0091298CDFF8BC
:108CF00000830191698A049D0A919EF80C100D91E0
:108D0000A8FB05E1AC48DFF8C8C20078DCF800C079
:108D1000DFF8E0A2DFF8BCB20893490801EB41019B
:108D2000691AC9B203F1FF3801380691490002916E
:108D3000B8F1030FC1B20CF480504FF000050C974E
:108D400007910B90A8BF4FF003080B460994002A27
:108D500000F0C3809949009831F8151081424FEA1C
:108D60004507C0F0BA800198814200F2B68009F54B
:108D700096704AF82500012B09B240F2E7802BF8E3
:108D8000071001354545E2DDDDE908349D422ADA68
:108D90008B49089405EB450701EB4707DFF834B230
:108DA000079C24390291002A00F0B58002990098AE
:108DB00031F8151088424FEA450800F2AC8001985E
:108DC0008842C0F0A88009F596704AF82500012C69
:108DD00009B240F211812BF808100135AB4207F1BE
:108DE0000607E0D1089C714B1B78002B40F02681D0
:108DF0006C4B012204201A701BF0FAFC7148674B7F
:108E0000C1681B68426803615B1A934202D9002360
:108E100080F825306C4B1F78614B1B780393002F33
:108E200000F02481694A6A4B117B1B68614A03F494
:108E30008053B2F81EB0B2F812A0002900F04381AE
:108E40006449654D83B1AAE1022A40F02481427849
:108E500002EB820202EB820202F2EE2201339F4217
:108E600021F8022B00F0028115F8132005EB4300D6
:108E7000002AE9D1DAB2022A40F25D81032A40F0E9
:108E80000A815A46EAE7474A127882F0010214E75B
:108E9000DFED527A524A38EE678ABDEEC88A18EE84
:108EA000103A1BB21B0382FB0312DB17C3EBA213A6
:108EB000002800F02A81C5F57A7212B203FB02F392
:108EC00043F30F332B4407EE903A464BF8EEE77A24
:108ED0000122C4ED037A1A700EE45AF82510A9EBAA
:108EE00001010029FFF64DAF3B4810F815106F0047
:108EF0003844002900F0D180022940F0C98041782F
:108F000001EB810101EB810101F2EE2127484FF0D5
:108F1000000404702FE75AF82510A9EB010100297D
:108F2000FFF65BAF2C4810F815104FEA4508404497
:108F3000002900F0BD80022940F0A780417801EBB4
:108F4000810101EB810101F2EE2140E71C48029C06
:108F500096F864E107EB050C00EB4C000153BEF101
:108F6000000F06D1049C022C7FF609AF0C9986F8FD
:108F700064114188B0F804E0114830F81C007144D5
:108F8000014408B2184981FB0041184CA1EBE07183
:108F9000E05309B2F3E600BF6A20002074C5002048
:108FA00061BA00207810002064BA002092380020B6
:108FB000049D002018D8002070D80020C818002078
:108FC000EC180020349300207C9E0020CCA20020CE
:108FD0008CD8002040DA0020ACA5002000007A44A4
:108FE000D34D621010790020565555553819002080
:108FF000ABAAAAAA089D0020069896F864C127F893
:109000001010BCF1000F06D1049802287FF6E3AEE1
:10901000012186F86411B7F800C07988B8886144E6
:10902000014408B2824981FB001C824921F80800F2
:10903000ACEBE07109B2CEE67F4B05937F48062189
:1090400021F0DCF800287FF4D3AE7D4A7D4B106917
:109050001B689168D3601B1A8B4207D97A490B6849
:10906000012023F004030B6082F82500039B282BCA
:1090700005D1DFF8DC81754BB8F80620DA80059A57
:10908000137801331370FFF762BA3BF808109EE6BD
:109090003BF807103AE70A88E0E6E9B2022948D926
:1090A0000329F5D10B99002940F09D8000992DE707
:1090B000E9B202293BD90329E7D10B99002940F0F5
:1090C000A480009983E6002B39D16149614D0DE000
:1090D000022A18D1427802EB820202EB820202F2EB
:1090E000EE2201339F4221F8022BBFD015F8132046
:1090F00005EB4300002AEBD1DAB2022A1DD9032A7C
:1091000001D15A46EDE70A88EBE7C5F5FA6212B2DB
:1091100003FB02F343F30F332B4407EE903A4E4B1D
:10912000F8EEE77A1870C4ED037AFFF7E5BA0A990A
:109130004DE60A99EAE6524690E65246D1E7DFF854
:109140001091444D3D4B88460EE0022A24D14878C8
:1091500000EB800000EB800000F2EE2008F1010837
:10916000B84529F8020B81D015F8182005EB480105
:10917000002AEAD15FFA88F2022A30D9032A4FF096
:109180001501184608D1009321F038F8009B0028FB
:109190000CBF50465846E1E7B9F80000DEE700236F
:1091A0000EE0022A19D1427802EB820202EB82021F
:1091B00002F2EE2201339F4221F8022B3FF456AF18
:1091C00015F8132005EB4300002AEAD1DAB2022A8F
:1091D00007D9032A01D15A46ECE70A88EAE7504644
:1091E000BCE75246E6E715211448CDE90E2321F0ED
:1091F00005F8DDE90E2300287FF458AF0D9900989B
:1092000000290A9918BF014680E615210B480993E9
:10921000079220F0F3FF079A099B00287FF451AFD3
:109220000D990A980029009908BF0146CFE500BFB3
:109230005655555538190020049D00206C460020D5
:109240003493002074C50020B496002064BA002036
:1092500040DA0020ACA5002010790020038A2DE917
:10926000F047B0F80C9019EA030928D00E460546DD
:109270004FF000474FF00008B9FA89F327FA03F2DC
:10928000D24391B21B3B09EA02092982042B13D86D
:10929000DFE803F0322920170300736A002B34D172
:1092A000EB6A1FFA83FA346A34B1236820465146C8
:1092B00098476468002CF8D1B9F1000FDCD1BDE803
:1092C000F0873068696B036889B29847B9F1000F7D
:1092D000D2D1F4E77068A96B036889B29847B9F1F5
:1092E000000FC9D1EBE7B068E96B036889B2984712
:1092F000B9F1000FC0D1E2E7F068296C036889B2C8
:109300009847B9F1000FB7D1D9E703F1FF3A1FFA37
:109310008AFAC6F82480C6E7744B75482DE9F041F7
:1093200070220124734E1C70002153F031FE724AEA
:109330007249734D002330460B60136019F0E0F959
:109340002146204619F020FA2146062019F01CFA81
:109350006F7A6C4A6C4B128E93FBF2F3391C18BF78
:1093600001210820C6F8903119F00EFA95F80A800C
:1093700018F100014FF0090018BF012119F004FA9B
:10938000AB7B002B79D0614C002F40F0818018F12D
:10939000000118BF01215E4D0A2019F0F5F92B6874
:1093A000D80777D4990700F191800121052019F0A1
:1093B000EBF9584B0720197819F0E6F901210B2039
:1093C00019F0E2F921680C20C1F3C01119F0DCF9A1
:1093D00029680D20C1F3C00119F0D6F929680E20C3
:1093E000C1F3800119F0D0F92B685A0756BF2168E4
:1093F0000121C1F3C0110F2019F0C6F92168102016
:10940000C1F3404119F0C0F921684B054FD4C1F3B5
:109410000041122019F0B8F9216811F4802104D01C
:109420003D4B1968003118BF0121132019F0ACF928
:1094300021681420C1F3C06119F0A6F90121192097
:1094400019F0A2F901211A2019F09EF90121152025
:1094500019F09AF90121162019F096F90121172027
:1094600019F092F92D4B196800314FF0180018BF10
:109470000121BDE8F04119F087B9EB7B234C002BAB
:1094800082D1216811F4802185D0002F3FF47FAF75
:10949000012180E7224B1B680A2BB8BF0A23012158
:1094A0000220C6F8903019F06FF92B687AE7012195
:1094B000112019F069F91B4B21685B78083B012BDF
:1094C0009CBF4FF4FA63C6F85034A0E70121032093
:1094D00019F05AF9144BDB6C0A2BB8BF0A2301218F
:1094E0000420C6F8D03019F04FF95EE7100D0010D7
:1094F000E42D00100C110020E02D00100C0D0010C8
:1095000088930020C8D9002040420F008CD800204A
:109510000C8900209081002038310020D8350020AF
:109520004804001070D800208C110010034B012259
:109530004FF400101A701BF05BB900BF8844002084
:10954000022838B5044637D81E4A1F491F4D0C70F3
:1095500000EB401300EB430302EB430318462B6080
:109560003FF020FE42F028FE2B689FED195A93F839
:109570007E20DFED185A9FED186A184906EE902AF2
:1095800093F8822093F8803007EE102A07EE903A85
:10959000F8EEE66AB8EEC77AF8EEE77A104A114BB1
:1095A00066EE856A27EE257A67EE867AC1ED006A57
:1095B00082ED007AC3ED007A601CC0B2BDE838408D
:1095C0001BF0B0B8043E00208CD50020BC960020D3
:1095D0005655D53F6F12833A17B7D138841600100D
:1095E000881600108C1600102DE9F04F9C4B9D4DF5
:1095F0001B7895F80090DB0785B0804641D59A4CE2
:109600009A4EB9F1010F6AD0C0F08D80B9F1020F06
:109610002BD0E37B83B1A38973B1954B1B785BB1EE
:109620002BF0FCFD002800F01881237C83422CBF26
:1096300001220022327000E03278217A632908D8B2
:109640008C48B9F1020F037800F08980002B40F0BC
:1096500098808949A37B914538BF914681F8009055
:10966000002B53D105B0BDE8F08F844A844B12889B
:109670001B889A42CDD9834A834B1268C3F8902144
:1096800068E07E4F784C3A88A9F10303012B40F241
:10969000A9807B88D31A002BB8BF5B42142B07DC50
:1096A000E388934200F28B8021889142C0F087804A
:1096B0006E4E764B1B78022BA3D17A883B886C497F
:1096C0009B1A002BB8BF5B42142B714A097891801A
:1096D000CCBF00230123B9F1010FD38094D1684B93
:1096E000664A1B88617C12885B1A9A4253DD694B7B
:1096F0001B88934238BF4FF00009624A38BF85F893
:109700000090614B1268C3F8902182E7B9F1010F14
:1097100000F09D80B9F1020FA4D1072005B0BDE88B
:10972000F04F1AF0D1BE5B4B544A1B88617C128803
:109730005B1A9A42534AE4DC5349E37D1268D1F83C
:10974000901103EB8303521A03EB8303B2EB830FF5
:10975000FFF65FAF4FF0010985F8009059E783B934
:109760000125C0F804800570C1F164014A4D03FB76
:1097700001F385FB0351DB17A3EBA1536433437063
:1097800067E74368454DA8EB0303AB42C8BF417090
:109790003FF75FAFE8E73B4A3B49237E1268D1F8C9
:1097A000901103EB8303521A03EB8303B2EB830F95
:1097B000FFF62FAF4FF0020985F8009029E7B2EBD2
:1097C000430F2A4E3FF775AF294832492C4A0023F0
:1097D0004FF0030986F8009085F8009003700B8025
:1097E000138066E7E388934229D82188914226D3E3
:1097F0007B88D31A002BB8BF5B42142B3FF758AFBE
:109800001A4E237D4FF0000E86F800E085F800E048
:10981000002B45D0164AF1461370A1881D4AB4F8B2
:1098200002C017489BB211FB03F111801CFB03F32C
:10983000104A0380642100235170536039E7B2EB72
:10984000430FD5DCB9F1030F3FF432AF21E7082015
:1098500005B0BDE8F04F1AF037BE02223270ECE6D8
:1098600030930020C64B002088930020D44B00206A
:1098700076930020CC4B00207220002070930020B3
:10988000CA4B002074C50020D017002061BA002008
:1098900064BA0020C84B00206BCA5F6B7F969800AB
:1098A000304923880968B2FBF3F20132082A91F9A2
:1098B0007210DFF8BC90A8BF0822D3B2914289F899
:1098C00000304AD0002948D02749DFF8A8C091F8D5
:1098D00000B00BF10101ACFB01A0400800EB40001F
:1098E000081A5845029038D020494FF0860A0AFBE2
:1098F000001E9EF972E0964527D0CDE900CA039379
:109900004FF0FF3A014603E09CF972E0964527D0FC
:1099100001F1010C0099A1FB0C314908019B01EBFD
:109920004101ACEB01019C46104BBAF1000F0CFB5E
:10993000013C03DABEF1000F08BF824659450846D4
:10994000E2D1039B5046002807DBC0B2FFF7F8FDC9
:1099500099F8003095F800905FE74FF000095CE758
:10996000039BF0E7BC9600208CD50020043E00202D
:1099700076930020ABAAAAAA6D4B1B68B3F5FA7FB9
:1099800010B500F2C4806B4BDA885C899889D9895C
:10999000B2F57A6F84BF4FF47A62DA801A89B2F531
:1099A0007A6F84BF4FF47A621A81B4F57A6F84BFFC
:1099B0004FF47A645C81B0F57A6F88BF00201A8A10
:1099C00088BF9881B1F57A6F84BF4FF47A61D981ED
:1099D000B2F57A6F84BF00221A8284429CBF0020B5
:1099E0005881914298BF0022998B98BFDA81DA8B17
:1099F0009142997884BF00229A83012902D14E4A6C
:109A0000597011704D484E4A04784E48012C08BFD9
:109A1000024692F84C200A2A6CD0DFED4B7A9FED7B
:109A20004B7A0C2A18BFF0EE477A012966D0484CD1
:109A3000A278062A97BF4749DFED476A01EB82010A
:109A4000D1ED006A217900292ED0013A032A63D989
:109A5000424B9A78022A04BF00229A70404A5378F7
:109A6000052B0FD83F49404803EB031301EB43019B
:109A700013780160022B0DD9002111703B4A3C4B39
:109A8000136010BD002353701378374835490160C7
:109A9000022BF1D8364A03EB431103EB410302EBEF
:109AA0004303324A136010BD5B78234907EE103A36
:109AB0000A78B8EEC77A67EE277A07EE102AB8EE72
:109AC000C77A27EE277AF4EEC76AF1EE10FABFDD07
:109AD00086EEA77AFDEEC77A17EE903A102BA8BF54
:109AE0001023012BB8BF0123DBB29A4238BF1A46BC
:109AF0000A70ADE70129DFED1F7A98D1DFED1E7AFC
:109B00009FED1E7A0A2A18BFF0EE477A8FE74FF0D2
:109B1000005020F043F936E7B7EE000A80EE260A3F
:109B200051F0F0FF2388984228BF184620808FE725
:109B300048040010983F002094A10020180C001049
:109B4000500B0010880A00100AD7A3396F1203398E
:109B500078BA002038D005086F12033894350020F9
:109B60008CD500208C340020C0960020BC960020AC
:109B7000043E00205304E9380F506E3A6F12833AC6
:109B8000074B1B7853B9074B00F1200250F8041B18
:109B900043F8041B9042F9D1012070470020704720
:109BA000A14C0020704C002008B5094B1B780146E1
:109BB00013B1084B1B7843B91522064853F026FA17
:109BC000054B012083F8940108BD0020FCE700BF8D
:109BD000A04C0020504C0020D017002008B5094BA5
:109BE0001B78014613B1084B1B7843B90522064880
:109BF00053F00CFA054B012083F8940108BD0020B6
:109C0000FCE700BFA04C0020684C0020D0170020CB
:109C100038B5164C94F8D231002B154B14BF0122E5
:109C200000221A700BD0052204F5DC71114853F0A4
:109C3000EDF9152204F2BD110F4853F0E7F994F83D
:109C4000D331002B0D4B14BF012200221A700CD00F
:109C50000B4C0C4A04F12005234603CBAB421060A9
:109C600051601C4602F10802F6D138BDD017002021
:109C7000A04C0020684C0020504C0020A14C00203B
:109C800068190020704C002038B50C4B1B789BB92C
:109C90000B4B0C4C03F1200518685968224603C28F
:109CA0000833AB421446F7D1074B012483F8D34164
:109CB000FFF7AEFF204638BD0020FCE7A14C002096
:109CC000704C002068190020D017002038B50B4CCC
:109CD00094F8945185B10522094904F5DC7053F0DC
:109CE00095F91522074904F2BD1053F08FF90123AD
:109CF00084F8D231FFF78CFF284638BDD0170020FA
:109D0000684C0020504C0020F0B50C2934D8DFE816
:109D100001F08A3333335F33333334333333070063
:109D2000048C9689B2F802C01788744D24F48054CC
:109D30002404240C0484038C8488818B23F4005332
:109D400021F4E6411B0409041B0C46EA0C06090C2D
:109D500043EA063341EA0721A8429BB2A4B289B282
:109D600000F09E8005F58065A84200F09980926819
:109D70008480818302640384F0BD048C9589B2F8E9
:109D800002E017885D4E24F480742404240C0484BB
:109D9000038CB0F804C0818B23F400731B0421F002
:109DA000730145EA0E041B0C090443EA0423090C61
:109DB000B0429BB21FFA8CF541EA07015BD0504CD0
:109DC000A04258D0926885808183C2630384F0BD2D
:109DD000048C9589B2F802E0B2F800C0474E24F036
:109DE00010042404240C0484038C8788018B23F042
:109DF000200321F4E6411B0409041B0C45EA0E0470
:109E0000090C43EA041341EA0C21B0429BB2BFB2F1
:109E100089B25BD03A4CA04258D0926887800183C7
:109E200082630384F0BD048C9589B2F802C0178860
:109E3000324E24F001042404240C0484018C848810
:109E4000038B21F0020123F0730309041B04090CA6
:109E500045EA0C051B0CB04241EA0501A4B243EAF5
:109E6000070324D0264DA84221D092688480038322
:109E700042630184F0BDD489168A578A23F40063B3
:109E800043EA04234FF6FF341C40938825F44055E1
:109E90003E4344EA032345EA06149BB2A5B291E788
:109EA000158A24F4804444EA8514A4B25FE7D68975
:109EB000158A578A21F008013143968824F44074AA
:109EC00021F004013D4331432C43CEE7D489168A67
:109ED000B2F812C023F0800343EA04134FF6BF74B4
:109EE0001C40938827F4406546EA0C0644EA0313B5
:109EF00045EA86049BB2A7B28FE700BF000001408D
:109F0000000401402DE9F0474FF40C720021344861
:109F1000344D354E354FDFF8E480DFF8E490DFF85C
:109F2000E4A053F035F8324A3248DFF8DCC0DFF8FD
:109F3000DCE002F51C6426E0B3F1804F2FD0B34281
:109F400032D0BB4232D0634532D0734532D0434524
:109F500032D04B4532D0534532D027498B4232D094
:109F600001F580618B4231D0A1F598318B4230D020
:109F700001F580618B422ED001F580618B422CD09F
:109F80002032944209D013688342D5D101216B6CF1
:109F900020320B4394426B64F5D1BDE8F087012178
:109FA0002B6C0B432B64EBE70221F9E70421F7E765
:109FB0000821F5E71021F3E72021F1E70221E6E788
:109FC0004FF48031E3E74FF40031E0E74FF48021B4
:109FD000DDE74021E4E78021E2E74FF48071DFE72D
:109FE00034760020003802400004004000080040A1
:109FF00054D0050800000140004401400014004016
:10A000000004014000400140000C004000100040EE
:10A010002DE9F843304D2B8AB5F80C8018EA030877
:10A0200027D02E4E4FF00047B8FA88F327FA03F2F4
:10A03000D24391B21B3B08EA02082982042B15D8AF
:10A04000DFE803F0372D23190300D6F82C32002B5C
:10A0500039D1EB6A1FFA83F9D6F8284234B1236864
:10A060002046494698476468002CF8D1B8F1000FA3
:10A07000DAD1BDE8F883D6F80802696B036889B2C3
:10A080009847B8F1000FCFD1F3E7D6F80C02A96BCF
:10A09000036889B29847B8F1000FC5D1E9E7D6F84F
:10A0A0001002E96B036889B29847B8F1000FBBD181
:10A0B000DFE7D6F81402296C036889B29847B8F133
:10A0C000000FB1D1D5E703F1FF3900231FFA89F959
:10A0D000C6F82C32C0E700BF0020004034760020D4
:10A0E0002DE9F843304D2B8AB5F80C8018EA0308A7
:10A0F00027D02E4E4FF00047B8FA88F327FA03F224
:10A10000D24391B21B3B08EA02082982042B15D8DE
:10A11000DFE803F0372D23190300D6F8DC31002BDC
:10A1200039D1EB6A1FFA83F9D6F8D84134B12368E4
:10A130002046494698476468002CF8D1B8F1000FD2
:10A14000DAD1BDE8F883D6F8B801696B036889B243
:10A150009847B8F1000FCFD1F3E7D6F8BC01A96B4F
:10A16000036889B29847B8F1000FC5D1E9E7D6F87E
:10A17000C001E96B036889B29847B8F1000FBBD101
:10A18000DFE7D6F8C401296C036889B29847B8F1B3
:10A19000000FB1D1D5E703F1FF3900231FFA89F988
:10A1A000C6F8DC31C0E700BF00180040347600205C
:10A1B0002DE9F843304D2B8AB5F80C8018EA0308D6
:10A1C00027D02E4E4FF00047B8FA88F327FA03F253
:10A1D000D24391B21B3B08EA02082982042B15D80E
:10A1E000DFE803F0372D23190300D6F8B431002B34
:10A1F00039D1EB6A1FFA83F9D6F8B04134B123683C
:10A200002046494698476468002CF8D1B8F1000F01
:10A21000DAD1BDE8F883D6F89001696B036889B29A
:10A220009847B8F1000FCFD1F3E7D6F89401A96BA6
:10A23000036889B29847B8F1000FC5D1E9E7D6F8AD
:10A240009801E96B036889B29847B8F1000FBBD158
:10A25000DFE7D6F89C01296C036889B29847B8F10A
:10A26000000FB1D1D5E703F1FF3900231FFA89F9B7
:10A27000C6F8B431C0E700BF004801403476002082
:10A280002DE9F843304D2B8AB5F80C8018EA030805
:10A2900027D02E4E4FF00047B8FA88F327FA03F282
:10A2A000D24391B21B3B08EA02082982042B15D83D
:10A2B000DFE803F0372D23190300D6F86431002BB3
:10A2C00039D1EB6A1FFA83F9D6F8604134B12368BB
:10A2D0002046494698476468002CF8D1B8F1000F31
:10A2E000DAD1BDE8F883D6F84001696B036889B21A
:10A2F0009847B8F1000FCFD1F3E7D6F84401A96B26
:10A30000036889B29847B8F1000FC5D1E9E7D6F8DC
:10A310004801E96B036889B29847B8F1000FBBD1D7
:10A32000DFE7D6F84C01296C036889B29847B8F189
:10A33000000FB1D1D5E703F1FF3900231FFA89F9E6
:10A34000C6F86431C0E700BF004001403476002009
:10A350002DE9F843324D2B8AB5F80C8018EA030832
:10A3600027D0304E4FF00047B8FA88F327FA03F2AF
:10A37000D24391B21B3B08EA02082982042B15D86C
:10A38000DFE803F03B31271D0300D6F83C31002BFA
:10A390003DD1EB6A1FFA83F9D6F8384134B123680E
:10A3A0002046494698476468002CF8D1B8F1000F60
:10A3B000DAD11D491D48BDE8F843FEF74FBFD6F876
:10A3C0001801696B036889B29847B8F1000FCBD1C7
:10A3D000EFE7D6F81C01A96B036889B29847B8F17A
:10A3E000000FC1D1E5E7D6F82001E96B036889B217
:10A3F0009847B8F1000FB7D1DBE7D6F82401296CF4
:10A40000036889B29847B8F1000FADD1D1E703F1E5
:10A41000FF3900231FFA89F9C6F83C31BCE700BFB9
:10A42000000401403476002014780020001C004015
:10A430002DE9F843304D2B8AB5F80C8018EA030853
:10A4400027D02E4E4FF00047B8FA88F327FA03F2D0
:10A45000D24391B21B3B08EA02082982042B15D88B
:10A46000DFE803F0372D23190300D6F83C31002B29
:10A4700039D1EB6A1FFA83F9D6F8384134B1236831
:10A480002046494698476468002CF8D1B8F1000F7F
:10A49000DAD1BDE8F883D6F81801696B036889B290
:10A4A0009847B8F1000FCFD1F3E7D6F81C01A96B9C
:10A4B000036889B29847B8F1000FC5D1E9E7D6F82B
:10A4C0002001E96B036889B29847B8F1000FBBD14E
:10A4D000DFE7D6F82401296C036889B29847B8F100
:10A4E000000FB1D1D5E703F1FF3900231FFA89F935
:10A4F000C6F83C31C0E700BF0004014034760020BC
:10A500002DE9F843304D2B8AB5F80C8018EA030882
:10A5100027D02E4E4FF00047B8FA88F327FA03F2FF
:10A52000D24391B21B3B08EA02082982042B15D8BA
:10A53000DFE803F0372D23190300D6F8C430002BD1
:10A5400039D1EB6A1FFA83F9D6F8C04034B12368D9
:10A550002046494698476468002CF8D1B8F1000FAE
:10A56000DAD1BDE8F883D6F8A000696B036889B238
:10A570009847B8F1000FCFD1F3E7D6F8A400A96B44
:10A58000036889B29847B8F1000FC5D1E9E7D6F85A
:10A59000A800E96B036889B29847B8F1000FBBD1F6
:10A5A000DFE7D6F8AC00296C036889B29847B8F1A8
:10A5B000000FB1D1D5E703F1FF3900231FFA89F964
:10A5C000C6F8C430C0E700BF000C0040347600205D
:10A5D0002DE9F8432F4D2B8AB5F80C8018EA0308B3
:10A5E00027D02D4E4FF00047B8FA88F327FA03F230
:10A5F000D24391B21B3B08EA02082982042B15D8EA
:10A60000DFE803F0352B22190300D6F89C30002B2D
:10A6100037D1EB6A1FFA83F9D6F8984034B1236832
:10A620002046494698476468002CF8D1B8F1000FDD
:10A63000DAD1BDE8F883B06F696B036889B29847D7
:10A64000B8F1000FD0D1F4E7F06FA96B036889B2BD
:10A650009847B8F1000FC7D1EBE7D6F88000E96B57
:10A66000036889B29847B8F1000FBDD1E1E7D6F889
:10A670008400296C036889B29847B8F1000FB3D100
:10A68000D7E703F1FF3900231FFA89F9C6F89C3098
:10A69000C2E700BF00080040347600202DE9F843EF
:10A6A0002C4D2B8AB5F80C8018EA030825D02A4EC9
:10A6B0004FF00047B8FA88F327FA03F2D24391B279
:10A6C0001B3B08EA02082982042B13D8DFE803F0B9
:10A6D000322920170300736F002B34D1EB6A1FFA65
:10A6E00083F9346F34B1236820464946984764683B
:10A6F000002CF8D1B8F1000FDCD1BDE8F883306D43
:10A70000696B036889B29847B8F1000FD2D1F4E7BA
:10A71000706DA96B036889B29847B8F1000FC9D171
:10A72000EBE7B06DE96B036889B29847B8F1000FA9
:10A73000C0D1E2E7F06D296C036889B29847B8F19F
:10A74000000FB7D1D9E703F1FF3900231FFA89F9C8
:10A750007367C6E700040040347600202DE9F84313
:10A760004FF080452B8AB5F80C8018EA030825D0F5
:10A77000294E4FF00047B8FA88F327FA03F2D24384
:10A7800091B21B3B08EA02082982042B13D8DFE8A8
:10A7900003F0322920170300F36C002B34D1EB6A4D
:10A7A0001FFA83F9B46C34B12368204649469847B0
:10A7B0006468002CF8D1B8F1000FDCD1BDE8F88353
:10A7C000B06A696B036889B29847B8F1000FD2D1BB
:10A7D000F4E7F06AA96B036889B29847B8F1000FF3
:10A7E000C9D1EBE7306BE96B036889B29847B8F1E0
:10A7F000000FC0D1E2E7706B296C036889B29847FB
:10A80000B8F1000FB7D1D9E703F1FF3900231FFAE0
:10A8100089F9F364C6E700BF347600202DE9F843D8
:10A82000324D33493348FEF719FD2B8AB5F80C80B9
:10A8300018EA030827D02E4E4FF00047B8FA88F3E5
:10A8400027FA03F2D24391B21B3B08EA020829829D
:10A85000042B15D8DFE803F0372D23190300D6F8B1
:10A860008C31002B39D1EB6A1FFA83F9D6F8884175
:10A8700034B123682046494698476468002CF8D1D3
:10A88000B8F1000FDAD1BDE8F883D6F86801696B3A
:10A89000036889B29847B8F1000FCFD1F3E7D6F833
:10A8A0006C01A96B036889B29847B8F1000FC5D154
:10A8B000E9E7D6F87001E96B036889B29847B8F107
:10A8C000000FBBD1DFE7D6F87401296C036889B2A9
:10A8D0009847B8F1000FB1D1D5E703F1FF39002354
:10A8E0001FFA89F9C6F88C31C0E700BF0044014067
:10A8F00034760020000001402DE9F8432C4D2B8ACE
:10A90000B5F80C8018EA030825D02A4E4FF000470E
:10A91000B8FA88F327FA03F2D24391B21B3B08EA54
:10A9200002082982042B13D8DFE803F0322920170C
:10A930000300736A002B34D1EB6A1FFA83F9346A7F
:10A9400034B123682046494698476468002CF8D102
:10A95000B8F1000FDCD1BDE8F8833068696B03689B
:10A9600089B29847B8F1000FD2D1F4E77068A96BAB
:10A97000036889B29847B8F1000FC9D1EBE7B06816
:10A98000E96B036889B29847B8F1000FC0D1E2E7DC
:10A99000F068296C036889B29847B8F1000FB7D105
:10A9A000D9E703F1FF3900231FFA89F97362C6E77B
:10A9B0000000014034760020F0B40568AB0AA3F52E
:10A9C0008013522B5AD8364CE45C0D2C56D8437960
:10A9D000B5F80CC0022023FA00F6B04087B2A00000
:10A9E0003346061903EB46032E4E00294ED047EAA4
:10A9F0000C0703F1040C46F8231046F82C20AF8115
:10AA00002023282717FB0437F319EFF31181502275
:10AA100082F31288021906EBC202D2F810C0BCF110
:10AA2000000F03D046F807C013690433021906EB80
:10AA3000C202576917B11F6053690433021906EB4C
:10AA4000C202976917B11F6093690433021906EBBC
:10AA5000C202D76917B11F60D36904330022C9B29B
:10AA60001A6081F31188044406EBC406336A3BB9CB
:10AA7000AB8923F001031B041B0CAB81F0BC7047B6
:10AA8000AB8943F00103AB81F0BC70472CEA0707A8
:10AA900003F1040CAF8146F8231046F82C20AFE7F1
:10AAA0000C1506083476002010B503687D487E4CEE
:10AAB0000139834282B0246889B200F0B180A0F5E8
:10AAC0008060834200F0AC8000F58040834200F05B
:10AAD000828000F5806083427DD000F580608342F3
:10AAE00079D018886408B4FBF2F4013CA4B282B2B5
:10AAF000B3F1804F0AD06D48834207D000F58060E3
:10AB0000834203D000F58060834202D122F07002BC
:10AB100092B26748834200F0918000F580608342E2
:10AB200000F0958022F4407200F56C4092B28342AE
:10AB30001A80D9621C8540F09380012100221A8678
:10AB4000998219885B4841F00101834219804AD0FB
:10AB5000B3F1804F00F08F80544A934200F08D8013
:10AB600002F58062934200F08A8002F5806293428F
:10AB700000F0878002F58062934200F0848002F545
:10AB80008062934200F0818002F5704293427ED051
:10AB900002F5705293427CD002F5806293427AD0E3
:10ABA00002F58062934278D0A2F59832934276D033
:10ABB00002F58062934215D002F58062934208BF8D
:10ABC0000D2210D002A84FF0012340F8043D2EF0D2
:10ABD00059FB02B010BD1888B4FBF2F4013CA4B2DA
:10ABE00082B285E70C22344B03EBC20201A892F833
:10ABF000E1498DF80440012300228DF805308DF8DD
:10AC000007308DF806202EF03DFB1B2C0FD02E2C8C
:10AC1000DFD12A4B019301A82EF034FB02B010BD06
:10AC20001888B4FBF2F4013CA4B282B26EE7244B64
:10AC3000019301A82EF026FB02B010BD01201A805E
:10AC4000D9621C8598821A8802431A8084E7012001
:10AC50001A80D9621C8598821A8802431A8077E785
:10AC6000104A93423FF469AF01229A821A8842F057
:10AC700001021A806CE70122B5E70222B3E7032242
:10AC8000B1E70422AFE70522ADE70622ABE70722D2
:10AC9000A9E70822A7E70922A5E70A22A3E70B22D2
:10ACA000A1E700BF0004014088BC00200004004070
:10ACB000001000400000014038D005082C010001C0
:10ACC000190100012C4B98423DD0B0F1804F3CD08F
:10ACD000A3F57C4398423AD003F58063984238D07C
:10ACE00003F58063984236D003F58063984234D0F0
:10ACF00003F58063984234D003F57043984232D014
:10AD000003F5705398422AD003F5806398422CD003
:10AD100003F5806398422AD0A3F59833984228D04F
:10AD200003F58063984207D003F58063984208BF1B
:10AD30000D2202D0002070470C22104B03EBC203FF
:10AD400093F8E00970470022F7E70122F5E70222B5
:10AD5000F3E70322F1E70422EFE70522EDE70822FB
:10AD6000EBE70622E9E70722E7E70922E5E70A22FF
:10AD7000E3E70B22E1E700BF0000014038D00508FF
:10AD8000800AA0F58010522808D8054B1B5C0D2BBB
:10AD900004D8044A134493F94C0A704700207047C2
:10ADA0000C15060838D0050870B40E4E1024334632
:10ADB0000125002203E001324E2A0BD01C79A0426B
:10ADC00003F12003F7D18D4207D0013201354E2A1D
:10ADD000EDB2F3D1002070BC704706EB421070BC9E
:10ADE000704700BF54D00508002330B40F4A1D46F9
:10ADF000012404E00133072B0DD012F8204C30EA77
:10AE0000040402F12002F5D1A94207D00133013533
:10AE1000072BEDB2F1D1002030BC7047044A02EBA1
:10AE2000431330BC93F8600A704700BFBADA0508D4
:10AE300038D005082DE9F843214C06460F46002579
:10AE400014F8010C58B12378194643B1FFF7ACFF51
:10AE5000014620B10068FFF793FFB04222D00135D0
:10AE6000152D04F10304EBD1164BD3F80090B9F182
:10AE7000000F21DD03F104084146002402E0013403
:10AE8000A14519D08D682868FFF77AFF864201F541
:10AE90008071F4D16B79BB42F1D108EB042303F14B
:10AEA000FC000AE04B79BB42D9D1074810F81530B5
:10AEB00000EB45000BB9D7E70448BDE8F88300BFB5
:10AEC00095BA00201C000010D4BA002074DB0508DD
:10AED0002DE9F04128B3154E002402E00134152C71
:10AEE0001FD065002B19F718F35C8342F6D17B78ED
:10AEF000ABB1884619461746FFF756FF064600686D
:10AF0000FFF73EFF7179FFF795FF03784BB9084BC8
:10AF10001D4403F814806F703046BDE8F0811B6853
:10AF2000FFDE00263046BDE8F08100BF94BA002065
:10AF3000D4BA002010B40B49002301E0152B0CD02B
:10AF400003EB430201338C5C84420A44F6D151780E
:10AF500018B111B15DF8044B26E700205DF8044BF1
:10AF6000704700BF94BA00202DE9F8439B490B7845
:10AF7000A3F11702022A0FD9994A12F833000028C8
:10AF800040F02B82D800024452782AB1954A12F838
:10AF90003330002B00F08B82934F944D97F808903C
:10AFA000DFF87082002426462A5B12F0010C05EBC4
:10AFB000040306F1010100F0E481CEB2510801F072
:10AFC00077319308511AD00803F03333CB1A00F0CD
:10AFD00011315B1A03EB231303F00F33A8FB031E9D
:10AFE0004FEADE1ECEEB0E2EA3EB0E0EBEF1010FCE
:10AFF00005EB0400494604F108040EDDBEF1020F22
:10B0000040F0C481BCF1000F02D012F42F7F04D1B4
:10B0100030F01AFE002800F0B981302CC4D1013E76
:10B02000022E00F2B381022019F094F9704B1B78C4
:10B03000022B00F0FA81002800F03C826D4E4FF4A4
:10B040007A6C334606F5C97E00254FF064085A88AD
:10B05000B2F57A6FB3F84C2088BFA3F802C0B2F5FE
:10B060007A6F9A8888BFA3F84CC0B2F57A6FDA88F5
:10B0700088BFA3F804C09988B2F57A6F84BF002214
:10B08000DD809142B3F86010B3F8622098BF9D80D4
:10B09000914293F8712088BFA3F86050013A632A67
:10B0A00093F8722088BF83F871800132D2B2092AE6
:10B0B00088BF83F8725003F16B00194600228C7A26
:10B0C00010F8019F0132A14528BF0570032A01F144
:10B0D0000601F4D186337345B9D1DFF83C8198F885
:10B0E0000230042B00F0828143B9B8F80030B3F588
:10B0F000F07F84BF4FF4F073A8F80030FEF73CFCFB
:10B100003D483E4C81783E4D103020F0F5F8E17915
:10B1100004F1080020F0F0F8617D04F1160020F041
:10B12000EBF82C68374B2340002B00F0C781E10778
:10B1300000F19A81620400F19E81230700F1A2814F
:10B14000A00400F1A681210440F140810023FB739B
:10B1500087F8233043F0E0FB002800F0E5807B7E99
:10B16000032B00F0E1805A1E012A40F2F4800023F4
:10B170003383A6F89E30A6F8243143F0CDFB002897
:10B1800040F0E8800023E20486F84F3086F8D5309E
:10B1900086F85B3140F1E6801B4BDA79022A08BF62
:10B1A00001224FF0070008BFDA7143F0B3F810B185
:10B1B000072043F055F84FF4806019F0CBF80028D1
:10B1C00000F0DA80114F3C4604F17D057837617953
:10B1D00081B3207860B30E4B23E000BF54480020B9
:10B1E0008C4E0608E448060818D80020C8D900206C
:10B1F00084300020043E00205C480020C44400202D
:10B200008CD800200960000234400020509D0020AE
:10B21000559D00208180808078BA00200633AB42A3
:10B2200008D013F8052C8A42F8D11A78002AF5D0F4
:10B2300043F016F80634A742C9D198F80230082B1B
:10B2400000F0E6804FF400701EF0A8FD4FF40010EF
:10B250001EF0A4FD9B4C4FF000701EF09FFD4FF0C0
:10B2600080601EF09BFDA388002B40F0F580964A7D
:10B27000136813F07F4F1CBF00231360936823F4FF
:10B28000007323F002030BB1002393601379013B99
:10B29000042B84BF0123137198F8023098F806201C
:10B2A000053B032B7AD898F81030002188F8041059
:10B2B000002B6FD0854BDB7B002B6FD022B1844BF2
:10B2C0001A7842B91B7933B9002386F87E3086F8A4
:10B2D000043186F88A317F4BB3F8762002F00F01F3
:10B2E000032966D8C2F30312022A62D8B3F8782081
:10B2F00002F00F01032957D8C2F30312022A53D8D0
:10B30000754B764A5C7850781978844257D900207A
:10B310005870002952D192F8EA209978914201D9C7
:10B3200000229A70BDE8F8830023B3817382A6F8E7
:10B330009230A6F89830A6F81831A6F81E3143F0DE
:10B34000EBFA00283FF413AF7B7E5A1E012A3FF62A
:10B350000EAF00E07B7E023B022B3FF613AFE20410
:10B360003FF51AAF23067FF517AF4FF4806018F052
:10B37000F1FF00287FF426AF4FF000601EF00EFDB5
:10B3800020E793F90230142B7FF418AE544816F0DE
:10B3900041FE48E698F80530012B8BD1002A93D066
:10B3A000002388F806308FE740F60122A3F87820C2
:10B3B000A6E74FF42062A3F8762097E798801078EC
:10B3C0008842A8D2002119709980A4E7FB7B002B4A
:10B3D00064D0002387F82330BCE6D80014186468D2
:10B3E000002C7FF4D0AD17240C70CCE54FF48050C6
:10B3F0001EF0D4FCB8F81830B3F57A7F37BF4FF49D
:10B400007A7298F8023098F80230A8F818206BE6A3
:10B4100098F80630002B3FF415AF98F81030012B48
:10B4200004BF022388F810300CE700283FF406AE72
:10B430002C4E2D4B317890F90240FF2503F130005E
:10B4400093F90620A24202D10139C9B29D71083395
:10B450009842F5D13170F1E52078FFF76BFD0028B7
:10B460007FF405AFA08002E720481EF097FC2C680F
:10B4700062047FF562AE1E481EF090FC2C68230724
:10B480007FF55EAE1B481EF089FC2C68A0047FF59A
:10B490005AAE19481EF082FC2C6854E642F20103B1
:10B4A0001C423FF457AE002387F8233052E618239E
:10B4B0000B7071E580201EF071FCBFE544F00804BC
:10B4C0002C6034E6A0D60020648100208CD50020BA
:10B4D0009CA10020241E0020209300203436002050
:10B4E000C8D9002032810020FCD900200860000269
:10B4F00009200002016000020940000208B101B108
:10B5000052E40020704700BF10B40A49002301E054
:10B51000152B0AD003EB430201338C5C84420A44AE
:10B52000F6D110465DF8044B704700205DF8044BDF
:10B53000704700BF94BA00209A4AF0B402F5C47074
:10B54000994F9A4D012603E00832904200F0208185
:10B550009379002BF8D1136803F13F4101F57E0187
:10B56000890A795C01F01F044909032906FA04F4E9
:10B5700000F01481042900F00D81022902D1696CC8
:10B580000C436C649188CC070DD51C6824F003042F
:10B590001C601C681C60DC6824F00304DC60DC6850
:10B5A00044F00104DC608C070DD51C6824F00C0409
:10B5B0001C601C681C60DC6824F00C04DC60DC6827
:10B5C00044F00404DC604C070DD51C6824F0300402
:10B5D0001C601C681C60DC6824F03004DC60DC68E3
:10B5E00044F01004DC600C070DD51C6824F0C00486
:10B5F0001C601C681C60DC6824F0C004DC60DC6833
:10B6000044F04004DC60CC060DD51C6824F4407482
:10B610001C601C681C60DC6824F44074DC60DC681E
:10B6200044F48074DC608C060DD51C6824F44064FE
:10B630001C601C681C60DC6824F44064DC60DC680E
:10B6400044F48064DC604C060DD51C6824F440543E
:10B650001C601C681C60DC6824F44054DC60DC68FE
:10B6600044F48054DC600C060DD51C6824F440447E
:10B670001C601C681C60DC6824F44044DC60DC68EE
:10B6800044F48044DC60CC050DD51C6824F44034BF
:10B690001C601C681C60DC6824F44034DC60DC68DE
:10B6A00044F48034DC608C050DD51C6824F44024FF
:10B6B0001C601C681C60DC6824F44024DC60DC68CE
:10B6C00044F48024DC604C050DD51C6824F440143F
:10B6D0001C601C681C60DC6824F44014DC60DC68BE
:10B6E00044F48014DC600C050DD51C6824F440047F
:10B6F0001C601C681C60DC6824F44004DC60DC68AE
:10B7000044F48004DC60CC040DD51C6824F0407443
:10B710001C601C681C60DC6824F04074DC60DC6821
:10B7200044F08074DC608C040DD51C6824F0406407
:10B730001C601C681C60DC6824F04064DC60DC6811
:10B7400044F08064DC604C040DD51C6824F0405447
:10B750001C601C681C60DC6824F04054DC60DC6801
:10B7600044F08054DC6009047FF5EEAE196821F0E6
:10B770004041196019681960D96821F04041D960C9
:10B78000D968083241F080419042D9607FF4E0AE40
:10B79000F0BC7047296B0C432C63F3E6296C0C4317
:10B7A0002C64EFE600BB00205C4D06080038024028
:10B7B0002DE98048013085B0C3B20393954C964F74
:10B7C000DFF860A2954D964E0A2302934AF058FD89
:10B7D0004FF4FA73DFF850E201934FF01008DAF8F3
:10B7E0000430C3F30803002B40F0D280EFF3118341
:10B7F000002B40F0CD802068AA6823689842FAD1D7
:10B8000033689A42F7D8D7F800C04FF47A7101FB39
:10B810000CF39B1AB3FBFCF301FB00304FF47A7C72
:10B820004FF00109DAF80430C3F30803002B40F0AD
:10B830009180EFF31183002B40F08C802368A9687E
:10B8400022689342FAD132689142F7D83A680CFBE9
:10B8500002FBABEB0101B1FBF2F10CFB03131B1A72
:10B86000B3F57A7FDED3019B013B0193B7D10398F7
:10B870004AF05AFB4FF47A73DFF8ACE101934FF0D2
:10B880001008DAF80430C3F30803002B40F0A1805D
:10B89000EFF31183002B40F09C802068AA68236896
:10B8A0009842FAD133689A42F7D8D7F800C04FF4DB
:10B8B0007A7101FB0CF39B1AB3FBFCF301FB003024
:10B8C0004FF47A7C4FF00109DAF80430C3F308032F
:10B8D00013BBEFF31183FBB92368A9682268934275
:10B8E000FAD132689142F7D83A680CFB02FBABEB15
:10B8F0000101B1FBF2F10CFB03131B1AB3F57A7FC4
:10B90000E2D3019B013B0193BBD1029B013B02931C
:10B910007FF45CAF4FF014F8EFF3118188F31288D5
:10B92000D5F808B02B68DB0344BFCEF80090D5F8FB
:10B9300008B02368DEF80020C9B281F311883968A5
:10B9400013440CFB01F2A2EB0B02B2FBF1F20CFB75
:10B950000323D2E7EFF3118188F31288D5F808B0FA
:10B960002B68DB0344BFCEF80090D5F808B02368FD
:10B97000DEF80020C9B281F31188396813440CFB4A
:10B9800001F2A2EB0B02B2FBF1F20CFB032366E720
:10B99000EFF3118388F31288D5F808C02A68D20320
:10B9A00004D50122CEF80020D5F808C02068DEF8C2
:10B9B0000090DBB283F3118839684FF47A724844FF
:10B9C00002FB01F3A3EB0C03B3FBF1F302FB00302A
:10B9D00024E7EFF3118388F31288D5F808C02A68AA
:10B9E000D20304D50122CEF80020D5F808C0206883
:10B9F000DEF80090DBB283F3118839684FF47A7275
:10BA0000484402FB01F3A3EB0C03B3FBF1F302FB8D
:10BA1000003055E774C5002078C5002010E000E034
:10BA20007CC5002000ED00E070C500202DE9F04F3E
:10BA300085B0CDE902109B4DDFF878A2029B013B57
:10BA40000293013300F02A814AF01AFC964C974F7A
:10BA5000DFF864E2964E4FF4FA7301934FF010084A
:10BA6000DEF80430C3F30803002B40F0F680EFF358
:10BA70001183002B40F0F1802068AA682368984267
:10BA8000FAD133689A42F7D8D7F800C04FF47A71E8
:10BA900001FB0CF39B1AB3FBFCF301FB00304FF4EA
:10BAA0007A7C4FF00109DEF80430C3F30803002B61
:10BAB00040F0B580EFF31183002B40F0B080236895
:10BAC000A96822689342FAD132689142F7D83A685D
:10BAD0000CFB02FBABEB0101B1FBF2F10CFB03131E
:10BAE0001B1AB3F57A7FDED3019B013B0193B7D1DB
:10BAF000039B6F4E581CC0B24AF016FADFF8B8E14B
:10BB00004FF47A730193DEF80430C3F308034FF067
:10BB10001008002B44D1EFF31183002B40D1206893
:10BB2000AA6823689842FAD133689A42F7D8D7F8BE
:10BB300000C04FF47A7101FB0CF39B1AB3FBFCF3CA
:10BB400001FB00304FF47A7C4FF00109DEF804303D
:10BB5000C3F30803002B44D1EFF31183002B40D132
:10BB60002368A96822689342FAD132689142F7D8D3
:10BB70003A680CFB02FBABEB0101B1FBF2F10CFBF1
:10BB800003131B1AB3F57A7FE0D3019B013B0193AA
:10BB90003FF454AFDEF80430C3F30803002BBAD0EF
:10BBA000EFF3118388F31288D5F808C02A68D2030E
:10BBB00004D50122CAF80020D5F808C02068DAF8B8
:10BBC0000090DBB283F3118839684FF47A724844ED
:10BBD00002FB01F3A3EB0C03B3FBF1F302FB003018
:10BBE000B0E7EFF3118188F31288D5F808B02B681D
:10BBF000DB0344BFCAF80090D5F808B02368DAF830
:10BC00000020C9B281F31188396813440CFB01F29A
:10BC1000A2EB0B02B2FBF1F20CFB0323B1E7EFF353
:10BC2000118188F31288D5F808B02B68DB0344BF74
:10BC3000CAF80090D5F808B02368DAF80020C9B235
:10BC400081F31188396813440CFB01F2A2EB0B025B
:10BC5000B2FBF1F20CFB032342E7EFF3118388F30D
:10BC60001288D5F808C02A68D20304D50122CAF880
:10BC70000020D5F808C02068DAF80090DBB283F322
:10BC8000118839684FF47A72484402FB01F3A3EB40
:10BC90000C03B3FBF1F302FB003000E705B0BDE895
:10BCA000F08F00BF10E000E074C5002078C50020D0
:10BCB0007CC5002070C5002000ED00E0224B5B68D1
:10BCC000C3F3080330B4D3B9EFF31183BBB91F4AF0
:10BCD0001F4D20481368846811688B42FAD1296887
:10BCE0008C42F7D81C4A11684FF47A7202FB01F0BB
:10BCF000001B30BCB0FBF1F002FB03007047EFF318
:10BD00001182102383F3128803F1E023D2B29C68DE
:10BD1000196811F4803F11491EBF012008609C681A
:10BD20000A4B18680B6882F311880B4A11684FF4AC
:10BD30007A72034402FB01F0001B30BCB0FBF1F04F
:10BD400002FB0300704700BF00ED00E074C5002057
:10BD50007CC5002010E000E078C5002070C5002000
:10BD60002DE9F04F054B2DED028B1C78ABB03CB1AB
:10BD70002BB0BDEC028BBDE8F08F00BF5C930020C0
:10BD8000DFF880B3DBF800305F05F1D5039011F0E8
:10BD90009BFCC24B1B78012B00F04582C04B1B78EB
:10BDA000002B3CD0BF4D0399D5F8F832BE4ACB1AD0
:10BDB000934200F27D82DFF8509399F80060002EE4
:10BDC00000F0A083B94A16684EB3B94FD5F80C33CA
:10BDD0000398F968C31A8B4221D395F80833002BD6
:10BDE00000F0DB8695F81173B24995F810C3086826
:10BDF000013BDBB2013785F80833FFB2002B00F0BE
:10BE0000638616F8011B85F8117301EB0C031660AD
:10BE100085F8103333F0E6F9039BC5F80C33FFF7D0
:10BE20004DFFA54B93F8008000F57A70B8F1010F33
:10BE3000209000F0C081A14B1B78002B00F0C78040
:10BE40009F4F3B68002B00F0C2809E4B954D1B68B6
:10BE500004931A46D5F81833D31A632B40F2B780EF
:10BE6000DFF8A892984EDFF8A88241202EF05CFF00
:10BE7000B9F9023086FB0320DB17C3EBA00080B2C8
:10BE80002EF036FFB9F9003086FB0320DB17C3EB39
:10BE9000A00080B22EF02CFFB9F9043086FB0320FD
:10BEA000DB17C3EBA00080B22EF022FF98F8001041
:10BEB000386833F097F995F81CA31AF0010600F0E2
:10BEC0000E86DFF85092D9F8003098066FD57F4B78
:10BED0007F4E1B78990742F17581337D042B8CBF0F
:10BEE00003230223059347202EF01EFF30682EF017
:10BEF000CBFE70682EF0C8FEF389764A3868A2FB44
:10BF00000323C3F3471A514633F06CF998F8001035
:10BF1000D9F800208AEA010312F0140F88F80030E3
:10BF200016BF6D4BB06818682EF0AEFE059B367DCF
:10BF3000386843EA8606F6B2314633F053F998F88A
:10BF4000003038685E40314688F8006033F04AF9C6
:10BF500095F81CA3BAF1000F29D1604E4F202EF0A6
:10BF6000E3FE30682EF090FE70682EF08DFE504695
:10BF70002EF08AFE0121386833F034F9534A98F8DC
:10BF800000301678386806F0010683F00103314668
:10BF900088F8003033F026F998F80030386873409C
:10BFA000194688F8003033F01DF995F81CA3049B5E
:10BFB0004B4AC5F818330AF10103DBB2A2FB0312A6
:10BFC000D20802EB8202A3EB420385F81C33DFF8B0
:10BFD000488198F80030022B00F05983344D6B7C77
:10BFE000032B00F067833F4B1B78002B3CD03E4F68
:10BFF0003B68CBB32B4DFFF761FED5F82833049097
:10C0000044F61F62C31A93422ED995F82E33002BA3
:10C0100001F04283013B85F82E3395F82F33002B36
:10C0200001F01C82013B85F82F3395F83233002B49
:10C0300000F0E886013B85F8323395F83693B9F184
:10C04000000F00F0F58509F1FF3985F8369395F872
:10C050003783B8F1000F01F0CD8408F1FF3885F87F
:10C060003783049BC5F82833204B1B78002B40F006
:10C07000A3821F4B1B78002B00F094801D4B1B7874
:10C08000002B40F094801C4B1B78002B3FF470AECB
:10C09000044F1A4C1A4D07F58F663FE0A997002010
:10C0A000B6970020D01700203F0D0300D89600203F
:10C0B00088010020D0960020B7970020C497002068
:10C0C000A096002074C50020676666666C93002009
:10C0D000B0D900201F85EB51AC96002048310020DC
:10C0E000CDCCCCCCCC970020D0970020FC98002061
:10C0F000F496002073450020D6970020DC9700209E
:10C10000E09700208CD80020DC960020B49300201B
:10C11000A49600200C890020269C0020206833F083
:10C120005DF800283FF424AE206833F04FF82B78F8
:10C13000804673B1013B20682B7033F04FF8002824
:10C140003FF416AE206833F041F82B788046002B80
:10C15000F0D14D490322304650F001FF97F8781492
:10C1600087F87B84023911F0FF0100F08C823144A2
:10C1700032464FF6FF7312F8010B1B1A91429BB225
:10C18000F9D11A0A1FFA88F89045C7D197F87A248E
:10C19000DBB29A42C2D13D482EF02AFB2B781844DC
:10C1A0002870BBE73A4B1B78002B7FF46CAF0398E9
:10C1B0002FF0F0FA67E7374E306800283FF43BAEC7
:10C1C0004FF000098DF8789033F008F830B3324F13
:10C1D000324D306832F0FAFF83B27E2B00F02284B9
:10C1E0003A7CD6F800C0002A40F0638395F8131318
:10C1F000002900F0BE811B2B85F8132340F06083DB
:10C20000604632F0EBFF002800F0E884306887F8E1
:10C21000108032F0E3FF0028DBD1002020AA1EA905
:10C220002EF09CFD07E61E4B1B68002B3FF4B6ADBD
:10C230001A4D0399D5F8EC321A4ACB1A93427FF77C
:10C24000ADADDFF8689095F8F032D9F80070C5F818
:10C25000EC120133BE0785F8F03201F12D8617F09C
:10C26000340F41F0158695F8F062390701F18E839D
:10C2700016F0070701F00683282E01F059870A4BB4
:10C280005E201B68984789E5491C0020481C002057
:10C2900025970020C496002088010020D017002098
:10C2A0006893002047E80100F88A00200C890020EC
:10C2B000CF4BD0481B88D049D04E4F7A3168D04AF6
:10C2C0000533A0FB0303D5F8FC02081A4FF47A717A
:10C2D000DB0801FB07F15FFA83FC00271B0A884299
:10C2E00082F81EC0D37782F814C053759770177107
:10C2F00080F0D683C34BC4481B68C44EC449B6F90A
:10C3000000C00F68DFF84083896880FB03E6DB1715
:10C31000C3EB661303F5FA739BB293761B0AD376CD
:10C3200088FB079388FB0198FF17C917C7EBA30782
:10C33000C1EBA8010CF5EA43DFF810E317773033BF
:10C340003F1282F8201009121B12B24E9EF800E034
:10C35000577782F8211080FB0C874FEAEC71C1EB14
:10C36000671182F82330AC4B96F814A083F81AA01A
:10C3700078310CF1300C1EF0020F82F8241082F894
:10C3800022C000F04C83D6F800E0A44AD6F804C0DE
:10C39000DFF8BC82DFF8BC9282FB0E314FEAEE7709
:10C3A00082FB0C32C7EBA1574FEAEC71C1EBA252F2
:10C3B00008FB07E108FB02C808EB48084FEA4803FE
:10C3C00001EB41010493490089FB0138049B89FB7F
:10C3D00003394FEAA943B6F80E90B668089607EB02
:10C3E000870709EBC90907EB870602EB82024FEAD0
:10C3F00089070596079702EB8202049F864E0692F4
:10C400004FEAA848CA174FEADE7EBAF1050F86F850
:10C4100009E04FEAE77A824EA8EB02073A4606FBAC
:10C42000121205997FB207EB8109049FA3EB0A085A
:10C430004146794B06FB1878089F4FEADC7C80FB6D
:10C44000076E83F80EC04FEAE776069B754FDFF85C
:10C4500008C2C6EB6E1649B201EB830106F5FA730A
:10C460000493079BBCF800C0A7FB03376A4B1E462A
:10C4700083F813C0049B89B283F3100304934FEA3B
:10C48000112380FB02EA1FFA89F980FB08E005937B
:10C490004FEAE878049BDFF8C4E186F80A904FEA97
:10C4A000E272C8EB6010C2EB6A124FEA19284FEA39
:10C4B000971786F80B804FEA222AC3F30728059BBB
:10C4C0003374BEF800E0F1734FEA20294FEA1C2CC8
:10C4D0004FEA172134BF32233323327386F80DA07D
:10C4E0007074049886F81290707586F81680F7714B
:10C4F000317286F814C0F37686F81CE0039BC5F809
:10C50000F83258E4DFF85881D8F8000032F066FEBF
:10C51000C0B201280FD90228434F40F042837B79F3
:10C52000002B41F0F384D5F800330399BA68CB1A95
:10C53000934281F04F863D4A1668002E3FF46FAC5F
:10C5400099F80030002B7FF440AC394BD8F800004C
:10C550001B689B781E3B012B41F2D38438300221AB
:10C560002FF062F80122002389F8002085F81033AB
:10C5700052E47D2B01F0D08495F8162322B180F08F
:10C580002003DBB285F81613B5F8142395F81213BF
:10C590001A44062992B267D805EB010E60460131B4
:10C5A000A5F814238EF8D43185F8121332F016FE54
:10C5B00000287FF40EAE30E61E4D2A7832B11E4BB5
:10C5C0001E49186832F0DAFD00232B701C4E3578B6
:10C5D000002D7CD0DFF88C90D9F86030002B40F033
:10C5E0003182184B039A3470C3F8702441E500BFC0
:10C5F00070930020CDCCCCCCD48A002074C5002010
:10C60000F4970020AC9600201F85EB51BA930020D0
:10C61000A4930020B0D90020209800206BCA5F6B43
:10C6200040420F00D34D621088010020D8960020B0
:10C63000D4960020A8970020F89800206897002042
:10C64000FE980020D0170020676666666C93002075
:10C65000806967FF83DE1B436E930020181E002055
:10C66000D096002008990020D3B203EB1222FF2AB3
:10C6700087F81080A5F8142340F01B81604632F043
:10C68000ADFD9B48CAE5FF224FF6FF737AE5FFF741
:10C6900015FB984B1B68C01A40F6B833984200F25D
:10C6A0001B81954E33793A2B01F04384002388F89F
:10C6B000003098E4914B186832F084FD00283FF474
:10C6C00092AC022200236A7488F800308BE48C4C10
:10C6D0002278002A40F030818A4C94F82B51002DAA
:10C6E00040F06482884A89491268096891422DD8CD
:10C6F00094F82021002A41F0CD8494F82131002BB8
:10C7000041F07F8794F82231002B41F0CA8794F8DA
:10C710002331002B41F0C38794F82431002B41F0E2
:10C72000BC8794F82531002B41F0B58794F8263169
:10C73000002B41F0B88794F82731002B41F0A984F1
:10C7400094F828310825002B41F0A484704D714CD9
:10C75000D5F870242178704B93FBF1F31344039ABE
:10C760009A42FFF486AC114695F874346B4AC5F8CA
:10C770007014D65CF70744D5DFF8B8819FED688A5E
:10C78000B8F9023007EE903AF8EEE77A654B21935C
:10C7900067EE887A2AAFFDEEE77AA3F13D0247F80B
:10C7A000282D17EE902A91B240F6C80223F8402CAB
:10C7B0001E2203F83E2C38461EF0BEFEB8F90030AB
:10C7C00007EE903AF8EEE77A384667EE887AFDEEA3
:10C7D000E77A17EE903A99B21EF0AEFEB8F904303F
:10C7E00007EE903AF8EEE77A384667EE887AFDEE83
:10C7F000E77A17EE903A99B21EF09EFE38462FF077
:10C8000061F8B00701F1AA86710701F16A86330762
:10C8100043D5444B444F21932AAEA3F13D0246F841
:10C82000282D41F2C811022203F83E2C23F8401CA7
:10C83000304639681EF068FE304679681EF064FEA6
:10C84000FB89242101FB03F14FF0640830463231AB
:10C8500091FBF8F189B21EF06FFE3B8A03EB830374
:10C86000590089B230461EF067FE304B304A1B68D3
:10C870009342A8BF134623EAE37393FBF8F303F54F
:10C880007A7189B230461EF057FE209B3A7D591CC2
:10C89000209130461A702FF015F895F874342178ED
:10C8A000013393FBF1F201FB123385F87434FFF787
:10C8B000E0BB604632F092FC00287FF48AACACE426
:10C8C0000D2B7FF4A3AC6046A5F8142332F086FC50
:10C8D00000287FF47EACA0E40D4AB2F81E3300219C
:10C8E0000133A2F81E3388F80010FFF77CBB00BFAD
:10C8F000A41900202C9C0020149C0020549E002091
:10C90000FD9800208420002074C500203C310020C8
:10C91000D017002004990020A08601000099002073
:10C9200058A08B4168970020B0D90020AC96002019
:10C9300020A10700B4930020AE4EAF4B0093A6F1A8
:10C940003F01C827CDE91E1606F8407CAB4BAC4A28
:10C95000AC4920A81DF00EFF1E9E731C1E9335705F
:10C960001E9B2922591C1E911A701E9BEA22591CDB
:10C970001E911A701E9B5A1C1E9220A81F704EF00A
:10C9800051F8471C20A93A461E984EF0DBFF1E9A2C
:10C99000D31901331E93D5551E9B5A1C1E921D7030
:10C9A0001E9B5A1C1E921D701E9B5A1C1E921D70AF
:10C9B0001E9B5A1C1E921D701E9B5A1C1E921D709F
:10C9C0001E9B5A1C1E921D701E9B5A1C1E921D708F
:10C9D0001E9B5A1C1E921D701E9B5A1C1E921D707F
:10C9E0001E9B5A1C1E921D701E9B5A1C1E921D706F
:10C9F0001E9B5A1C1E921D701E9B012299182AA86C
:10CA00001E911A7050F8303D9B1B33702EF05AFF68
:10CA10007D4B039A2570C3F87024FFF72ABB2D22A3
:10CA2000DA766BE530688DF8789085F8129385F8A2
:10CA3000138387F8109032F0D1FB00287FF4C9AB44
:10CA4000FFF7EBBBDFF8E481002550270BE01D4426
:10CA5000EFF3118387F31288D9F86020954218DA32
:10CA6000DBB283F3118819F805A0681C51464844CD
:10CA700000222DF0FBFF0AF101030028E7D0414618
:10CA80003A202DF055FF0AF1010A0443E4B255445F
:10CA9000DEE70022DBB2C9F8602083F31188A0E54D
:10CAA0005A4B31681B78C5F8FC12013B012B41F24F
:10CAB0001E83574B1B78013B012B3FF61BAC162105
:10CAC00001239170137115E40CF10103614685F89F
:10CAD000117385F8103332F085FBFFF79DB94D4B8C
:10CAE0001B88DA0501F122825E0601F16F83D80707
:10CAF00001F1158413F0020F0CBF4FF0040A4FF040
:10CB00000C0A454A454B1678DB7806F001060BB156
:10CB100046F0020653202EF007F9414B1B8803EB29
:10CB20008303580080B22EF0E3F800202EF0E0F8E6
:10CB300037F09CFB3B4BC0EB002083FB00230344FE
:10CB40004FEAE079C9EB6329B9F1FF0FA8BF4FF0B5
:10CB5000FF095FFA89F94946386832F043FB98F8D3
:10CB60000030386889EA03094AEA0606002188F895
:10CB7000009032F037FB3146386832F033FB98F8DA
:10CB8000003038687340DBB2194688F8003032F064
:10CB900029FB95F81CA3FFF7DDB92EF07BFDFFF70D
:10CBA0003BB92EF067FD01237B71C4E4114B84F87F
:10CBB0002B212AA8A3F13A021B4940F8282D4FF453
:10CBC000327223F83C2C43F8401C21932EF07AFE5D
:10CBD0000D4B039AC3F87024FFF74BBA30688DF8F9
:10CBE000788087F8108032F0F9FA00287FF4F1AAF3
:10CBF000FFF713BB6897002093D500201455060853
:10CC00001C55060828550608D0170020C64B0020E2
:10CC1000D44B0020B09300203093002034930020A8
:10CC20007093002003082080C8057DEAF9B8030846
:10CC30006E4B95F83EE3B3F90220B3F90010B3F957
:10CC400004309FED6B6A85F8E19107EE103A694B6D
:10CC500085F8E0E11B6820938EF06A0383EA0313F2
:10CC600006EE901AD9B20B0983F0D50343EA0123EB
:10CC700083EAC1031BB283EA0311C3F307265342BD
:10CC8000C9B207EE903A86EA111646EA0126F8EE96
:10CC9000E77AF8EEE66AB8EEC77A86EAC10636B2F7
:10CCA00067EE867A66EE866A27EE067A002086F0C0
:10CCB000C80CCDED227ACDED216A8DED237A24903A
:10CCC000259026900DF180088CEA0C1CB8E80F0026
:10CCD0005FFA8CFCC6F3072686EA1C1646EA0C2689
:10CCE00086EACC06DFF814C136B2ACE80F0086F055
:10CCF0001E0398E8070083EA0313DBB2C6F3072696
:10CD000086EA131646EA03268CE807000EF10108AE
:10CD100086EAC303C822ACF110064FF005094FF0B4
:10CD20001E0E41F6FE4185F8E22185F8369385F81E
:10CD3000E3E1A5F8DE1106F11C0285F83E83A5F8B3
:10CD4000DC3116F8011B594081EA0111C9B208090A
:10CD500080EA132343EA012383EAC10109B28BB2BB
:10CD60009642A5F8DC31ECD181F0270181EA01116E
:10CD7000C9B21E0A86EA111686EA012686EAC106AB
:10CD800036B2B3B24FEA132AF6B2DFF86C90A5F8C8
:10CD9000DC3185F801A285F8006205F5EF7C05F528
:10CDA000FF78DCF80000DCF80410DCF80820DCF880
:10CDB0000C30CE46AEE80F000CF1100CC445F14625
:10CDC000EFD1DFF83C80BCF80030AEF8003008F15D
:10CDD000240985F88A6385F88BA318F8011F386841
:10CDE00032F000FAC145F8D1FFF731B9B493002011
:10CDF00088C3E43A74C50020381B0020B419002011
:10CE0000371B0020DFF87093D9F8003019229806FC
:10CE100085F832237FF511A9D14BD24E1B789907A3
:10CE200041F17382337D042B8CBF4FF0030A4FF026
:10CE3000020AFEF743FF338AB268209003EB8303B4
:10CE40005B00ADF89A3002EB820233682293F189DD
:10CE500096F814C073688DF89DC020A852004FF05A
:10CE600000084FF0FF3ECDF894E08DF89CA024928E
:10CE70002393ADF89810CDF8848084460590BCE8E3
:10CE80000F00DFF8F0E2AEE80F009CE80F00AEE81C
:10CE900007007146182221F81C39069195F83E13B7
:10CEA00085F8E32181F0780383EA0313DAB21309EA
:10CEB00083F0F60343EA022383EAC2031BB283EA48
:10CEC0000312D2B2C3F3072383EA121343EA022305
:10CED00083EAC2031BB283F0C80282EA0212D2B212
:10CEE000C3F3072383EA121343EA022383EAC2034C
:10CEF0001BB283F0180C8CEA0C1C5FFA8CFCC3F399
:10CF00000722481C82EA1C1242EA0C2285F83E03E2
:10CF1000069885F8E01182EACC0CC82341F6FE623F
:10CF2000014685F8E181A5F8DCC11E30A5F8DE21B7
:10CF300085F8E23111F8013B83EA0C0383EA03131D
:10CF4000DBB21A0982EA1C2242EA032282EAC30304
:10CF50001BB21FFA83FC8142A5F8DCC1EAD183F041
:10CF6000180383EA0313DBB24FEA1C2282EA13128E
:10CF700082EA032282EAC3031BB29AB27A49A5F875
:10CF8000DC21DBB2120A07910A92099385F8032289
:10CF900085F802328A4605F5EF7C05F5FF78DCF866
:10CFA0000000DCF80410DCF80820DCF80C30D64671
:10CFB000AEE80F000CF1100CC445F246EFD16B4BFC
:10CFC0000893DCF80000CEF80000099A85F88C235D
:10CFD0000A9A85F88D2303F126089A461AF8011F4C
:10CFE000386832F0FFF8D045F8D1FEF767FEB16837
:10CFF0008046D9F8000001EB810110F0140FD6E94A
:10D0000000324FEA410601F0B1815949096801EB4C
:10D0100081014900CDE90A2109932DF019FE95F807
:10D020003EA3ADF89A008AF06A0080EA00105FFA29
:10D0300080FC4FEA1C1080F0D50040EA0C2080EA0A
:10D04000CC0000B280EA001C5FFA8CFC0A9A0B99B3
:10D05000099BCDF88080C0F307204FF0000980EADB
:10D060001C10CDE92226CDE9241940EA0C2080EAE3
:10D07000CC00DDF814C02193ADF8989006B2BCE85E
:10D080000F0086F0C80888EA08185FFA88F8DDF80B
:10D0900018E085F8E191C6F3072686EA1816AEE88F
:10D0A0000F0046EA08269CE8070086EAC80636B262
:10D0B00086F0210383EA03138EE80700DBB22D4AD2
:10D0C0000692C6F3072686EA13160AF1010246EA1B
:10D0D000032185F8E0A185F83E23264A81EAC303AF
:10D0E000212641F6FE40C8219446A5F8DC311C32C9
:10D0F00085F8E361A5F8DE0185F8E2111CF8011B53
:10D10000594081EA0111C9B2080980EA132343EAB0
:10D11000012383EAC10109B28BB29445A5F8DC3141
:10D12000ECD181F0680181EA0111C9B21E0A86EAD8
:10D13000111686EA012686EAC10636B2B3B24FEA74
:10D14000132AF6B2DFF82080A5F8DC3185F801A2B9
:10D1500085F8006205F5EF7C05F5FF790EE000BF6C
:10D160006C930020B0D90020381B0020371B002012
:10D17000AC960020B41900200C890020DCF80000D7
:10D18000DCF80410DCF80820DCF80C30C646AEE809
:10D190000F000CF1100CCC45F046EFD1BCF800307C
:10D1A000AEF80030079B85F88A63089E85F88BA34C
:10D1B00003F1230816F8011F386832F013F8B04560
:10D1C000F8D1A44A95F83EC3DFF88C8285F8E0C117
:10D1D000D2E9002321938CF0EB0383EA0313D9B245
:10D1E0000B0983F0C50343EA012383EAC1031BB2A1
:10D1F00083EA0311C9B2C3F3072383EA111343EA95
:10D20000012383EAC1031BB283F0C80686EA06162F
:10D21000F6B24FF0000E2092C3F30723059ACDF823
:10D2200088E083EA161307CA43EA062383EAC603A3
:10D230000FFA83F9069B85F8E1E189F0310683E86E
:10D24000070086EA0616F6B2C9F3072383EA161327
:10D2500043EA062383EAC60395F8E46195F8E501FD
:10D2600095F8E61195F8E7211BB25E4086EA0616AE
:10D27000F6B2C3F3072383EA161343EA062383EACD
:10D28000C6031BB2584080EA0010C0B2C3F30723A4
:10D2900083EA101343EA002383EAC0031BB2594018
:10D2A00081EA0111C9B2C3F3072383EA111343EAE8
:10D2B000012383EAC1031BB25A4082EA0212D2B2AE
:10D2C000C3F3072383EA121343EA022383EAC20368
:10D2D00095F8E86195F8E90195F8EA1195F8EB21E0
:10D2E0001BB25E4086EA0616F6B2C3F3072383EA52
:10D2F000161343EA062383EAC6031BB2584080EAAA
:10D300000010C0B2C3F3072383EA101343EA0023DB
:10D3100083EAC0031BB2594081EA0110C0B2C3F3D3
:10D32000072181EA101141EA002181EAC00109B216
:10D330004A4082EA0212D2B2C1F3072383EA1213EF
:10D3400043EA022383EAC20395F8EC6195F8ED0104
:10D3500095F8EE1195F8EF211BB25E4086EA0616AD
:10D36000F6B2C3F3072383EA161343EA062383EADC
:10D37000C6031BB2584080EA0010C0B2C3F30723B3
:10D3800083EA101343EA002383EAC0031BB2594027
:10D3900081EA0111C9B2C3F3072383EA111343EAF7
:10D3A000012383EAC1031BB25A4082EA0212D2B2BD
:10D3B000C3F3072383EA121343EA022383EAC20377
:10D3C0001BB283F0270686EA0612D2B2C3F3072601
:10D3D00086EA121646EA022686EAC20636B2B2B2D9
:10D3E0000CF101034FEA122EF6B24FF0310C40F669
:10D3F000FE40C82185F83E33A5F8DC2185F8F061B0
:10D4000085F8E3C1A5F8DE0185F8F1E185F8E211C0
:10D41000D8F80C30D8F80000D8F80410D8F8082054
:10D42000B8F8109008F5C57CACE80F00079BACF885
:10D43000009085F87A63089E85F87BE303F1130872
:10D4400016F8011F386831F0CDFEB045F8D1FEF76F
:10D45000F4BD00BF48310020AE1900208849894A38
:10D460008978126809920A2285F82F23002900F092
:10D470008986854A012910880A9041F25A8350888A
:10D480000890022900F04F8790880790032901F047
:10D49000E983D0880690042901F0DE831089059085
:10D4A000052901F0D4830629B2F80A9001F0CB8354
:10D4B0000729968901F01483B2F80E8036F0D6FE63
:10D4C00095F83EA3099B20938AF0300383EA031367
:10D4D000DBB21A096D4985F8E0A182F07A02C0EB4F
:10D4E000002042EA032282EAC30381FB00210144B7
:10D4F000C217C2EB61220A994FF0000E61F30F0EC2
:10D5000007994FF0000C61F30F0C059900201BB236
:10D5100061F30F00002166F30F0183EA0316C3F3E2
:10D5200007230593089B63F31F4E069B69F31F4077
:10D5300063F31F4C68F31F41059BCDE921ECF6B264
:10D54000CDE92301FF2A83EA1613A8BFFF224FF07B
:10D5500000098DF895208DF8949043EA062C0DF182
:10D560008008B8E80F008CEAC60636B286F0C80E0E
:10D57000DFF81CC18EEA0E1E5FFA8EFEC6F3072688
:10D58000ACE80F0086EA1E1343EA0E2398E8030076
:10D5900083EACE031BB283F023024CF8040B82EA29
:10D5A0000210C0B2C3F3072282EA101242EA00223C
:10D5B0002CF8141982EAC0000AF1010A232641F26C
:10D5C000FE62C82385F83EA3A5F8DC010CF1160124
:10D5D00085F8E19185F8E361A5F8DE2185F8E2316F
:10D5E0001CF8013B434083EA0313DBB21A0982EAC9
:10D5F000102242EA032282EAC3031BB298B28C458E
:10D60000A5F8DC01ECD183F0F40383EA0313DBB269
:10D61000060A86EA131686EA032686EAC306D5F8C2
:10D62000E211D5F8E621D5F8DE01D5F8EA31DFF8C8
:10D6300064C0ACE80F0036B21FFA86F9D5F8EE01E7
:10D64000D5F8F211D5F8F621A5F8DC914FEA192E9C
:10D65000F6B2ACE8070085F8FA6185F8FBE105F25F
:10D66000673805F2853985F885E385F8846318F80D
:10D67000011F386831F0B6FDC145F8D1FEF7D5BCC1
:10D6800070D8002074C5002040DA002003082080F4
:10D69000B4190020381B0020CA4B1A6802F0080396
:10D6A000002B48F603414AF60B404BF60F4349F670
:10D6B000074604BF03460E4612F0040F18BF1E466D
:10D6C0009306C14B1B7848BF46F480464FF01901C2
:10D6D00048BF46F02006022B85F82E1340F2BB858A
:10D6E00064204FF0FF3A4FF0000995F83E832096F2
:10D6F00088F0F10282EA0212D2B2130983F0E70342
:10D70000C6F3090143EA0223CDE9216183EAC2039A
:10D710004FF0000E1EB2ADF88E90ADF890A08DF8CF
:10D720009E00ADF88CE0CDF892E0CDF896E0CDF813
:10D730009AE086EA06190DF1800CBCE80F005FFA4A
:10D7400089F9C6F3072686EA191646EA092686EA03
:10D75000C906DFF8949285F8E1E1A9E80F0036B236
:10D760009CE80F0086F0C80C8CEA0C1C5FFA8CFC5D
:10D77000C6F3072686EA1C16A9E8070046EA0C212C
:10D7800081EACC0109B281F0010080EA001029F899
:10D79000023BC0B2C1F3072282EA10121B0C09F847
:10D7A0001E3942EA0022012682EAC00041F6FE71DB
:10D7B000C82208EB0603A5F8DE1185F8E36185F8B9
:10D7C000E22109F11F0185F8E081A5F8DC0185F867
:10D7D0003E3319F8013B434083EA0313DBB21A09D5
:10D7E00082EA102242EA032282EAC3031BB298B201
:10D7F0008945A5F8DC01ECD183F07C0383EA0313AF
:10D80000DBB2060A86EA131686EA032686EAC30610
:10D8100036B2B3B24FEA132AF6B2DFF8D091A5F8C8
:10D82000DC3185F804A285F8036205F5EF7C05F587
:10D83000FF78DCF80000DCF80410DCF80820DCF8E5
:10D840000C30CE46AEE80F000CF1100CC445F1468A
:10D85000EFD1DCF80000CEF80000DFF894819CF8EE
:10D8600004308EF8043008F1270985F88D6385F8B7
:10D870008EA318F8011F386831F0B4FCC145F8D107
:10D88000FEF7CBBBFF202CF0AFFE002800F0418557
:10D890000378FF2B00F0408590F9011002202DF055
:10D8A00015FFFF202CF0A0FE002800F0688403780C
:10D8B000FF2B00F06484B0F90C304449444A897E5F
:10D8C00003EB830303EB830349089B0093FBF1F312
:10D8D00082FB0312D917C1EBA20109B23D4F03200D
:10D8E0002DF0F4FE7B7A002B40F0EB84D9F8003069
:10D8F0009A0640F159844FF400502EF01DF800288C
:10D9000040F03785344E4FF480602EF015F8002833
:10D9100040F07986718A95F8F022337DB1F5967FD3
:10D9200008D902F00F02072A04D842F20F738B4283
:10D9300028BF0B46294FFA79CAB1203B07EE903A2F
:10D940009FED277AF8EEE77AF6EE006A67EE877ABF
:10D95000BEEE007AF5EEC07AF1EE10FA58BFB0EEE6
:10D96000667A77EE877AFDEEE77A17EE903A052031
:10D9700019B22DF0ABFE4FF480502DF0DDFF0028E2
:10D9800040F0168595F8F062FEF776BC4FF4007013
:10D990002DF0D2FF00283EF46BAC16F003077EF4A6
:10D9A00067AC104A0A23B2F9041091FBF3F114207A
:10D9B0002DF08CFE39461C202DF088FE95F8F06283
:10D9C000FEF756BC0C8900207220002078BA002097
:10D9D0006766666688930020B0D90020D48A00204C
:10D9E000E4380E3FB4930020B4190020381B002007
:10D9F000371B00208A4B1B68052285F837239A06BF
:10DA000003F0140140F1C883864BDFED877ADA8991
:10DA100008EE902AF8EEE88A68EEA78A002900F05E
:10DA2000FA85824BDFED807A93ED008AB8EEC88AE2
:10DA300028EE278A2DF00CF995F83E937C4BADF833
:10DA40009000B3F906607B49CDED218A89F022036D
:10DA500083EA0313DAB21309B6F5FA6F83F05903B8
:10DA6000A8BF4FF4FA6643EA022383EAC203B6F57D
:10DA70007A7F1BB2B8BF4FF47A76A6F57A7C83EA38
:10DA800003126420D2B2C3F3072600FB0CF386EA2C
:10DA90001216A1FB03134FF0000E20A946EA02263E
:10DAA000C3F38F13CDF880E0CDF88CE08DED228AA2
:10DAB00086EAC206ADF892308A4636B20591BAE8D7
:10DAC0000F0086F0C80C8CEA0C1C5FFA8CFCC6F3C5
:10DAD0000726DFF878E1DAF800A085F8E09186EA19
:10DAE0001C16AEE80F0046EA0C2686EACC0212B2FB
:10DAF00082F04A0383EA03137146DBB2C2F30722C2
:10DB000082EA131241F810A942EA032282EAC3030F
:10DB100009F101094FF04A0E41F2FE4C0026C820DF
:10DB200006910A4685F83E93A5F8DC31143185F854
:10DB3000E3E1A5F8DEC185F8E16185F8E20112F8BC
:10DB4000010B584080EA0010C0B2060986EA132390
:10DB500043EA002383EAC00000B283B28A42A5F8F8
:10DB6000DC31ECD180F0140080EA0010C0B21E0A53
:10DB700086EA101686EA002686EAC00636B21FFA42
:10DB800086FC2D4BD5F8E211D5F8DE0107934FEA5C
:10DB90001C2ED5F8E621D5F8EA31A5F8DCC1DFF86E
:10DBA00098C0B5F8F6A185F8F9E1ACE80F00D5F812
:10DBB000EE01D5F8F211ACE80300F6B205F26739D0
:10DBC000ACF800A085F8F86185F88263CA4685F84C
:10DBD00083E305F283361AF8011F386831F002FB3F
:10DBE0005645F8D1154B164A1B781278013B12F0B6
:10DBF0000101DBB214BFC0224022172B03D8114809
:10DC0000034493F85C8C104B1B889B071ABF42F0AF
:10DC1000100200230123002940F02C83032017E089
:10DC20000C890020B0D900200AD7233CAC960020F4
:10DC300040DA0020D34D6210381B002054480020E9
:10DC40003093002038D00508B0930020B41900208C
:10DC500095F83EA320938AF0460383EA0313D9B2D2
:10DC60000B0983F0920343EA012383EAC1031BB249
:10DC700083EA0311C9B2C3F3072686EA111646EAFE
:10DC8000012686EAC10636B286F0C80C8CEA0C1C66
:10DC90005FFA8CFC00238DF886200321059A8DF80D
:10DCA0008480C6F307268DF885308DF887008DF8BF
:10DCB000881086EA1C1607CA46EA0C2686EACC06B5
:10DCC00036B2DDF818E085F8E33186EA061CAEE8E6
:10DCD00003005FFA8CFCC6F3072181EA1C1141EABC
:10DCE0000C2181EACC0195F8E4C18EF8002009B23C
:10DCF0008CEA010C8CEA0C1C5FFA8CFCC1F3072245
:10DD000082EA1C1242EA0C2295F8E56195F8E601D8
:10DD100095F8EBE185F8E13182EACC0212B2564087
:10DD200086EA0616F6B2C2F3072181EA161141EA25
:10DD3000062181EAC60109B2484080EA0010C0B25B
:10DD4000C1F3072282EA101242EA002282EAC002EC
:10DD500095F8E7C195F8E86195F8E90195F8EA11B9
:10DD600085F8E0A112B28CEA020C8CEA0C1C5FFA76
:10DD70008CFCC2F3072282EA1C1242EA0C2282EADD
:10DD8000CC0212B2564086EA0616F6B2C2F3072259
:10DD900082EA161242EA062282EAC60212B2504013
:10DDA00080EA0010C0B2C2F3072282EA101242EAEF
:10DDB000002282EAC00212B2514081EA0111C9B2C6
:10DDC000C2F3072282EA111242EA012282EAC10268
:10DDD00012B28EEA020E8EEA0E1E5FFA8EFEC2F3B9
:10DDE000072282EA1E1242EA0E2282EACE0295F849
:10DDF000ECE1C24E13B28EEA030282EA0212D2B200
:10DE0000C3F3072383EA121343EA022383EAC2031C
:10DE10001BB283F0320282EA0212D2B2C3F30723AA
:10DE200083EA121343EA022383EAC2031BB299B2C4
:10DE300040F6FE18C8204FEA112C0AF10102DBB2AD
:10DE4000A5F8DE8185F8E20185F83E2385F8EEC16C
:10DE500085F8ED313068B268A5F8DC117168B6F864
:10DE60000CA006F5C57607C6079A86F802E0A6F864
:10DE700000A002F1100885F878C385F8773319F807
:10DE8000011F386831F0AEF9C845F8D1FEF7E9B89E
:10DE90004FF400602DF050FD28B1994B3020B3F9BC
:10DEA00000102DF013FC95F8F062B00700F0E98146
:10DEB000D9F80070FEF7D9B970202DF03DFD00288B
:10DEC0003EF4CDA98F4F2426A7F15008B7EC017A74
:10DED000D8ED007A67EE277A3046FDEEE77A013614
:10DEE00017EE903AC3EB431103EB8103D90009B25B
:10DEF000F6B22DF0EBFB272EE8D1D9F80070FEF733
:10DF0000AEB9022131F05AF9FEF72CBB039BC5F8DC
:10DF100000337E71FEF70FBB604685F8168331F043
:10DF20005DF900287EF455A9FEF777B9B246FEF7F1
:10DF3000E8BDB178304637F0B5F900287EF4B6ABCD
:10DF4000714B186831F04AF900287EF447A86F4FEA
:10DF50006F4DF378BA7C059395F82033049304232E
:10DF600007927B74002A00F04F84FE7C694BDFF837
:10DF7000BCA10136F6B206EB460903EB8909F3B200
:10DF8000152B31465046FB7406F1010600F2AB85B5
:10DF90001CF034F928B999F80830FF2B09F10C0965
:10DFA000EDD1FB7CDFF87C911A465B4B06920C2688
:10DFB00006FB0236D6F8481B089108464CF032FDA5
:10DFC000D6F84C3B0793C6B218464CF02BFD5FFACF
:10DFD00080FA069B089906EB0A02083203F00F0C40
:10DFE0000AEBC60089F8072023F00F0289F80A20FF
:10DFF00089F80DC0324689F80E0009F10F004DF086
:10E00000A1FC079B06F10900194609F106035246D7
:10E0100018444DF097FC99F8072002F1010AC2B1AB
:10E02000013A09F1070E3D4B5EFA82FE09F1060640
:10E03000002216F8011F51408A00C80882EA4102F6
:10E0400000F018004A4043FA00F14A40B645D2B207
:10E05000EFD1334B05980AF803204BF0C5FABB7C8F
:10E06000013B5FFA83FA87F812A0BAF1000F00F0C3
:10E070005E83049E244B99F802201868294931F0E8
:10E080007DF8032385F820637B7488F80030FDF762
:10E09000AABF0725244B94F82A2121932AAFA3F184
:10E0A0003901A3F1400647F8281DC821101D03F8C7
:10E0B000401C4FF4E4734EF67D2170707180384639
:10E0C00002FB0541B380B5711DF014FA209B721C50
:10E0D0009B1A737038462DF0F5FB63190C4A00212A
:10E0E00083F82011039BC2F87034FDF7C2BF1021E2
:10E0F000022391701371FEF7FDB800BFAE19002026
:10E10000BA930020DC110010549E002088010020EA
:10E11000D017002080DB050838D005080007090E5D
:10E120008ED9002088D9002068970020C89600204A
:10E13000B54AB64B1668B64FA3FB06239B0BA7FB4D
:10E1400003214909C1EB0111A3EB8103190209B2B3
:10E150000023172085F8F0322DF0B8FAAD4BA3FB61
:10E1600006239B09A7FB03125209C2EB0212A3EB81
:10E17000820319B218202DF0A9FAFEF780B8002109
:10E18000FFF7ACBB0E468946CDE90511CDE9071175
:10E190000A918846FFF792B9DFED9F8A00297FF444
:10E1A00040ACB0EE688A45E419077FF5EBAB9B4BBA
:10E1B00093E8030020AB83E8030018462DF09EFA95
:10E1C000FFF7E0BB01230593FDF78DBE4FF0100A6A
:10E1D000FEF797BC0126D8F800007E7130F0F6FFFC
:10E1E0000490D8F8000030F0F1FF049B5A068246F4
:10E1F00000F0A180802800F027827F2B7EF49BA96D
:10E20000874A1378002B00F0BB840AF0F003E02B60
:10E210007EF491A995F80923824E0AF00F0A002A8C
:10E2200000F090840022737085F809237E4F3B78BC
:10E23000002B00F0C584AAF1070ABAF1070F00F21B
:10E24000BB84DFE81AF0E104B904B204B904F204B3
:10E25000B904EE046804754A537A927A002B40F0B0
:10E26000BD81002A40F04584914664204FF0FF3A7A
:10E27000FFF73BBA6E49C97800290CBF042005207E
:10E28000E6E44FF480602DF057FB00283FF410AE19
:10E29000684A694B1768D5F8EC224FF064089A4237
:10E2A00098BF0027102097FBF8F631B22DF00EFA38
:10E2B00008FB167109B221202DF008FA95F8F062DA
:10E2C000F6E501202DF038FB002840F0C380BB7A32
:10E2D000002B3FF40BAB02202DF02EFB002840F06A
:10E2E000658204202DF028FB00283FF4FFAABB899B
:10E2F000002B40F06B82514B996881F3100109B2F9
:10E3000004202DF0E3F9FFF7F1BA4FF0010AFEF710
:10E3100090BD0146FFF7C2BA3946FFF7BFBA4FF0CA
:10E32000080AFEF7EEBB1E469946CDE90533079372
:10E330009846FFF7C3B83A4B1A78002A40F0898113
:10E34000BAF18A0F00F06F81BAF18E0F7EF4F3A854
:10E3500099F80030002B7DF435AD394A394B136004
:10E360002D2385F808331668FEF7EAB83146FEF724
:10E3700051BE354B1B789B0700F1A7814FF480609D
:10E380002DF0DAFA314E00283FF4C4AA4FF000080D
:10E390004FF06409012098FBF9F739B22DF096F996
:10E3A00009FB178109B209202DF090F9FFF7B2BAE5
:10E3B000254B1A7800239007CDE91E3300F15F81C9
:10E3C00095F8F432012B00F05A81B7F90030DFEDF7
:10E3D000206A07EE103AB7F9023007EE903AB8EE2D
:10E3E000C77AF8EEE77A27EE267A67EEA67ABDEED0
:10E3F000C77AFDEEE77A20A88DED207ACDED217A5F
:10E400002DF07CF9FFF7BEBA74C5002073B2E74562
:10E4100089888888D34D62100000000078DB0508E9
:10E42000333400204C980020DF9600208893002091
:10E4300034930020AC9600203F4B4C00A493002066
:10E44000D8960020F49700206C930020B0D90020CB
:10E450000050C347DFF82C83BC4E98F80020002AF8
:10E4600040F0C2811346110189B241EA0321C3F38E
:10E470000323194309B20620A5F8F2222DF026F94C
:10E48000B348B5F8F2123388067A98F80020C07ABB
:10E490000131012E03F105034FF00A0CA5F8F21229
:10E4A00093FBFCF399B200F0958101EB81039EB2DE
:10E4B00010B10AB196FBF2F64FF0640A3A20B6FBAF
:10E4C000FAF80FFA88F12DF001F90AFB186189B208
:10E4D0000A2305313B2091FBF3F109B22DF0F6F848
:10E4E000F5E69C4BDFF8C0822193C82223F8402C2C
:10E4F00098F80020A3F140073D3B2093D2074FF04E
:10E500002103BB7040F10281934B1B88580500F139
:10E51000CC80190500F1F880DA0500F1F380D80706
:10E5200000F18F83990740F184838C4920AB184612
:10E5300005931CF0CFFF98F80030DA0740F14081D6
:10E54000209B874A0598591C209100211970209B17
:10E550009B1A7B702DF0B6F9FEF759B97D4B7C4ABA
:10E560007A49D27A219340F6C82023F8400C08203B
:10E5700003F83E0C3D3B20930B88002A40F0978027
:10E5800020A805330A2193FBF1F189B205901CF014
:10E59000D3FFDDF81480734F0A223B6893FBF2F33C
:10E5A000404699B21CF0C8FF26F038FEBF68209B99
:10E5B0003A0C591C20911A70209B3A0A591C209140
:10E5C0001A70209B5A1C20921F70209B5A1C20926C
:10E5D000187040462DF076F9FEF716B95B4B1B8894
:10E5E00003EB83034FEA43091FFA89F9002A00F07D
:10E5F00087825C4BB3F900A026F010FE40B2FFF713
:10E6000074B8012546E5584B1B789F077FF5BEAED1
:10E61000D6F80880BCE693ED028AB8EEC88A28EEE8
:10E62000278AFFF707BA514B1B689E067DF583AF1B
:10E6300099F80030002B7DF4C5AB4D4A4D4B13606B
:10E640002D2385F808338EE64B4B1A78002A3DF4CB
:10E6500072AFD5F80423002A08DD48480A2AB8BF5B
:10E660000A220021C0F85024C5F804134FF47A623E
:10E6700040F6B831BA600022F9601A7060E6D6E957
:10E68000002301211EA885F8F412CDE91E232DF0E8
:10E6900035F8FFF777B90525FCE40425FAE40325EE
:10E6A000F8E40225F6E40625F4E435493EE7354A68
:10E6B00020A8117893FBF1F10A23053191FBF3F1C6
:10E6C00089B205901CF038FF63E72F4E2F4BF1897C
:10E6D0004FF4F36707FB01F1112091FBF3F109B24D
:10E6E0002CF0F4FFF389642107FB03F393FBF1F3B0
:10E6F00093FBF1F201FB123109B219202CF0E6FF75
:10E70000FFF701B9224911E722490FE7224B1B68A5
:10E71000D3B9DBF800301B067FF5F6AE124B1B7841
:10E7200003F00303032B3FF4EFAE1C49FEE6DBF8D6
:10E7300000301B4A190616787FF59CAC50462CF029
:10E7400065FF87F814A095E41649EFE67093002062
:10E75000D48A002068970020B09300200455060852
:10E7600029970020A49300206C9300200C8900209E
:10E77000D896002020980020333400200C1100206F
:10E78000E854060876930020B0D90020A086010046
:10E79000F4540608F0540608B4960020E054060825
:10E7A000CC960020D854060830930020BB4A0A2398
:10E7B000116891FBF3F1282009B22CF087FF90E556
:10E7C000209B2A22591C20911A70B9E626F026FDBA
:10E7D00001B295E518B112B193FBF2F399B209B207
:10E7E00039202CF073FF72E5B5F8F202338890FB04
:10E7F000F2F14FF0640C02FB11010CFB03235000FB
:10E800008AB2B3FBF0F32EE6A54BA64E1A8B93ED1E
:10E81000167AD3ED157A93ED145ADFF8B4A2716825
:10E82000DFF8B0E2D6F800C09F48BEF800E0DFEDA8
:10E830009F5ADFF8A49206EE102A984A136892684D
:10E840001D92B2681792328A1692F2891392327D23
:10E850000E92BAF900201592B8EEC66A944A069351
:10E8600012881492C7EE066A924A934BB2F90020BE
:10E870000D92B3F904200C92B3F902200B92B3F974
:10E8800000200A928D4A12681C9287EE867A4A14FA
:10E890000029B8BF49428CEAEC7302F480424FEA87
:10E8A0006C46A3EBEC7342F40052B1FBF0FC00FBAE
:10E8B0001C1106F4804A099142EA0C02C5EE067A60
:10E8C000B3FBF0F100FB113304984AEA010192B264
:10E8D000062600F0F00C89B21092099A12910CF100
:10E8E000100A66EEA56A4FF47A7106FB03F30698E8
:10E8F000B3FBF1F39BB2CDF820A006FB02F211931B
:10E90000B2FBF1F2FDEEE66A93B20EFB00F00F935C
:10E910000EF1050E90FBF1F327EE257A09930A23F9
:10E920009EFBF3F31B939DF82030089316EE903A6C
:10E93000BDEEC77A1BB267EEA57A1A9317EE103AAE
:10E94000FDEEE77A1BB2199317EE903A049E89F810
:10E950000AC01BB209F10D0A18933046089B834286
:10E960005ED9574B0C2202FB0032431E92F8506BCB
:10E9700046EA00128AF800200AF10101142B00F285
:10E98000A481DFE813F0A0019E019C019A01980187
:10E9900096019401920190018E0185017C017A011A
:10E9A00078017601A201C600C400C200C0001500B3
:10E9B0001A9B434A324492F8502C012A0DD9023A4C
:10E9C000D2B202F1020CE2448C460CF8013BD44571
:10E9D0004FEA1323F9D101321144092EDBB201F1C0
:10E9E000010A08D0364A0C2606FB002223F06003F9
:10E9F00092F8512B13430B702CF0EEFD314BAAEB28
:10EA00000302049B83420BD22D490C2303FB00130A
:10EA100093F8503B0B4493F8503C1344102B9DDD6E
:10EA2000284BDFF8B8E0AAEB03010631C9B241F088
:10EA30004003064689F8073001F1010A0020079BD0
:10EA400012E09CF807C083EA0C0C4FEA8C034FEAF3
:10EA5000DC0283EA4C0302F0180283EA0C034EFA4C
:10EA600002F253400130DBB2C2B2914209EB000C1A
:10EA7000E7D8154A05980AF802304AF0B5FD3B7D03
:10EA8000002B7FF4F7AA114B1B689A067FF5F2AAB8
:10EA90002CF096FD01233B75FFF7ECBAA493002000
:10EAA0008C110010B0D900208096980000007A44A4
:10EAB0006E930020BA930020B4930020AC960020FF
:10EAC00038D0050895D900208ED900200C89002067
:10EAD000181E00207093002088D900200007090E1E
:10EAE0009846FEF7EBBC162B04BF0023FB74FFF720
:10EAF00058BA774A9946B2F900A06420FEF7F5BDEE
:10EB00004FF0FF3A78E5199B53E7189B51E7179BA5
:10EB10004FE7169B4DE704204CF098FE99F8003023
:10EB2000002B7DF44FA96B4AAD23166085F808339E
:10EB300019E41E469946CDE90533CDE907339846D9
:10EB4000FEF7BCBC7378012B7FF470ABAAF1070A07
:10EB500085F80933BAF1070F2ED801A353F82AF02C
:10EB6000FDEB0008B9EB0008A9EB0008B9EB0008C1
:10EB70002BEC0008B9EB000823EC000817EB0008A9
:10EB800020A804924CF0A0FE5348049A4FF47A73E4
:10EB900041F28831C0F85034FB60239B1670C5F8F1
:10EBA0000433B960FFF731BB4C4F3B7823B14C4B7A
:10EBB0000121186813F018F800204CF047FEADE76B
:10EBC0004848AAF1070A0DF0FDFB0CF0D1FD73785F
:10EBD000BAF1070FF0D801A252F82AF011EC0008A0
:10EBE000B9EB0008ABEB0008B9EB00082BEC000810
:10EBF000B9EB000823EC000817EB000803204CF0E9
:10EC000025FE0CF0B5FD89E703204CF01FFE85E7DB
:10EC1000032004934CF01AFE049B012B7FF47EAF7B
:10EC2000EFE702204CF012FE78E701204CF00EFED8
:10EC300074E72D4B2D491A782D4B002A08BF194631
:10EC400074E42C4972E41E469846FEF737BC1E4613
:10EC500099469846FEF732BC1E469946059398465B
:10EC6000FEF72CBC1E469946CDE905339846FEF7C3
:10EC700025BC159B9DE6149B9BE6139B99E6119B77
:10EC8000A5F82433129BA5F82633D5F8243390E653
:10EC90000F9BA5F82433109BA5F82633D5F8243311
:10ECA00087E60E9B85E60D9B83E60C9B81E60B9B1E
:10ECB0007FE60A9B7DE6099B7BE61D9B79E61C9B14
:10ECC00077E6069B75E61B9B73E64FF0FF3370E615
:10ECD000A4930020D89600200C110020DF9600207D
:10ECE000E0960020E497002095300020105506089B
:10ECF00008550608FC5406082DE9F04F754B1B78A3
:10ED0000013B012B83B040F2C780734B0093734AE1
:10ED1000734BDFF80092934280F0D980DFF8F881DE
:10ED2000CDF8049003F118069B464FF0010A6D4C94
:10ED3000258862197DB142450DD2052D0BD936F8D3
:10ED4000183C6188C3F30B0399426AD014462588A6
:10ED50006219002DEFD156F8101C58461CF01CFC0F
:10ED60004FF0000A5D4B0BF1180B9B4506F118069E
:10ED7000DDD3DDF80490FCF7F7F85B4AD37B012B79
:10ED800075D0022B6CD02024137852785748584DF8
:10ED90005849594E02EB021200EB420203EB4310BA
:10EDA00003EB40032A60554A01EB430314603360D0
:10EDB0003FF0C0FD524B30684FF0FF321A603AF01E
:10EDC000F1F93FF0D5FC4F4B009C1A8918794E4958
:10EDD000C4F87C14642303FB02F2C8210A4413FB29
:10EDE00000110023C9E90112C9E90333C9E9053358
:10EDF000C9E9073389F8243089F8253012F036FC48
:10EE000094F88214B4F880043DF076FB06F0FCFD23
:10EE1000304B1B78013B012B2BD9504603B0BDE88A
:10EE2000F08F637913F0030390D156F8101C94F817
:10EE3000049058461CF0B0FB36F8182CB9EB123F82
:10EE40008ED136F8143C56F8100CAA1FC3F30B03EE
:10EE50009A4204F10601A8BF1A464CF073FD81E7FF
:10EE60002A4B9B79002B0CBF202428248CE72824D4
:10EE70008AE7FCF723FF264B00991B68C1F8F400D2
:10EE8000C9F80C3002220123504681F8F02089F89D
:10EE9000253003B0BDE8F08FDFF87890FCF70EFF67
:10EEA000D9F80C300C49009103F2DC53022281F8AE
:10EEB000F020C9F80C30094A094B00F5B71000F5ED
:10EEC000587093420C46C1F8F400FFF427AF4FF09E
:10EED000010A50E770D80020D0170020E008000891
:10EEE00090010008024000088CD500208C340020DE
:10EEF000C0960020043E0020BC96002010000010A8
:10EF0000340C002034400020E830002078BA002083
:10EF100074C5002034930020008000082DE9F04FD4
:10EF20008DB0FCF721F8714B1B78013B012B40F2AF
:10EF3000BA806F4ADFF8DC916E4BB2F8742C6E4FDA
:10EF4000DFF8D481ADF80620A3EB090300934FF05E
:10EF5000030A0026CDE90866CDE90A66009BCDF8D4
:10EF600018900793D8F81030002BC0F2948001233A
:10EF70008DF82C30F323C8F80C300222BDF806308F
:10EF8000ADF8083002A906A81AF0EAFE022202A98A
:10EF90004FF6FF701BF04EFC584BBB42834629D204
:10EFA0001C46A58823888DF81560C5F30B05C3F3AF
:10EFB0000B00A91D1B0B0622ADF81010ADF81200B6
:10EFC00004A906A88DF814301AF0CAFE5846062285
:10EFD00004A91BF02FFCA16883462A4606A81AF054
:10EFE000BFFEA16858462A461BF024FC1834BC42D8
:10EFF0008346D6D3022203A906A8ADF80C601AF006
:10F00000AFFE022203A958461BF014FC40BAC343CA
:10F01000022204A906A8ADF810301AF0A1FE099842
:10F0200048BB0A989DF82C3033B968B1BAF1010A8F
:10F0300090D10520FCF7BCFBD8F8103043F000431A
:10F04000C8F810300028F1D199F80030AC2BF0D17D
:10F0500099F80130BE2BECD11BF006FC0028E8D05B
:10F06000224B1B78013B012B2FD9254B00221A7014
:10F070000DB0BDE8F08F08ABC0F1040200211844C8
:10F080004DF086FF0A9818B908A906A81AF0C9FD1C
:10F09000CDE90960C6E71B4BC8F8043003F188339B
:10F0A000C8F8043063E7FCF709FE174A1749D3682C
:10F0B00000F5B71000F5587003F2DC530224C1F8D4
:10F0C000F40081F8F040D36033E7FCF7F7FD104916
:10F0D0000E4A0D4B0C68C2F8F4000121022082F8A0
:10F0E000F000DC6083F82510BFE700BF70D8002077
:10F0F00038D0050800800008E008000890010008EA
:10F10000D88000202301674534930020D0170020C9
:10F1100074C5002000400008003C024008B5064BC2
:10F1200002229A73FFF7FAFEFFF7E6FD0120BDE821
:10F13000084015F0F7BA00BF8CD500202DE9F04744
:10F14000CE4C2DED028BA36820469847002800F096
:10F15000D480CB4B1B780122042B84F85C2000F078
:10F16000D080B4F91A3006EE903AB4F91C3007EEAC
:10F17000103AB4F91E3007EE903AF8EEE66AB8EEAF
:10F18000C77AF8EEE77AC4ED146A84ED157AC4ED17
:10F19000167ABC4B1B88002B60D0BB4B94ED142A15
:10F1A000D4ED152A94ED163A93ED008AD3ED054A75
:10F1B00093ED090AD3ED0E3AD3ED120A93ED174AF7
:10F1C00093ED011A93ED065AD3ED0A1A93ED0F6AE7
:10F1D000D3ED137A93ED187AD3ED045AD3ED0D6A7B
:10F1E000E8EE024AE0EE223AA3EE204AA1EE025AED
:10F1F000A1EEA26AA3EE277A93ED038AD3ED167AE5
:10F2000093ED020AD3ED0C0A93ED0B1AD3ED151A08
:10F21000C4ED144A65EEE45AA8EE645A66EEE36A59
:10F22000D3ED144A83ED055A67EEC47AE0EE025A34
:10F23000A0EEE36AE1EE226AA4EE617AE3EE247ABC
:10F24000C3ED065AC4ED153A83ED0E6AC3ED0F6A9D
:10F2500083ED177AC3ED187A84ED164A94F82210DC
:10F2600009296BD0894810F06FF8894E894D328892
:10F27000D5F87C34002A40F02781874A126852076B
:10F2800000F1BF80B3F9002094ED156A94ED167A71
:10F2900094ED145A814905EE902AB3F90220B3F98E
:10F2A000043006EE902A07EE903AF8EEE55A7C4BD1
:10F2B0000A68D3ED003A93ED014AD3ED024AF8EE25
:10F2C000E66AF8EEE77A75EE655A76EE666A77EEEC
:10F2D000677AC4ED145A34EE266A73EEA55A34EEFA
:10F2E000A77A0132C3ED005AC4ED156A83ED016AB5
:10F2F000C4ED167A83ED027A0A60BDEC028BBDE89C
:10F30000F087B4F91A00B4F91C10B4F91E20654B4B
:10F3100007EE900AF8EEE76A07EE901AB8EEE77A81
:10F3200007EE902AF8EEE77AC4ED146A1880598047
:10F330009A8084ED157AC4ED167A2AE794ED157A51
:10F34000D4ED0D6AD4ED0E7A94ED0F2AD4ED145A53
:10F35000D4ED0A2A94ED0B3AD4ED0C3A94ED166AEA
:10F3600094ED104AD4ED114A94ED125A4E4B67EECB
:10F37000266A67EE277A27EE027AE5EEA26A1B7804
:10F38000E5EE837AA5EEA37AE6EE046AE6EE247A49
:10F39000A6EE057AC4ED146AC4ED157A84ED167AEA
:10F3A000002B7FF462AF414B93ED046AD3ED035A17
:10F3B00093ED052A93ED013AD3ED002AD3ED023AFD
:10F3C00093ED064AD3ED074A93ED085A27EE866A75
:10F3D00067EEA55A67EE827AA6EE836AE6EEA25A37
:10F3E000E6EEA37AF0EE466AE7EE045AE7EE246A08
:10F3F000E7EE057AC4ED145AC4ED156AC4ED167A29
:10F4000033E72B4E3288322A00F0F180002A40F098
:10F410003D8128480278002A3FF434AF264ED5F8C3
:10F42000A424D5F8A074D5F89C1486FB02ECD2175E
:10F43000C2EB2C12B4F818C0A2EB0C029A8086FB27
:10F44000012C86FB0726FA17C2EB261200271B4E5B
:10F450000770C917C1EB2C11194819805A80022373
:10F460007781B7818373FFF759FDFFF745FC0120D2
:10F4700015F058F9D5F87C3404E700BF8C11001062
:10F4800061BA0020E0440020E4440020DC110010B8
:10F4900080780020D01700208CD80020F8A200200F
:10F4A000FCA2002064BA002051020020F048002095
:10F4B000327E0020307E00201F85EB51E43000209A
:10F4C0008CD5002000000000B2F5C87F18BFD5F829
:10F4D000842494ED147A0EBF5FED067A07EE902A2D
:10F4E000F8EEE77A4FF0000C77EE877A0020C4F848
:10F4F00050C0FDEEE77A1880378817EE902AB7F5EE
:10F50000C87FC5F884245BD0D5F8881494ED156ABB
:10F51000D4ED166AC4F854C007EE901AD5F88C14CE
:10F520005880B8EEE77A07EE901AF8EEE77A37EEF1
:10F53000067A77EEA67ABDEEC77AFDEEE77A17EE89
:10F54000108A17EE901A012FC4F858C0C5F88884A5
:10F55000C5F88C14988030D1DFF890C1B4F818E069
:10F56000C8318CFB01A9C917C1EBE911C83208F1F8
:10F57000C808A1EB0E0E8CFB02A95849A3F804E0C1
:10F580008CFB08ACD2174FEAE878C2EBE912C8EB63
:10F59000EC18DFF85CC11A80A3F8028002234881CE
:10F5A00088818CF80E30FFF7B9FCFFF7A5FB3846D1
:10F5B00015F0B8F83788D5F87C34013F37805CE621
:10F5C00094ED157AD4ED167AC4F854C0BDEEC77A1E
:10F5D000FDEEE77A17EE102AC5F8882417EE902A78
:10F5E0005880C5F88C24C4F858C09880E5E73B4A99
:10F5F0001968D2F80A20C5F898249FED397AB3F932
:10F600000420C5F89014A5F89424D4ED146ADFED15
:10F61000347A37EE267A0022C4ED147ABDEEC77A2A
:10F620001A80328817EE101A322AC5F89C1405D0B9
:10F63000D5F8A02407EE902AF8EEE77A94ED157A33
:10F64000328877EE877A0020FDEEE77A002117EE08
:10F65000907A322A6065C5F8A074598033D094ED51
:10F66000167AA065D5F8A404998007EE900AF8EE02
:10F67000E77A012A77EE877AFDEEE77A17EE900AAD
:10F68000C5F8A40409D0013A3280C2E6D5F89C241A
:10F6900007EE902AB8EEE77AB7E71248124B0170EE
:10F6A0000B201A7014F010FFD5F87C34D5F8902494
:10F6B0001A600A49B5F99474D5F898049F80328885
:10F6C000C1F80A00DFE7D4ED167AA065FDEEE77A0F
:10F6D000998017EE901AC5F8A414D4E7E4300020FE
:10F6E00000000000347E00202F7E00201F85EB519B
:10F6F0008CD500202DE9F84F8046274C274DDFF8A8
:10F70000A490274EFCF7DAFADFF89CE0DFF89CC003
:10F710004FF0100A4FF47A77DCF80430C3F3080393
:10F72000CBB9EFF31183B3B92368A9682268934278
:10F73000FAD132689142F7D8DEF8002007FB02FBCD
:10F74000ABEB0101B1FBF2F107FB03131B1A4345BD
:10F75000E2D3BDE8F88FEFF311818AF31288D5F870
:10F7600008B02B68DB0304D50123C9F80030D5F8B5
:10F7700008B02368D9F80020C9B281F31188DEF8F7
:10F780000010134407FB01F2A2EB0B02B2FBF1F2F3
:10F7900007FB0323DAE700BF74C5002010E000E098
:10F7A0007CC5002070C5002078C5002000ED00E079
:10F7B0002DE9F04FDFF834C1494CDFF834E1DFF8D0
:10F7C0003481484E824648481AF1FF3AC0F086809C
:10F7D000DCF80430C3F30803002B5ED1EFF3118390
:10F7E000002B5AD10568A26803689D42FAD133689C
:10F7F0009A42F7D8DEF800704FF47A7101FB07F3F4
:10F800009B1AB3FBF7F301FB0535DCF80430C3F3B7
:10F8100008034FF010094FF47A77F3B9EFF311832F
:10F82000DBB90368A16802689342FAD13268914259
:10F83000F7D8DEF8002007FB02FBABEB0101B1FBC0
:10F84000F2F107FB03135B1BB3F57A7FBCD2DCF844
:10F850000430C3F30803002BE0D0EFF3118189F3E8
:10F860001288D4F808B02368DB0304D50123C8F854
:10F870000030D4F808B00368D8F80020C9B281F38A
:10F880001188DEF80010134407FB01F2A2EB0B0213
:10F89000B2FBF1F207FB0323D5E7EFF3118310224C
:10F8A00082F31288A1682268D20303D50122C8F826
:10F8B0000020A168D0F80090D8F80050DBB283F3A4
:10F8C0001188DEF800704FF47A724D4402FB07F3A2
:10F8D0005B1AB3FBF7F302FB053596E7BDE8F08F43
:10F8E00010E000E07CC5002074C5002000ED00E0C1
:10F8F00078C5002070C5002008B5012100202FF038
:10F900009DFF012108462FF099FF012102202FF0D1
:10F9100095FF114B1B7803F00503052B18D0002130
:10F9200008462FF08BFF002101202FF087FF0021D8
:10F9300002202FF083FF3220FFF73AFF00202FF044
:10F94000E1FC01202FF0DEFC02202FF0DBFCF2E7CF
:10F950003CF02EF9E3E700BF2C81002030B4EFF338
:10F960001183102282F31288084809490268094D60
:10F97000094C013202608A682A6000222260DBB2F0
:10F980000A6883F3118830BC704700BF74C500203B
:10F9900010E000E07CC5002070C500200E4B1B88E5
:10F9A000014643B90D4B0E4A1B7810680BB981F024
:10F9B00001012FF029BF0B4B5A691AB11A6810B90F
:10F9C00010605874704708480849008891FBF0F1AE
:10F9D00001201160587470474CC500204EC50020AE
:10F9E00050C5002054C500206CC5002020A1070090
:10F9F00038B52C4B5C69226C636E002A30D0626C87
:10FA0000C2B1998A1A88CD0792B204D5100744BFB3
:10FA10004FF6F7721A8099891A88C90692B201D5F1
:10FA2000D20600D438BD626B0AB19047636E1A8863
:10FA30009B8838BD99891A88090692B2E1D51206C9
:10FA4000DFD5D4E909128A4218D0A1692569885CFA
:10FA500098800132B2FBF5F105FB1122A262D0E7DA
:10FA600099891A888D0692B2C9D59006C7D5E26ADF
:10FA70004AB19888216B9047636EC0E7DA6822F03C
:10FA80008002DA60BDE79B88E2696169DBB28B5472
:10FA9000E269E068636E0132B2FBF0F100FB112213
:10FAA000E261ACE76C11001038B52C4B9C68226CFD
:10FAB000636E002A30D0626CC2B1998A1A88CD0771
:10FAC00092B204D5100744BF4FF6F7721A80998995
:10FAD0001A88C90692B201D5D20600D438BD626B2D
:10FAE0000AB19047636E1A889B8838BD99891A8835
:10FAF000090692B2E1D51206DFD5D4E909128A428D
:10FB000018D0A1692569885C98800132B2FBF5F1B3
:10FB100005FB1122A262D0E799891A888D0692B25C
:10FB2000C9D59006C7D5E26A4AB19888216B90473B
:10FB3000636EC0E7DA6822F08002DA60BDE79B8876
:10FB4000E2696169DBB28B54E269E068636E01329D
:10FB5000B2FBF0F100FB1122E261ACE76C11001086
:10FB600038B52C4B1C68226C636E002A30D0626C56
:10FB7000C2B1998A1A88CD0792B204D5100744BF42
:10FB80004FF6F7721A8099891A88C90692B201D580
:10FB9000D20600D438BD626B0AB19047636E1A88F2
:10FBA0009B8838BD99891A88090692B2E1D5120658
:10FBB000DFD5D4E909128A4218D0A1692569885C89
:10FBC00098800132B2FBF5F105FB1122A262D0E769
:10FBD00099891A888D0692B2C9D59006C7D5E26A6E
:10FBE0004AB19888216B9047636EC0E7DA6822F0CB
:10FBF0008002DA60BDE79B88E2696169DBB28B5401
:10FC0000E269E068636E0132B2FBF0F100FB1122A1
:10FC1000E261ACE76C1100102DE9F04FB74C23788E
:10FC2000222B8DB000F04C81B54B1D78002D59D1A1
:10FC3000B44BB54C93F800A0DFF804B3DFF804939D
:10FC40000AF0010A04F52876A4F10B0854F80B0C0D
:10FC500040B12FF0C3FA0746002840F0F08014F8B6
:10FC6000033C3BB9E034B44205F10105EED10DB0DF
:10FC7000BDE8F08FD9F8002054F8071C521A632A07
:10FC8000F0D9012B00F02A83022BEBD19F4BA04926
:10FC9000DB78A04AA048CBF8B405003318BF012395
:10FCA0000B7054F80B3C9D491160CBF8A834944973
:10FCB000CBF8B035CBF8B835402301228BF8BC35F2
:10FCC00097488BF8BD750A7019F08EFF4FF40050FD
:10FCD00014F08EFD934819F071FF8BF800768BF8C5
:10FCE0000176BFE78B4B1B68002BC0D0DFF850922A
:10FCF000DFF830A219F052FF09F59668D9F8A80488
:10FD00002FF06CFA0028B2D0D9F8A8042FF05EFAD0
:10FD100009280346D9F8AC6419D03F2817D016B982
:10FD2000042800F0D5820C2B00F065827F2B40F078
:10FD3000B480002EE2D0013E09EB060300227A488F
:10FD4000C9F8AC6483F8B02419F038FFD6E7002E68
:10FD500053D1764B354603F55877002D46D01033F6
:10FD6000BB42FAD1DFF8E0B12868DBF80020845DFF
:10FD7000935D9C42304402EB060140F0AD82741E5C
:10FD80004444324613B9FD2A40F2108204F8013F80
:10FD90000132C9F8AC2410F8013F11F8017F9F42ED
:10FDA000F0D00AB15D4513D0614819F007FF5D45F9
:10FDB00008D855F8100B19F001FF092019F0E5FEDD
:10FDC0005D45F6D9504619F0F9FED9F8AC24002665
:10FDD000964293D2741E444414F8010F19F0D5FED4
:10FDE000D9F8AC3401369E42F6D387E703F110020E
:10FDF000BA421D46B6D01346AFE74C4C4FF0000B4D
:10FE000004F558775D4602E01034BC420DD032460E
:10FE1000216840461BF020F80028F5D1A346002DAC
:10FE2000F2D125461034BC42F1D1002D9CD1BBF15A
:10FE3000000F3FF463AF3E4819F0C0FEB9E7D9F8B0
:10FE4000003044F8073C0023C5EBC50704F8033C29
:10FE5000A4F10B0308EB4717009354F80B0C2FF099
:10FE6000BDF900283FF4FEAE54F80B0C2FF0AEF9AC
:10FE700014F8021C4B1E02460B2B00F2A481DFE893
:10FE800013F06B01620156012E011C010001D0002C
:10FE9000B200A5007E0065003300002E00F06F81E7
:10FEA0000A2B00F0B9810D2B00F0B681FF2E3FF632
:10FEB00025AFA3F12002D2B25E2A40F269811DE78C
:10FEC0001C4B1868002800F06E812FF0D1FC2378BD
:10FED000194A222B10807FF4A7AE184B1B68003301
:10FEE00018BF012353809FE694F8CE30934200F070
:10FEF000CD80002304F8023CAFE700BF61BA0020C8
:10FF00005C93002030930020E7D200208CD50020A5
:10FF1000100D00102CD900204DC50308841D0020B1
:10FF2000705506083C55060850550608B0DC050813
:10FF3000345506086094002064BA0020F887002039
:10FF4000D017002074C5002000E00508114694F881
:10FF5000CE0001921AF060FCD4F8C530019A84F802
:10FF6000CE00F9180133C4F8C530CA72D4F8C920DC
:10FF700093427FF472AF0C2304F8023C6DE7D4F88F
:10FF8000C530F9180133C4F8C530CA7294F8CE00F0
:10FF9000019311461AF040FC019B84F8CE00052B1A
:10FFA0007FF45BAFB4F80120B4F803302178A4F8F3
:10FFB000C1200022C4F8C93084F8C310C4F8C52099
:10FFC000002BD8D00B2304F8023C46E794F8CD3040
:10FFD00094F8CE105340914284F8CD3089D1062355
:10FFE00004F8023C39E7114694F8CE0001921AF069
:10FFF00013FCD4F8C53094F8CD10019A84F8CE00E3
:020000040801F1
:10000000F81851400133C4F8C53084F8CD10C272DD
:10001000D4F8C92093427FF420AF092304F8023CAE
:100020001BE7D4F8C530F9180133C4F8C530CA72DB
:1000300094F8CDC094F8CE00019382EA0C0C1146DE
:1000400084F8CDC01AF0E8FB019B84F8CE00072BA2
:100050007FF403AFB4F80530C02B3FF64AAFB4F8D5
:100060000320A178A4F8C1200022C4F8C93084F884
:10007000C310C4F8C520002BCFD0082304F8023CDD
:10008000EBE694F8CD3093427FF433AF0D2304F8C0
:10009000023C14F801CCBCF1000F00F0DF80BCF191
:1000A000010F00F05481002304F8023CE034B44214
:1000B00005F101057FF4CAADD9E5D4F8C530F918CA
:1000C0000133C4F8C530CA7294F8CD00D4F8C91011
:1000D00042408B4284F8CD207FF4BFAE7FE7D4F856
:1000E000C530F9180133C4F8C530CA7294F8CD1080
:1000F000022B82EA010284F8CD207FF4AEAE237891
:10010000C02B3FF6F6AE6178FF2900F03F81002258
:10011000C4F8C930A4F8C11084F8C320C4F8C520BD
:10012000002B3FF45CAF052304F8023C95E60A235C
:100130003C2A04F8023C0BD03E2A7FF4DAAE0123BD
:1001400004F8013C89E604233C2A04F8023CF3D17C
:10015000002304F8013C80E600234D2AC4F8C53092
:1001600084F8CD3084F8CE3050D0582A7FF404AFD4
:100170000322022304F8022C84F8C4306DE6A3F1B4
:100180002002D2B25E2A3FF6B9AD202B3FF4B6ADC5
:1001900009EB06021846013682F8B034C9F8AC649F
:1001A00019F0F3FCAAE5814A108096E6511C09EB90
:1001B00001004A44202482F8B044C9F8AC140A462D
:1001C00080F8B034EEE5242A1CD0BAF1000F03D039
:1001D0000D297FF442AE5CE7754B93F832309342C1
:1001E00005D0232A04BF022304F8033CF0E70123CF
:1001F00004F8033CECE76F4819F0E0FC504619F0B6
:10020000DDFC7BE5012304F8023C26E6022284F8AB
:10021000C43004F8022C20E619F0E2FC23216648E1
:100220004CF0CDFE002866D0A0EB0802C9F8AC2443
:10023000002A7DD0531E09EB030191F8B014202948
:1002400040F0AE80023A4244002B6FD012F8011900
:10025000202903F1FF3051D10346F5E7574BADF8A4
:100260002CC00FCB04AF87E80F000DF1300ED4F88F
:10027000C9204EF824CDA11894F8C3300991B4F8E0
:10028000C110ADF828101F464FF0010CD4F8D10072
:100290000894734604AA08A98DF82A708DF82EC018
:1002A00014F0AEFAE0B9039F002304F8023C002FDB
:1002B0003FF4D8AC54F80B0C13F080FFE03454F842
:1002C000EB0CB847B44205F101057FF4BFACCEE4B6
:1002D000404633F065F811E5324662E54AF030FBFE
:1002E000049A374B059204A9009894F8C42004930B
:1002F00012F078FAD7E7D9F8AC2499E7C9F8AC340A
:100300004B44304C002283F8B02404F5587702E0C7
:100310001034BC4246D02168404632F083F90028B0
:10032000F6D0BC423ED2E36898470023C9F8AC340B
:100330004FF48072002140464CF02AFE224B1B787D
:10034000002B3FF4DBAC504619F038FCD6E4D4F86F
:10035000C930B4F8C1200894234409936E2A4FF0A1
:100360000003ADF82E30CDF82A30ADF828207FF408
:100370009AAE08A81BF0A8F808A81BF099F808A8DE
:100380001BF096F808A81BF093F88CE6052B7FF677
:10039000B0AD0122072384F8C42004F8023C5CE5D8
:1003A0001346ADE709481AF047F8BEE764BA0020E3
:1003B000C8D9002044550608801C002010E005081C
:1003C000ECF40020B0DC05085C93002054550608CE
:1003D00010B5164B42681B7803F00303032B21D1A1
:1003E000134B1B88DBB1134B1349B3F90030B1F940
:1003F00004100A2491FBF4F15B1A1B0103F5B953B5
:1004000014334FF4B471B3FBF1F3C3F1080303F0F9
:100410000F0360331370436800225A7010BD052328
:100420001370F8E72D231370F5E700BF6C930020DD
:100430006E930020181E0020B4930020436872229F
:100440001A70436873225A70436874229A70436822
:100450000022DA7070472D4A0A23B2F9001091FB8E
:10046000F3F383EAE371A1EBE3715A2930B505DDBB
:10047000002BB4BF6FF0B301B421CB1A24498C78A0
:100480003CB9244C2478E5072AD4234C247824074B
:1004900026D4097AB32903D81F49097809071FD43C
:1004A000B2F902100A2291FBF2F103B9C1B181EA5B
:1004B000E17583EAE374A5EBE175A4EBE374B5EBB6
:1004C000440F426813DAB4EB450F10DA002908DD57
:1004D000002BCCBF6E2362231370436800225A7036
:1004E00030BD002BCCBF6A2366231370F5E7A5420D
:1004F00005DD0029CCBF602368231370EDE7002BD6
:10050000CCBF6C2364231370E7E700BFB4930020D3
:10051000181E0020309300206C9300200E4B416881
:10052000B3F904300A2293FBF2F31B0103F5B9532C
:100530004FF4B4721433B3FBF2F3084A03F00F0321
:1005400013441A680A605A684A601B7A0B7243683F
:1005500000225A72704700BFB493002020E00508C3
:10056000034B93F88130002B0CBF0D200E207047F9
:10057000181E0020054B93F881302BB94FF4A4735B
:100580005843642390FBF3F0704700BF181E00200F
:1005900070B41D4CB4F8D830E8B903F00103C3B906
:1005A00094F8DC50ADB1194A02F1F00602E00133D3
:1005B000AB420ED052F8041B4904F8D594F8C81188
:1005C00004EB8101D1F8600146F823000133AB420E
:1005D000F0D170BC70475B08012B09D90A68A4F8F8
:1005E000D83002F5C332A03203F001030A60D6E727
:1005F0000B6803F5C333A03348F20502A4F8D820F2
:100600000B6070BC704700BF181E0020F81E002051
:100610002DE9F041A8BB2E4A92F8DC0060B32D4AC8
:100620002D4B92F800C092F901E092F90280CCF1D2
:10063000FF07ACF17F06FFB2F6B203EB800003F1D7
:10064000F002002403E0834202F1040214D053F8C4
:10065000041B8904F7D5E1B2A1EB0E0181EAE17533
:10066000A5EBE175012D09DD08218342D17004F16C
:10067000010402F10402EAD1BDE8F08179B96146D2
:10068000F3E7144B1A78F02A0ED802F10F00104A43
:1006900018700B6803F582431A330B60BCE74145C1
:1006A00014BF39463146E0E7094A93F9010092F850
:1006B000DE5093F902407F26A8421E7005DB64429B
:1006C00064B29C7020445870E3E70028FADAF6E739
:1006D000181E0020A0010020F81E00202DE9F04186
:1006E000354E78B196F85032002B45D0013B334A55
:1006F000DBB286F850321378DC0740D4304A0B68FE
:1007000013440B6096F8DC4034B32E492B4F002382
:1007100001F1F00C1D4602E00133A3421CD051F858
:10072000042BC2F303200628F6D13878C00715D56C
:1007300096F8500296F8DF8000EB050E9EFBF8F06D
:1007400008FB10E00128CCBF0020012058B901337C
:10075000A34205F10105E2D1BDE8F081E84300F0D4
:1007600001000028F3D0C2F3834206EB8202D2F8E4
:1007700060214CF82320EAE796F8DF30B6E7124A0A
:10078000124BB2F906201248A2F57A74642202FBD9
:1007900004F283FB0234D317C3EBA41303EB43032C
:1007A000C3EB031380FB0302DB17C3EB62130533B8
:1007B000084A92FBF3F2A2E7181E002030930020B3
:1007C000400D0300F81E002040DA0020D34D6210D7
:1007D0001F85EB5140420F00F0B54F4C94F8512269
:1007E000002858D1002A55D04C4BD3ED007AB3EEF7
:1007F000097AF4EEC77AF1EE10FA7ADCBBEE097AE8
:10080000F4EEC77AF1EE10FA4CBF08270027D3EDBB
:10081000017AB3EE097AF4EEC77AF1EE10FA6ADDE6
:1008200047F0010794F8DC50A5B33D48DFF8FCE041
:1008300000F1F00C002218E094F95462B142ACBF10
:100840000221002194F95562B34220DA94F95662EC
:10085000B342D8BF41F008010F421CBFDEF824307C
:100860004CF822300132954214D050F8043BD903A1
:10087000F8D594F9536203F00F01B142C3F30313A7
:10088000DADC94F95562B3424FF00101DEDB41F04E
:100890000401E1E7F0BD94F852320868ABB31F4B96
:1008A000204ED3ED007A93ED017A1F4DF0EEE77AFA
:1008B000B0EEC77AF4EEC77AF1EE10FAB8BFF0EEF8
:1008C000477AFDEEE77A82F0010217EE903A193B83
:1008D00003EB4303C3EB031386FB0376DB17C3EB86
:1008E000E613053395FBF3F3184484F851220860AE
:1008F00078E704278BE7BBEE097AF4EEC77AF1EECE
:1009000010FA48BF47F002078CE700F5433000F5C6
:10091000A070086066E700BF181E002078930020D2
:10092000F81E0020353AFC4440420F0020E0050844
:1009300070B40B4E96F8DC4084B106F1E002054637
:1009400006F5E876002352F8040B35EA000004BFF0
:10095000086846F823000133A342F4D170BC704705
:10096000181E002030B42A4B60B92A48027DCAB94B
:1009700093F8C9312849203301EB83014FF4A0607B
:1009800030BCD5E793F85722F2B1013A214883F8F9
:1009900057220A6802F5C32202F520720A60027D1E
:1009A000002AE5D01D4A12689106E1D51C4A93F849
:1009B0005712127892071AD511BB93F8CB3116490A
:1009C000203301EB8301D9E7124893F85842057DA3
:1009D000A54205D8042483F8582283F85742D8E763
:1009E0000134012283F8584283F85722D1E70029C5
:1009F000BED193F8CA310849203301EB8301BDE72A
:100A000093F8C7310449203301EB8301B6E700BFF7
:100A1000181E0020B0D90020F81E00200C890020EC
:100A20006C93002010B41C4AA0B91C4C92F85902D7
:100A30000B6823440B6010B15DF8044B704792F8CB
:100A4000C73117495DF8044B203301EB83014FF4A4
:100A500040706DE792F85A328BB1012B07D192F8B2
:100A60005902104C80F0010082F85902E0E792F838
:100A700059020D4C80F0010082F85902D8E70B684A
:100A80005DF8044B03F5742303F5107301200B602C
:100A900082F85902704700BF181E002040420F0024
:100AA000F81E002020A1070048E80100A8B93C4832
:100AB00090F85B326BB190F85C128A081341DB0747
:100AC0000AD501F00101032A06D8DFE802F05048F8
:100AD000403890F85D3253BB7047314890F85C3233
:100AE000013303F00F0380F85C323BB190F85B32C6
:100AF0000A6802F5C332A0320A60DBE7294A80F8AF
:100B00005B32527A002A43D1274AD2781AB143F095
:100B1000040380F85B32254A1278D2072FD58278F9
:100B2000002AE5D043F0080380F85B32E0E790F854
:100B30006A321F4901EB83014FF40030F8E61C4B89
:100B400003F13002002914BF19461146F4E7194B8E
:100B5000A3F11802002914BF19461146ECE7144B03
:100B600003F10802002914BF19461146E4E7104BAF
:100B700003F11802002914BF19461146DCE70E4A9A
:100B80001268002ACBD043F0010380F85B32C6E73D
:100B900090F85A22002AB7D0022380F85B32B3E7DC
:100BA000181E0020889300203493002030930020EA
:100BB00038E0050860E00508B496002090F8603041
:100BC00043B942690121072082F84430A2F8460067
:100BD00082F848107047034A0123E021C373517023
:100BE000184670474C9800204FF0FF3070474FF088
:100BF000FF30704770470020704700207047F0B406
:100C0000067ABEB1427A0D4C002120276AB100233A
:100C1000142B07DC072904EB030003DCC578202D27
:100C200018BFC77001339342F2D101318E4204F1F3
:100C30001504EBD10020F0BC704700BF4C98002099
:100C400010B50024C473FFF7DAFF024B01225A707B
:100C5000204610BD4C98002070B402EB42000C4CB2
:100C6000C0EBC000013B04440BE0142907D8072A5D
:100C700004EB010503D8EE78864218BFE870013115
:100C8000C9B213F8010F0028EFD170BC704700BF44
:100C90004C98002014290CD8072A0AD802EB4202EB
:100CA0000548C2EBC20202441144CA789A4218BFF6
:100CB000CB700020704700BF4C980020027A407A29
:100CC00002FB00F07047027A407A02FB00F07047A6
:100CD00000207047002070474FF0FF307047044BF2
:100CE00093F89523027293F896334372704700BFCE
:100CF000181E002000207047012070470120704717
:100D000000207047027A407A02FB00F07047002012
:100D100070470123C373184670470123C3731846F5
:100D200070474FF0FF307047704700207047012038
:100D3000704700207047027A407A02FB00F070474B
:100D4000002070474FF0FF30704770470020704719
:100D50000120704700207047027A407A02FB00F0C1
:100D60007047002070470020704700207047002027
:100D70007047002070471D290DD80F2A0BD810B4DA
:100D800006481E2414FB02110144002081F8983308
:100D90005DF8044B70470020704700BF181E00200C
:100DA000014B9888704700BFA0010020024B002033
:100DB000C3F8A005704700BF181E002000230222C0
:100DC0000271037043708370C3707047704703797A
:100DD00013F0020308D00369D0E90920013B101A7F
:100DE0001840C0B2181A7047184670470171704712
:100DF000704703799B070AD5436A8269D154436AD5
:100E000001690133B3FBF1F201FB12334362704716
:100E1000037913F0010306D0D0E90732C0689B1AAA
:100E20000138184070471846704710B5037913F021
:100E3000010301460ED0FFF7EBFF50B10B6A4A6980
:100E4000CC68D05C0133B3FBF4F204FB1233C0B2C4
:100E50000B6210BD1846FCE790F84F3830B53BB92F
:100E600090F84D1890F84E380124DAB2914200D82B
:100E700030BDB0F8565804FA03F22A43A0F85628B9
:100E80000133F2E7D0E90920131A5842584170475C
:100E90002DE9F04F774989B091F8A4350490002BE3
:100EA00042D091F8A53503F0FF06002B3CD1724BE0
:100EB000D1F8A8E59A790593002A0DF1200C0CBF12
:100EC00073462023B1F8B025019303924FF03C08FC
:100ED000B1F8B2254CF8046D91F8AC9591F8AD4598
:100EE00091F8AE3502924046019AB2421FD181F884
:100EF000AE35059B614A81F8AC95002098710123BD
:100F000081F8A535D2F86431D2F8682181F8AD4571
:100F100040F22A3159605062118841F0010111807C
:100F20001A6842F001021A6009B0BDE8F08F7645F8
:100F300036BF534A674602EB8607BD78FA78C5F19B
:100F4000FF05ADB2002D00F09080C5F1FF055543BF
:100F50003F88B7FBF8FA2D12BAF1050F00F288802E
:100F6000DFE80AF0033242536573EBB2551B7D4351
:100F7000B5FBF0F41C44E4B2049D012D0BBF250227
:100F8000150245EA024545EA04451D43009518252A
:100F900005FB06FB0027C7F11709012505FA09F92A
:100FA000009D19EA050F029DA946039D14BFCA467C
:100FB000AA4607EB0B09334D0137182F45F829A036
:100FC000E9D1013691468FE7B7FBF0F400FB1477C7
:100FD000BFB2EBB2C7F13C07551B7D43B5FBF0F543
:100FE0001D441446EAB2C7E7B7FBF0F300FB1377E2
:100FF0005FFA85F9BFB2551B07FB05F3B3FBF0F3AE
:101000004B441446DBB24A46B6E7B7FBF0F300FBAD
:101010001377BFB25FFA85F9C7F13C07551B7D43D3
:10102000B5FBF0F44C441346E4B24A46A4E7B7FBE0
:10103000F0F300FB1377ECB2BFB2551B7D43B5FB59
:10104000F0F525441346EAB296E7B7FBF0F300FB50
:101050001377BFB2ECB2C7F13C07551B05FB07F392
:10106000B3FBF0F32344DBB286E71346144683E771
:101070004A4681E7181E0020A0010020102F002002
:10108000E81F0020CC230020074A30B50023044687
:1010900002F5E875D2F8A815994200D830BD20684D
:1010A00045F823000133F5E7181E0020034B93F8A1
:1010B0006C0180F001004042704700BF102F0020FB
:1010C000034B0449DB7940685B42012219F052BBB3
:1010D000A00100200E6B0608064B07491A88074B33
:1010E00040681B68534342F2107293FBF2F219F00E
:1010F00041BB00BF7093002092610608A4930020BA
:1011000007B5074B1A68917A137A0191527A0092C7
:101110000449054A406819F02DFB03B05DF804FB53
:10112000BC9600209B6106089761060807B5074B2F
:101130001A68917D137D0191527D00920449054A00
:10114000406819F017FB03B05DF804FBBC96002063
:101150009B610608AA61060807B5074B1A68117C4F
:10116000937B0191D27B00920449054A406819F0B3
:1011700001FB03B05DF804FBBC9600209B610608F0
:10118000AE610608044A0549537812784068013375
:10119000013219F0EFBA00BF8CD50020B261060809
:1011A0001C4B1A6812F0200F13B502F004034468B8
:1011B00029D0194A1278920725D5184BB3F90000A7
:1011C000FFF7D8F964210A2290FBF1F301FB130128
:1011D00091FBF2F1124A92F881200029B8BF4942EE
:1011E000002A0CBF99229F22002BCDE90012B8BF24
:1011F0005B420C490028ACBF75227622204619F0CC
:10120000B9FA02B010BD002BD7D12D22227042684E
:101210005370F6E70C8900206C930020BA930020ED
:10122000181E0020B86106080B4B4068B3F9043063
:101230000A2293FBF2F31A0102F5B9524FF4B4718A
:101240001432B2FBF1F2C2F1080202F00F02603276
:10125000024919F08FBA00BFB4930020C661060896
:10126000034A044992684068072319F083BA00BF13
:10127000A4930020CD610608124A4068B2F86E318E
:1012800092F87021012A10D107EE903A9FED0E7A64
:101290000E49F8EEE77A7B2267EE877AFCEEE77A72
:1012A00017EE903A9BB219F065BA0A22534340F206
:1012B000FF3293FBF2F3092BA8BF09237B220449D9
:1012C00019F058BA102F00208925963E0E6B06089B
:1012D000D361060807B5124B406893F87A21114B89
:1012E0009AB19A89104B93F8813083B942F2107306
:1012F00053430E4A93FBF2F39D2200920C49702255
:1013000019F038FA03B05DF804FBDA89EAE7242320
:1013100053434FF47A7293FBF2F39E22EDE700BF42
:10132000102F0020B0D90020181E002040D2060047
:101330008363060830B5124A124B92F8D5204068F4
:101340001C7D85B0AAB10A215A8AB2FBF1F5B5FB22
:10135000F1F301FB13539BB202930B496423B2FBDD
:10136000F3F21F23CDE900421E2219F003FA05B063
:1013700030BD00941F231E22044919F0FBF9F6E743
:10138000181E0020B0D90020D9610608E7610608C0
:101390000C4B40681B688922002B10B402700EDAD7
:1013A0002D2242705B420224074993FBF1F2204454
:1013B00001FB12335DF8044B044919F0DBB9012439
:1013C000F2E700BFB0D9002080969800EF610608D0
:1013D0000C4B40685B689822002B10B402700EDA48
:1013E0002D2242705B420224074993FBF1F2204414
:1013F00001FB12335DF8044B044919F0BBB9012419
:10140000F2E700BFB0D9002080969800EF6106088F
:10141000044B1B78DB0703D40349406819F0AAB9D1
:10142000704700BF30930020F761060813B50849E4
:10143000B1F90640B1F90230B1F900200194B1F9D7
:10144000041000914068034919F094F902B010BDEE
:1014500064BA00200062060813B5094B1B689A2481
:10146000002BB8BF5B426421009493FBF1F240680B
:1014700001FB1233034919F07DF902B010BD00BF22
:10148000A49300201462060837B50378114A406817
:101490001A2B0CBFB2F90250B2F900500A211A2BD4
:1014A00095FBF1F408BF152201FB145118BF14225B
:1014B000002DB4BF2D2320230029B8BF4942002CA2
:1014C000B8BF644201910094034919F053F903B085
:1014D00030BD00BFB49300201F6206081E4B37B515
:1014E0001A68446812F0200F02F004032AD01B4A45
:1014F0001278920726D51A4B1A4D1868FFF73AF85A
:101500007F220A2390FBF3F3002B2270BCBF2D2215
:10151000627095F88150B4BF02200120002BB8BF43
:101520005B42002D4FF00A010CBF0F250C2593FBE9
:10153000F1F2009501FB123320440B4919F01AF91E
:1015400003B030BD002BD6D17F22227042682D21FE
:10155000517042689370F3E70C8900206C9300206F
:10156000AC960020181E0020BA610608084BD3F87C
:101570007C21002A0ADD074B03EB8203DA6C2AB1D7
:10158000054B06499B68406819F0F4B8704700BFE6
:10159000102F002020E00508A00100202D62060881
:1015A00037B504460846FEF7E5FF0AB1227001345C
:1015B0001B4B93F88130002B0BBF4FF4A5524FF417
:1015C0007A727E217D210CBF0F230C23824207DD1E
:1015D00014490246204603B0BDE8304019F0CAB8AD
:1015E0006423584390FBF2F0B0F57A7F90FBF3F25E
:1015F0000DDB0A23009190FBF3F00B4990FBF3F510
:1016000003FB1503204619F0B5F803B030BD009177
:1016100003FB12030549204619F0ACF8F5E700BFBB
:10162000181E00203862060835620608DE97060894
:101630000A4A127802F00302032A03464FF011020D
:10164000406802D1064B1988AAE702705A682D211A
:1016500051705B6800229A70704700BF6C93002045
:101660006E930020094B40681B7803F00303032BA3
:1016700007D1074B7122D3F880116423B1FBF3F13A
:101680008EE72D237122034919F074B86C93002062
:10169000102F00203D62060810B5174CA379C3B186
:1016A000A37EDFED166A07EE903AF8EEE77A144B68
:1016B00086EEA77AC0B203EB8000838907EE903AEA
:1016C000F8EEE77A67EE277AFDEEE77A17EE900AF2
:1016D00010BD0C4B1B6813F000630BD0C0B228F098
:1016E00083FF8089642310FB03F0A37E5B0890FBDB
:1016F000F3F0EDE71846EBE778BA00200000484326
:10170000EC1100108CD8002008B5FFF7C5FF3C2372
:1017100090FBF3F008BD074B93ED007AD3ED017A0F
:10172000B4EEE77AF1EE10FA03DD034940684BF0BE
:1017300053BC704700000010E863060810B50C4663
:10174000A8B9194B194993F8842123680B442360E5
:1017500002B110BD164991F8C73101EB830101F5C3
:10176000B0714FF48060BDE81040FFF7E1B832F08F
:1017700047FD32280ADD23680B4A03F5742303F57D
:1017800010730121236082F8841110BD064B93F879
:101790008421142882F00102C7BF83F884210549FF
:1017A000054983F88421D0E7102F002040420F0024
:1017B000181E002020A1070048E80100224B1B88CA
:1017C0005A0510B5446805D520462049BDE81040AB
:1017D0004BF002BC180505D520461D49BDE8104058
:1017E0004BF0FABB590605D520461A49BDE8104012
:1017F0004BF0F2BBDA0705D520461749BDE810408B
:101800004BF0EABB9B0705D520461449BDE81040C4
:101810004BF0E2BB25203CF00DFE28B120461049DC
:10182000BDE810404BF0D8BB0E4B93F885312BB17F
:1018300020460D49BDE810404BF0CEBB20460B4979
:10184000BDE810404BF0C8BBB093002042620608D0
:10185000476206084C62060851620608566206088E
:101860005B620608102F00206062060865620608A9
:10187000032811D8DFE800F00A0C0206074BD3F862
:101880008C017047064B1B78DB0701D4FAF716BAB8
:10189000024BD3F88801704700207047102F0020BA
:1018A0003093002037B504462A4800EB4303B3F8D1
:1018B000825005F00F0049B1611C032826D8DFE8EB
:1018C00000F02702021D9C2323700C4612B3C5F3BF
:1018D0000315FFF7CDFF3C21012D1F4BB0FBF3F3A8
:1018E00093FBF1F201FB123316D0022D24D01B49D9
:1018F000204603B0BDE8304018F03CBF184B1B78C1
:1019000013F0010F14BF9C239B23DDE72023DBE7AB
:101910009B23D9E71546DCE7642542F21071B0FB42
:10192000F1F0B0FBF5F105FB110000900D492046E8
:1019300018F020FF03B030BD0A250B49B0FBF1F0D1
:10194000B0FBF5F105FB110000900849204618F0A6
:1019500011FFEFE7181E002040420F006A620608E0
:101960003093002074620608A08601008362060896
:10197000037840680122053B114693E710B5044601
:101980001DF044FC0422034602496068BDE8104093
:1019900018F0F0BE0E6B06082DE9F0478678457802
:1019A00006F1020904464FF000085FFA89F90027A2
:1019B00005EB080AB8F1030FA06862D1E91C022FF9
:1019C000C9B258D10B234A462EF098FA0137052F99
:1019D000F0D108F10108B8F1070FE8D12D4B2E48DE
:1019E00093F89D202378013A302B2C4B4FEA82024A
:1019F000134440F2CF770BBF93F8D42093F8D6204E
:101A000093F8D5C093F8D7C030F9123030F91C00E4
:101A1000BB42A8BF3B46B3F57A7FB8BF4FF47A7399
:101A2000B8424FF47A71A8BF3846A3F57A7388425A
:101A3000C3EB031393FBF1F3C3F10E03B8BF0846E6
:101A4000DBB20322B3FBF2F202EB420EA3EB0E0376
:101A5000A0F57A70C0EBC000083390FBF1F132447E
:101A60002944DBB2D2B2C9B2A0682EF047FA0023F3
:101A70002373BDE8F087F2191623D2B22EF03EFA96
:101A8000A4E7022FA2D117234A465FFA8AF12EF06B
:101A900035FA9BE7181E002040DA002020E00508F8
:101AA00070B504466FF00205A2786178A068EEB2C6
:101AB000324407391323D2B2C9B22EF01FFAA278EA
:101AC0006178A068324407311323D2B2C9B201351C
:101AD0002EF014FA042DE7D16178A278A0680639B7
:101AE0000323C9B22EF00AFA6178A278A068063101
:101AF0000223C9B22EF002FA0023237370BD2DE930
:101B0000F0472A49054691F88C3091F88D202848F5
:101B100091F89B10B0F90040002902EB820214BF3B
:101B20004FF0FF31012152004C43574203EB830336
:101B3000BC424FEA430303DB9442A8BF1446274646
:101B4000B0F902205C424A43A24203DB9A42A8BF9A
:101B50001A4614461BB11922544394FBF3F4293C52
:101B60004FEA87086FF003064FF040094FF0090A6B
:101B700098FBF9F31B1B512B0FD893FBFAF101EBE8
:101B8000C1029B1AAA78A8680A446978803B31444C
:101B9000DBB2D2B2C9B22EF0B1F90136052EA8EBF4
:101BA0000708E5D100232B73BDE8F087181E00203D
:101BB000B493002010B5044632F058FB642343432D
:101BC0009B12632B60680449A8BF63230122BDE810
:101BD000104018F0CFBD00BFE96106081D4B9FED16
:101BE0001E7A9A681D4B4068B3F87C3007EE902A45
:101BF000F8EEE76A07EE903AF8EEE77A67EE877A52
:101C0000F4EEE76AF1EE10FA02D8154918F0B2BD09
:101C1000934202DA134918F0ADBD9B1A07EE903AD1
:101C2000114B124AB8EEE77AD3ED627AF8EE677A92
:101C30003C2167EE277A87EEA67AFDEEC77A17EE8B
:101C4000903AB3FBF2F393FBF1F201FB1233084934
:101C500018F090BDA4930020CDCCCC3D181E0020E0
:101C60009262060898620608102F002040420F007A
:101C70006A6206082DE9F0411B4D1C4E0746002400
:101C80003AF0D8FB4FF0880C05F1040E33787968F0
:101C9000A342214403DC00230B70BDE8F081F8B1BE
:101CA000D5ED007AFDEEE77A0EEB840317EE908A0D
:101CB000D3ED007AFDEEE77A17EE902AD5ED097A9A
:101CC000FDEEE77AA2EB080217EE903AD200A3EB02
:101CD000080392FBF3F3C3F188030B700134D5E7DB
:101CE00081F800C0FAE700BF200400108411001042
:101CF000F7B5174A174B92F85A221B884768022AF1
:101D000003F105044FF00A05064694FBF5F51DD0D6
:101D1000114A107893FBF0F02AF0D6FA38700A21B5
:101D2000706895FBF1F3632D01FB13534FF006012F
:101D300000914FF06402C8BF084994FBF2F2D8BF8B
:101D40000749013018F016FD03B0F0BD9720E5E714
:101D5000181E00207093002076930020356206083C
:101D60009E62060873B5104B46681C880F4B1B78A3
:101D700094FBF3F40E4B93F85A32022B054611D024
:101D800020462AF0A1FA307068686423062194FB8B
:101D9000F3F2009103FB12430649013018F0EAFC0C
:101DA00002B070BD9720EEE770930020769300207C
:101DB000181E0020DE9706081E4B1F4A9B8992685A
:101DC00013B50446D3B19A1A9A42A8BF1A4622EA1A
:101DD000E27207EE902A0B22B3FBF2F300EE103A08
:101DE000F8EEE77AB8EEC00A87EE800A49F044FEC2
:101DF000FCEEC07ACDED017A9DF8043062688A214C
:101E00001170012261689342ACBF8B208D208854F1
:101E100001320C2AF6D162688F2111735A1E092AE9
:101E200003D8626813448E225A70636800225A7382
:101E300002B010BD88930020A493002010B5044682
:101E400013203CF0F7FAD8B10AF036FB30B96068DD
:101E50000C491022BDE8104018F08CBC0AF042FB7F
:101E600064680346102228B120460749BDE81040A7
:101E700018F080BC20460549BDE8104018F07ABC37
:101E800010BD00BFA7620608AB620608AF62060875
:101E90000A4B93ED6D0A10B5F2EE047A20EE270A94
:101EA000044649F02FFE0A23054990FBF3F203FB99
:101EB00012036068BDE8104018F05CBC102F0020D1
:101EC000B4620608084B93F8813007EE900A4BB9CC
:101ED000F8EEE77A9FED057A9FED050AA7EE870AEF
:101EE00049F010BE704700BF181E00206766E63F2D
:101EF000000000422DE9F04F9D4F9E4C97F85A820A
:101F000089B00546F9F7DAFED4F8B831D7F8886019
:101F100023F40013C4F8B831F307814648D50020F4
:101F20003CF088FA002840D0934B1A68002A3CD035
:101F3000100204D5B2F5000F18BFA2F50002D4F8C4
:101F4000C0119FED8E7AA9EB010307EE903AF8EEEF
:101F5000677AF4EEC77AF1EE10FA05DCD4F8C40122
:101F600001238340134212D111B91723C4F8C4319D
:101F7000D4F8C431C4F8C09101200133182B28BF14
:101F8000002300FA03F11142F7D0C4F8C431D4F8A9
:101F9000C4217B4B7B49686803EB8203D3F8E420C0
:101FA00018F0E8FB09B0BDE8F08F0023C4F8C03199
:101FB000D4F8C83173B3744B1B78D9072AD4D4F83A
:101FC000CC019FED727A00F5921000F57860A0EBDD
:101FD000090307EE903AF8EE677A686867EE877A49
:101FE000FDEEE77AB8EEE77A17EE903AF1EE0C7A6A
:101FF000B4EEE77AF1EE10FA03DB654918F0BAFBAC
:10200000D0E70A2193FBF1F201FB1233614918F08A
:10201000B1FBC7E7B2050DD55F4BDB7853B15F4924
:10202000686818F0A7FBD4F8B83143F40013C4F87B
:10203000B831B7E7B30606D5BB7823B1584968680D
:1020400018F098FBAEE7700521D594F8D031012B3C
:102050001DD1544B68681B68990714D5524BB4F9CD
:10206000E021B3F9023051499B1A0A2293FBF2F3A3
:102070005A2B6FF05902A8BF5A239A42B8BF1A468A
:1020800018F078FB8EE74A4918F074FB8AE7B2042F
:1020900007D532F0B5F897F88030834201D9454929
:1020A000BEE7330407D5444B97F8D420DB799A4236
:1020B00001D24249B4E7700407D532F073F8B7F89B
:1020C000D230834201D93E49AAE7310704D5B8F19D
:1020D000020F01D13B49A3E732050FD52A4B1B78EC
:1020E000DB070BD53CF03CF940B1374B1B78D807E8
:1020F00004D594F81D320BB9344991E7F10414D595
:10210000214B1B78DA0710D53CF02AF968B12E4B29
:102110001B78DB0709D4D4F88C31A3F53713A3F56A
:10212000D863002B01DA2A497AE72A4B1B88580624
:1021300001D5294974E7310654D5284BB3F900007D
:1021400097F89A3098424DDBFFF7BCFE0246FEF747
:1021500007FA23490090134668687A2218F00AFBB0
:10216000D4F8B83143F40013C4F8B8311AE700BF0B
:10217000181E0020102F0020B49600200024F448E0
:1021800020E00508FB8C060830930020ACC52737FB
:10219000BF620608CA62060834930020D7620608A8
:1021A000E16206080C890020B4930020EC62060866
:1021B000F6620608FD620608A0010020C565060853
:1021C00006630608136306086C9300201D63060867
:1021D00028630608B0930020336306086C9600203D
:1021E0003C6306085E4B1B681A0174D5730672D5F2
:1021F0005C4A03921378C3F109035B08002604A824
:1022000020229E4221D1304457494AF0E5FE4FF04A
:10221000000A0336D146039B1B784B4501D90B2E90
:1022200016D908AB1E44002306F8103CBAF1000F83
:1022300051D004AA4D49686818F09CFAD4F8B83116
:1022400043F40013C4F8B831ACE682550136D8E740
:102250005FFA89FB584628F0C7F9454B19780BF10E
:10226000310211F00101D2B233D0B7F996B0BBF10F
:10227000FF3F2ED0B0F80CC064231CFB03FC3D4B89
:1022800093F81AE04FEA5E0E9CFBFEF39B45B4BF49
:102290001346522397F994E01EF1800F0DF1100CB4
:1022A00003D090F901B0F34553DA41B1B7F9981072
:1022B000B1F1FF3F03D040688842A8BF43239A4250
:1022C0000CF8063001D00AF1010A09F101090136C2
:1022D000A1E71346DEE7D7F888305A0704D5B8F1EE
:1022E000010F01D124499BE6DE050DD5204A127865
:1022F000D00709D5214A92F82520012A04D1204A85
:1023000012780AB91F498BE6990715D5184A127831
:10231000920711D497F85A2272B91B491B4A0878C0
:102320001B491288498A92FBF0F2914204D919495B
:10233000686818F01FFA35E6DB067FF533AE94F8CF
:102340002032002B3FF42EAE1349686818F012FAC1
:1023500028E654230029A9D10CF80630B3E700BFC2
:102360008CD800208411001048620608FB8C0608F7
:102370003093002078BA00204B63060818D800205C
:10238000582E0010576306087693002070930020A3
:1023900088930020636306086F6306080C4B1B6874
:1023A0001B0113B5044610D50A4BD3F8243293F918
:1023B0000100FFF787FD0246FEF7D2F806490090BC
:1023C000134660687A2218F0D5F902B010BD00BF3C
:1023D0008CD80020102F002079630608094B13B514
:1023E0000446B3F90000FFF76DFD0246FEF7B8F8AA
:1023F00005490090134660687A2218F0BBF902B0D4
:1024000010BD00BF6C960020826306082DE9F74FCF
:10241000154E4F7891F80280DFF850A0DFF850B0E9
:1024200081460D4600243378A34204DC00232B733D
:1024300003B0BDE8F08F2046C847504502465946D4
:10244000A8BF5246684618F095F902AB184408EB4D
:102450000402002300F8083CD2B26B463946A86853
:102460002DF056FD0134DEE7841100109F86010037
:102470004381060801460148C8E700BF0917010863
:1024800001460148C2E700BF9916010870B50D4C1E
:10249000054616460B4602460221D4F828022DF0C6
:1024A00037FD2A46084BD4F8280214212DF030FDC0
:1024B00033462A46D4F828021621BDE870402DF094
:1024C00027BD00BF102F0020899C060810B5802270
:1024D000044600214AF05CFD382204F1800000210E
:1024E0004AF056FD0D482246002350F82310C2F84A
:1024F000801001330E2B02F10402F6D11E2208498E
:1025000004F1C00049F01EFA0B22064904F1E40070
:1025100049F018FA032384F8EF3010BD38E00508BD
:1025200064E1050884E1050838B50C4C4FF490725D
:1025300004F51B7020214AF02BFD094B09491B684B
:10254000002001252D3384F89753C1F82C32C4F8AC
:102550008C03C4F8900384F8940338BD181E00203F
:1025600074C50020102F00200022C273DCE738B5AC
:10257000044602234FF4FA7032220021E37003254F
:102580000123E0802571228121706371A3721020E4
:10259000F8F72AFC607038BDF0B55C4C5C4DD4F89F
:1025A00030222B68DFED5B6A5B4E2968C4F830127D
:1025B0009B1A07EE903AF8EE677AB7EE007A67EE6C
:1025C000A67A3378F4EEC77AF1EE10FA88BFF0EE0F
:1025D000477A13F0010383B0C4ED8D7A0CD14F4AD2
:1025E0004F4812784F490380D2070B8031D4012322
:1025F00084F8543203B0F0BD01AB6A4604F50F71A4
:1026000004F50E7047F010F844484749019B009AC2
:102610000078DFF80CC1434FA1FB02E281FB03E12C
:10262000DB17C3EB61135209C107ACF800203B80F4
:10263000DDD533782D68DB0761D594F87A313B4ED0
:102640008BBBF3890F2B30D8B068D4F84032C11A55
:1026500005E0364ED4F84032B0682D68C11AD4F87F
:102660005022C4F840024FF47A73AA1A03FB01F314
:1026700040F2DC5193FBF2F31BB28B422C4AC4F8BC
:102680005052A8BF0B469342B8BF1346D6E900216B
:10269000A4F84C320123C4F84812C4F8442284F848
:1026A000543203B0F0BDB389CCE7224901AB081F17
:1026B0006A4646F0B9FF94F87A31B0684BB9D4F85D
:1026C0004032009AC11AD4F880311344C4F88031E2
:1026D000C5E7D4F84032DDED007AC11AF8EE677A2A
:1026E00007EE101A67EEA77AB8EEC77AE7EE077A18
:1026F000B1EEE77AFCEEC77A17EE902AE3E70B4ECD
:10270000D4F84032B068C11AA9E700BF102F0020EA
:1027100074C500206F12833A6C9300203093002020
:102720006E930020181E00201F85EB51B0D90020A9
:1027300024FAFFFF583100202DE9F04FB74C94F8F0
:10274000743185B0C5B2002B00F08580012B7FD19C
:1027500094F8E432082B7BD8DFE813F08B015901A1
:1027600027017A01D6019501B40148012F01D4F85F
:10277000E03294F8582201332121012AC4F8E032D2
:1027800084F8C81200F06E82022A40F00A81A44D3B
:10279000A44BB4F86C22DA81D5E90001B4F87022B8
:1027A0001A82722384F8C83250EA010340F0F9809B
:1027B000D4F87822002A00F0F480D4F874120029AA
:1027C00000F0EF80642301EA0300B2FBF3F703FBA0
:1027D000172C00EB80000CF5FA6C4600ADF804C035
:1027E000B7FBF3F0B1FBF3FC03FB1070BCFBF3F79A
:1027F00003FB17C78DF806008DF80A7042F21070BF
:10280000B2FBF0F2B2FBF3F703FB1722B1FBF0F0DF
:102810008DF80720B0FBF3F703FB17078248B1FBE5
:10282000F0F101A8B1FBF3F203FB12118DF809706E
:10283000ADF80C608DF8081018F06EF87B4B1A6834
:10284000861A61F10007C5E90067002384F8C432E5
:1028500005B0BDE8F08FA5F10A03222B74D8DFE89C
:1028600003F04B73734B737373737373737373737B
:102870007373737373737373737373734373737358
:102880007373127312006A4F94F8563294F85562BB
:102890000020F854002E6DD1664984F858623846FD
:1028A00048F0B6F8002800F040816349384648F007
:1028B000AFF8002800F039816049384648F0A8F8A0
:1028C000002800F0C4815E49384648F0A1F800288D
:1028D00000F0BD8138465B4948F09AF8002854D191
:1028E000032384F8583250E0002384F8553284F8EA
:1028F000563284F85732ABE794F8C432002B50D0EC
:10290000514901F1140313F8012D5A709942FAD17B
:10291000474F3B78402B40F20C81373B1B01DBB229
:102920007A78402A8CBF373A303AD2B2134494F8BE
:102930005722DBB29A423FF41AAF3F22002384F8B9
:10294000C82284F8C43283E794F856320E2B04D898
:1029500037495A1CCD5484F8562294F8C432002BBF
:102960007FF476AF94F857325D4084F8575205B043
:10297000BDE8F08F94F85832022B00F01A81032B37
:1029800000F0DB80012B00F03283013600232A2D7A
:1029900084F8556284F85632E4D1012384F8C432B5
:1029A00056E7002384F8C43252E7032384F8E65242
:1029B00084F8E75284F8E4324AE7244B0022A3F17A
:1029C000140184F8E42213F8012D5A709942FAD1C7
:1029D00094F8E732AB4200F02D81D4F848343F221E
:1029E0000133C4F8483484F8C82231E794F8E63259
:1029F0000822AB4284F8E4223FF42AAFD4F84834EA
:102A000001221344C4F8483484F8E52220E7622800
:102A100014BF0023022384F8E43219E7102F0020AA
:102A200058940020B0D9002040420F0074C5002007
:102A300090D800208066060888660608906606081A
:102A400098660608A0660608D8310020EC31002000
:102A500094F8E63294F8E72284F8E8521D44EDB287
:102A6000AB18042284F8E65284F8E73284F8E422B2
:102A7000EEE6B5287FF4ECAE0022012384F8E522CF
:102A800084F8E432E4E694F8E622B4F8EA3294F802
:102A9000E712154403EB0020EDB280B26B1806225A
:102AA000B0F5AC7F84F8E65284F8E732A4F8EA0285
:102AB00084F8E42277D90122002384F8E522A4F8DF
:102AC000EC32C5E694F8E622B4F8EC3294F8E7125A
:102AD0002A44D2B2B3F5AC7F114484F8E62238BF61
:102AE000E21803F1010338BF82F8F052B4F8EA2289
:102AF00084F8E7129BB29A42A4F8EC323FF6A8AEF3
:102B0000072384F8E432A3E694F8E63294F8E72247
:102B1000A4F8EA021D44EDB2AB18052284F8E6528F
:102B200084F8E73284F8E42292E6012384F85832EC
:102B30002BE71B0103F0F003F2E6022E00F08B807E
:102B4000032E05D147F050FB94F8556284F87D02BE
:102B5000032E7FF61AAF331F94F87C72C3F38703FA
:102B600003EB8707FD37FFB2102F3FF60EAFF21EC3
:102B7000A2EB830303F0FF03012B00F0E281042B9F
:102B80000BD1002047F030FB7B1E2344002294F839
:102B9000556283F8A00283F8B022D4F8C032013322
:102BA000C4F8C032F1E60023A4F8EC320028A7D024
:102BB0004EE6731E082B3FF6E8AE01A252F823F052
:102BC000252C01088B2901088B2901088B29010874
:102BD0008B2901088B290108052C0108F52B010818
:102BE000E52B0108002047F0FFFA94F85562C4F87D
:102BF0007802CAE6012047F0F7FA94F85562A4F883
:102C00007002C2E6012047F0EFFA41F21843D34ABE
:102C100094F8556203FB00F3A2FB03239B09A4F87D
:102C20006C32B2E6022047F0DFFA94F85562C4F83D
:102C30007402AAE6D4F8E03294F8E5220133C4F82D
:102C4000E032002A49D03E2384F8C83200E602234D
:102C500084F8583299E647F0C7FA94F8556284F838
:102C60007C0275E7BE480378672213F0020384F8FC
:102C7000C82200F06381BB4BD4F85C52D4F86012D8
:102C800094F864221D605960D4F86852B4F86E124A
:102C90001A7500229D60598284F8C422B24994F8C2
:102CA00067340A68B14D0078D4F850642D68C4F8D0
:102CB000546483F0010342F0200284F867348307F0
:102CC0000A60C4F850547FF5C3ADA64B1B7D042B9E
:102CD0007FF6BEADFFF760FCBAE594F8E83221213B
:102CE000023B84F8C8122E2B3FF6B2AD01A151F879
:102CF00023F000BFDB2E0108152F01085128010821
:102D0000512801087F2E0108512801085128010887
:102D100051280108512801085128010851280108AB
:102D2000512801085128010851280108512801089B
:102D3000512801083F2E0108512801085128010897
:102D4000512801085128010851280108512801087B
:102D5000512801085128010851280108512801086B
:102D6000512801085128010851280108512801085B
:102D7000512801085128010851280108512801084B
:102D8000512801085128010851280108512801083B
:102D9000512801085128010851280108512801082B
:102DA000512801085128010851280108B12D0108B6
:102DB00094F8F43284F87D324922102B84F8C8222A
:102DC00040F2DA80102384F87D32694AA2F1700162
:102DD000A2F16006A2F14005A2F150008946B0467A
:102DE000AE468446002792F808B092F809A009F888
:102DF00001BB013792F80BB008F801AB9F4212F803
:102E00000CAF0EF801BB0CF801ABECD3102B10D0BB
:102E10005A1E114416441544104400220133102B4D
:102E200001F8012F06F8012F05F8012F00F8012FF6
:102E3000F4D1D4F8C0320133C4F8C03242E0494B77
:102E4000D4F800039881D4F80403D88194F8651469
:102E5000D4F80823562084F8C802012042F21075E5
:102E600084F8660492FBF5F21A8200293FF4F0AC74
:102E7000002384F8653484F8663439480EE794F802
:102E8000FB524F23E90784F8C83204D594F8FA328C
:102E9000032B00F083803248037823F00203037091
:102EA000344984F86424D1E900232E4894F81F7330
:102EB000B4F81C6307751343468203D105F00C0573
:102EC0000C2D6DD094F86534002B3FF4C1AC94F810
:102ED0006634002B3FF4BCACCAE7224BD4F8F45262
:102EE0001F4894F864145D60D4F800230A2592FB0F
:102EF000F5F2D4F8F8529A6050221D6084F8C82286
:102F00000378002943D043F002030122037084F8C0
:102F10006524DCE794F8F5325322D80784F8C822F8
:102F200003D594F8F432032B34D00D4803780022F3
:102F300023F00203037084F86424C3E784F8C432E6
:102F4000ACE607F1FF38A044002088F8807247F013
:102F50004BF994F8556288F890021EE6D34D621042
:102F60006C930020B0D900200C89002074C500208B
:102F70000032002058940020002B7FF426AF4849EF
:102F800001F1100601F1300501F1200040E703F0E6
:102F9000FD03BAE7012384F8643493E701227FE755
:102FA0004048B4F9F862D4F8F052A6FB0023F717B2
:102FB00000FB0733D4F8F4623B4F3C4896FBF7FC28
:102FC00035A7D7E9006712EB050843F1000900684F
:102FD00018EB0C0249EBEC7312EB060843EB070904
:102FE000B8EB000269F10003C1E900236AE7B31EF0
:102FF000072B3FF6CAACDFE803F004433E34292137
:10300000140945F05BFEC4F85C02BEE4012047F001
:10301000EBF800EB80004000C4F8680294F85562B9
:10302000B3E4012047F0E0F800EB800000EB800003
:103030008300A4F86E3294F85562A6E4002047F0AD
:10304000D3F894F8556284F864029EE4184A3978FB
:10305000137830298CBF43F0020323F0020313706E
:1030600093E43B78572B7FF490ACD4F860325B420A
:10307000C4F8603289E445F021FEC4F8600284E4BB
:103080003B78532B7FF481ACD4F85C325B42C4F8BC
:103090005C327AE4AFF30080B0F5F79049000000AD
:1030A0009031002000840C2440420F0074C50020A1
:1030B0006C9300202DE9F843C24CD4F868340546DF
:1030C0004BB951E1D4F868042CF080F880B2FFF7D6
:1030D00033FBD4F8683418462CF080F80028F1D17E
:1030E00094F86024531E052B4DD8DFE813F006003A
:1030F0004C00060006009101650094F87461002EF2
:1031000000F09581012E3ED1D4F868042CF05AF8D5
:10311000C8B394F86034032B00F06D84042B00F0E6
:103120002884012B2FD1A84AD4F85C341168CB1A1B
:10313000C72B28D9D4F85834042B00F2D884DFF8F0
:10314000C8C2D4F86804DFF8C4E2C4F85C1403EB26
:1031500043030CEB8302002392F871818768714668
:103160001A4604E0102B00F0F08451F8042F974227
:10317000DEB203F10103F5D1B04500F001855EF840
:10318000281029F003FA914B1B6803F02003002B51
:1031900043D18F4E3378DA0707D494F8793123B9C5
:1031A0008C4A137823F0010313703BF0D9F80546DD
:1031B000002845D1BDE8F883D4F84C3494F8772141
:1031C0000133C4F84C3462B194F86134824A01335B
:1031D000DBB2A2FB0312920802EB82029B1A84F874
:1031E00061347C48794B027877491B687B4E22F02A
:1031F000020202700A680968C4F85024C4F85C141A
:103200000022012103F020033275C4F8582484F809
:10321000622484F86014002BBBD0D4F86C34EB1A11
:10322000002BB6DB6D4B1B7D042BB2D905F5123597
:1032300005F5F8750120C4F86C542CF063F8A8E784
:10324000674B1B8813F4006300F0B88094F8E431F6
:10325000002B00F0498194F860346249624AC978D1
:10326000126884F81C12A3F10503B3FA83F35B0917
:1032700084F80C32C4F8EC21F8F720FD94F85432AD
:10328000002B53D0594AD4F8EC3192ED147AD2ED98
:10329000164AD2ED155A92ED003AD4F87424C4F8C7
:1032A000743427EE077A9B1AA4EEA47A504A07EEEC
:1032B000903AA5EEA57AD4F87034C4F87004C01A18
:1032C000B1EEC76A4B4B12881B88A4F8F031434B10
:1032D000A4F8F4211A7DDB8984F8F821A4F8F631EA
:1032E000DFED452ADFED456A9FED455AD4ED823A80
:1032F00094ED804AF8EEE77A07EE100A67EEA27ABC
:10330000B8EE477A26EE036AC7EE875A66EE267A4B
:1033100065EEA66AE3EE857AE4EE056A84ED816ADD
:10332000C4ED827AC4ED7F5AC4ED806AF8F7C6FC1A
:1033300094F86034052B40F0A280264B1B7813F0E4
:10334000010200F09C80D4F878242E49821A8A4227
:1033500000F2D28094F87C34002B40F0908094F8F6
:103360007D5485F001058BE094F8678418F0020F16
:103370003FF4B6AE154E174A134F306812783968CD
:10338000C4F85834D7F8009084F8623440F0200034
:103390000523C4F85C1491073060C4F8509484F895
:1033A000603406D50D4B1B7D042B02D9FFF7F4F8D2
:1033B000306828F0020184F867142EE084F8E431C4
:1033C00049E700BF102F002074C500200C890020A1
:1033D000309300206C930020CDCCCCCCB0D9002011
:1033E000B093002034930020AC9600208C11001084
:1033F000181E00206E93002000247449CDCC4C3E52
:10340000CDCC4C3F3F420F0020E00508C81B06080A
:10341000A64ED4F850943068A54F3A6840F6C413CD
:10342000A2EB09029A4250D800F02003AFE6012A2D
:1034300000F0E181032A7FF4A6AE9D49D4F85C3404
:103440000A68D31AB3F57A7FFFF49DAED4F85834E6
:10345000C4F85C24002B00F01B83012B40F2328364
:10346000924B0A681B68C4F85C240522C4F85864AF
:1034700084F8626403F0200384F8602487E6002562
:1034800094F8E43184F81D52072B12D8DFE813F0CA
:10349000A6012001F000D3008100580008000E00B2
:1034A0004FF4000011F0A4F91BF01EFF002384F874
:1034B000E4313AF007FB94F8E4310BB13AF0B8FB91
:1034C000002384F85432BDE8F883002320F0200064
:1034D000396830600622C4F85C1484F86024C4F8AB
:1034E000583484F8623454E6012384F8E4313AF025
:1034F0009FFB3AF0E7FAAEE613F0020304BF2A4658
:103500001D466C4B94F89C141B7DC4F8780418BFBE
:10351000002284F87C2494F97E248B422CBF4FF047
:10352000FF330123D31800F16281022B00F3948151
:1035300084F87E3400F09381002384F87D349FE783
:10354000D4F8EC31D4ED827A632BD4BF9FED5A7A54
:10355000B7EE087A67EE877A94ED817AB4EEE77A6F
:10356000F1EE10FA08DD4FF4000011F041F91BF004
:10357000BBFE072384F8E431002301214FF470627D
:1035800084F81A12C4F81032C4F81432A4F81822BD
:103590008FE7B4F8F021B4F8A63493420BD3B4F813
:1035A000A404D4F8EC11642303FB00F39942DCBFBC
:1035B000052384F8E431414BDFED416A13ED016AE4
:1035C000D3ED007A9FED3F7A05EE902AF8EEE55AAA
:1035D000E5EE867A67EEA67AF4EEC77AF1EE10FA97
:1035E000B8BFF0EE477AFDEEE77AC82A17EE903AB8
:1035F00040F22581D4F80025D4F81012632B40F353
:103600001C818B42A8BF0B46632AC4F81032D4F841
:10361000143240F31F819A42A8BF1A4601200A21A2
:10362000B4F88034C4F8142284F81A0284F818120A
:1036300084F819323DE7B4F80435B4F8F021D4F831
:10364000B004C4F810029A4298BF0423B4F8862448
:1036500098BF84F8E431C4F81422B4F8803484F8B4
:10366000193201210F2284F81A1284F8182220E757
:10367000D4F8EC61D4F8B004D4F81032C4F81002D5
:103680009B1B002BB8BF5B42B3F57A7FBCBF032303
:1036900084F8E43101214FF4FA7240F60A7384F899
:1036A0001A12C4F81422A4F8183202E70C89002078
:1036B00074C50020B0D900209A99993F1C3400208D
:1036C0000000C842000000000AD7A339CDCCCC3D91
:1036D000B4F8F0341BB9B4F89434A4F8F034B4F866
:1036E00088341FED076A5FED075ADC4A06EE903A10
:1036F000B4F88C34127807EE103AB4F88A3407EE36
:10370000903AF8EEE66AB8EEC77AF8EEE77AD44B6C
:1037100066EE866A27EE067A67EEA57AC3ED006A42
:1037200083ED027AC3ED017AD30705D44FF400008C
:1037300011F05EF81BF0D8FDB4F8F031B4F89E2417
:103740009A4207D994F81C22062184F8E511002A30
:1037500040F06981B4F88454B4F88624C4F8002594
:103760009D4204D9053B1E2BB8BF1E239DB294F881
:10377000A824B4F88234A4F80455012A07EE903A3C
:10378000D4F8EC6100F0EF80022A40F0DD80C4F84C
:10379000B0643046B4F8A434B4F8A62406EE903AE7
:1037A000B8EEE67AF8EE676AAA1A76EEC76A07EE0E
:1037B000102AB8EEC77AF8EEE77A86EE876AA94A49
:1037C000022184F8E41107EE105AB8EEC77AA2EC91
:1037D000016AE6EE477AC2ED007A4DE7337813F0DE
:1037E000010341D1C4F8E831A4F8F23161E60023C5
:1037F00084F87E34A0E69C49D4F85C340A68D31A75
:10380000B3F57A7FFFF4BFACD4F85834C4F85C2425
:10381000002B00F01181012B40F24E81934B0A687E
:103820001B68C4F85C240322C4F8586484F86264FA
:1038300003F0200384F86024A9E46423E4E6B4F8E8
:1038400086048B4902FB00F2A1FB02129209C4F824
:103850000025D1E66422E1E6022384F87E340123C8
:1038600084F87D3400250BE694F8B434002B3FF443
:1038700020AE804BD4F8E801D3ED037A7E4AD4F829
:10388000EC31B4F8F251B4F8F011D2ED086AFCEE64
:10389000E77A9842B8BF184617EE903AF6EE007AEB
:1038A000A942F4EEE76A38BF29469BB20025F1EE43
:1038B00010FAA4F8C034C4F8E801A4F8F211C4F86E
:1038C000BC54C4F8B8547FF7F4ADDFED6C7AF4EE75
:1038D000E76AF1EE10FA7FF5ECADD4F8E814DFED0D
:1038E000687A07EE101AB8EE477AB4EEE77AF1EE8E
:1038F00010FA7FF5DEAD40F22E4083427FF6D9AD5F
:10390000A3F57A7307EE903AB8EEE77ADFED5D7AC9
:10391000E7EE267A4D1CFCEEE77A17EE903A9BB262
:1039200007EE903A002940F03F81F8EE677A02F105
:103930002803B0EE670AC3ED007A48F0E3F8C4F854
:10394000E854A4F8F004B4E5D4F8E82102F2DC501D
:1039500017EE902A642303FB02F39842B8BF18467F
:10396000C4F8B00416E7642000FB03F0C4F8B00408
:1039700010E794F87621002A00F0A88094F86224D9
:10398000002A40F0968084F86264D4F85834B22B50
:1039900000F2C5803C4AD4F868042B2B134494BF32
:1039A00093F8AC1193F8D8112BF01CFCD4F85834D0
:1039B00094F862240133C4F85834022A00F09E803F
:1039C000032A00F0C580294E3368032A03F0200340
:1039D0007FF6DDAB244A33681268C4F85C24052105
:1039E000002203F0200384F86014C4F8582484F8FB
:1039F0006224FFF7CCBB94F86134234A2349D4F8FE
:103A0000680403EB430302EB830393F8713151F82D
:103A1000231028F0BBFD144A144B12681B68C4F82D
:103A20005C240421DCE74FF4000010F0E1FE1BF001
:103A30005BFCB4F8F0318DE64FF49651D4F868048D
:103A400028F0A4FD094BD4F858241B68013203F078
:103A50002003C4F85824FFF79ABB00BF6C930020E2
:103A6000043400201834002074C500200C89002084
:103A70001F85EB5178930020D43300208FC2753F0F
:103A80000024744900007A4420E00508C81B060899
:103A900094F861344D4A4E49D4F8680403EB43036B
:103AA00002EB830393F8713151F8231028F06EFD77
:103AB000C8E7012A81D168E74649D4F868042BF0A9
:103AC00095FBBFE74449D4F86804F8E7434B444901
:103AD0001B680868C4F85824052184F8622403F0A0
:103AE0002003C4F85C0484F86014FFF750BB3B4B20
:103AF00012681B68C4F85C24032171E7D4F85834B9
:103B0000092B12D90F2B43D994F8782100230321D4
:103B1000C4F8583484F8621412BB304E5AE70023BC
:103B20000222C4F8583484F86224284AD4F868047D
:103B3000134493F88C122BF055FBD4F8583494F8B6
:103B400062240133C4F858343AE70026FFF714BB67
:103B500094F87831002BE0D0D4F85834432BDCD8DB
:103B60001A4AD4F86804134493F8BC122BF03AFBB9
:103B7000D4F8583494F862240133C4F8583422E756
:103B800094F861340C2202FB03C3D3F8741196E756
:103B900094F875110D4AD4F86804C1EBC1010A44C8
:103BA000134493F88F12C6E792ED0A6A07EE105A93
:103BB000F8EEE77AF8EE476A77EEC67A134687EEB4
:103BC000A67A283377EE067AB3E600BF20E0050830
:103BD000C81B0608A8660608C86606080C890020E7
:103BE00074C5002078B310B582B040F25514AA22F3
:103BF00000238DF80210ADF800408DF803208DF8F9
:103C00000430694655220DF103045340082213F095
:103C1000800F4FEA430318BF83F03103013ADBB250
:103C2000F5D1A14202D011F8012FEEE702688DF81C
:103C30000330536AAA228DF80420694605221BB17D
:103C4000984702B010BD70472BF076FAF9E770B5CF
:103C500090F8603044699AB073B94268537884F838
:103C60004430D1789378012243EA0123A4F8463006
:103C700084F848201AB070BD054602E020682BF099
:103C8000A5FA20682BF0AAFA0028F7D10146622293
:103C90000DF1060049F07CF9144A1549D2F81435A3
:103CA0000968144C92F8102503930B44179204935F
:103CB000114A6B69A6781148029040F2FF51ADF8A5
:103CC0000410CDE905235EB96078642202FB004050
:103CD00001A9043047F036FE01226B696670A270BC
:103CE0001868FF211AB0BDE870407BE7102F002054
:103CF00074C5002070D20020BD0B010830D2002016
:103D000090F8603063B910B50278032A0DD0042A08
:103D100019D0022A1C4C0FD0002384F8203510BD86
:103D2000194B002283F820257047174C84F8213561
:103D3000002384F8203510BD012384F821350023A9
:103D400084F8203510BD4268017E52780E4C012067
:103D5000814202F00F0284F8210509D00229DBD14B
:103D6000002AD9D0162084F8223510F0ADFBD3E715
:103D70002AB1152084F8221510F0A6FBCCE71620F6
:103D800010F0A2FBC8E700BF102F002008B5044BBD
:103D900093F8233513B901210DF026FF002008BD4B
:103DA000102F002038B50A4846F03CFE084AC0B241
:103DB0000023024420251918CCB2092C05D9054B43
:103DC0000B44002283F8242538BDD5540133F2E793
:103DD00034340020102F002038B50A4846F022FE67
:103DE000084AC0B20023024420251918CCB2142C72
:103DF00005D9054B0B44002283F8242538BDD55442
:103E00000133F2E734340020102F00202DE9F04177
:103E1000144C94F8965385421BD9064610468846A2
:103E2000174646F0FFFD04F51B73AA1B05FB08654A
:103E300082421D44A8BF024639462846164649F02C
:103E40007FF84444002814BF0123002384F88C33F6
:103E500001D1BDE8F081324639462846BDE8F0413F
:103E600047F070BD181E002030B583B014460D46D3
:103E70001A4601A8074916F07DFC074B93F89533C5
:103E8000A34204D901AA21462846FFF7BFFF00201C
:103E900003B030BDE0660608181E0020074890F801
:103EA0009503904207D908B5084611461A46FFF710
:103EB000ADFF002008BD0020704700BF181E002085
:103EC000082A07D808B5084611461A4627F047FCC5
:103ED000002008BD00207047F8B507460026F5B25F
:103EE0000024E0B220222946013427F038FC0C2CB3
:103EF000F7D10136092EF2D11B4D422201200021BB
:103F0000441C27F02CFC15F8012FE4B22046002AAF
:103F1000F5D197F90F302BBB144D14464D22E0B26A
:103F2000022127F01CFC15F8012F0134002AF6D1DC
:103F30000F4D2B2202200321441C27F010FC15F802
:103F4000012FE4B22046002AF5D10A4D2B2202208F
:103F50000421441C27F003FC15F8012FE4B220468D
:103F6000002AF5D10020F8BD0C670608FC6606089B
:103F7000F0660608E466060810B50024C473FFF76F
:103F8000ABFF204610BDF8B5084617465E1E16F872
:103F9000015F421CD4B239462A462DB1082F01D800
:103FA00027F0DDFB2046F2E72846F8BD70B50B4C44
:103FB0004FF0FF3504F528762368E034184643B106
:103FC00093F83830142B04D02BF004F9854228BF25
:103FD0000546A642F0D1284670BD00BFDCD20020C5
:103FE00010B50B4B0B4993F83D2593F83C350978F8
:103FF00082B00D321E330424027243728DF80440E5
:1040000021B901210DEB040044F014F802B010BDF9
:10401000102F00205C930020F0B518468BB01C4692
:104020000E46174646F0FEFC1E2828BF1E2003231E
:10403000214602460546002402A88DF804308DF87A
:1040400005708DF806608DF8074047F07BFC064B45
:104050001B7813B120460BB0F0BD291D01A843F019
:10406000E9FF0BB0F0BD00BF5C93002010B582B03B
:1040700000248DF8043001AB8DF80540FFF7CCFF2C
:1040800002B010BD00B5094B83B01B7804228DF837
:1040900004201BB1002003B05DF804FB01210DEBEF
:1040A000020043F0C7FF03B05DF804FB5C930020FF
:1040B00000B5094B83B01B7802228DF804201BB198
:1040C000002003B05DF804FB012101A843F0B2FF1A
:1040D00003B05DF804FB00BF5C93002000B5084B03
:1040E00083B01B7801218DF804101BB1002003B0B0
:1040F0005DF804FB01A843F09DFF03B05DF804FBED
:104100005C93002000B5074B83B01B7800208DF82E
:1041100004001BB9012101A843F08CFF03B05DF836
:1041200004FB00BF5C930020ECE710B5044619F0D7
:104130001FF818F09FFB084A084B127B93F84515AF
:1041400093F8443512F0400F14BF10220D220A4498
:104150001E332272637210BDA0010020102F0020B8
:1041600019F0D8B90F2A07D808B5084611461A46DB
:1041700018F00EF9002008BD0020704708B5044B68
:1041800093F849350BB919F015F9002008BD00BFA7
:10419000102F002010B5094C94F8460519F08CFA40
:1041A00094F8481594F8470519F0DAF94FF4F072CD
:1041B0002021034848F0ECFE002010BD102F002005
:1041C000B021002038B5A0F668040022606C354D9F
:1041D00003685A62A1F12903302B31D895F84A358A
:1041E0000133DBB2012B85F84A350BD995F84B35F5
:1041F00085F84A25B4F8562801335208A4F8562801
:1042000085F84B3595F84B250023082AA4F8583833
:1042100015D185F84B35B5F84C3501339BB2032BDE
:10422000A5F84C3508D92379DB0705D5E36A94F85E
:10423000560853B3216B98470023A4F8563838BD6D
:104240005B396C290ED8B4F8563885F84A255B08D6
:1042500043F08003A4F8563895F84B35013385F8C0
:104260004B35CFE794F85138002BCBD1012185F89D
:104270004A35A5F84C35802384F85118A4F85638EF
:1042800085F84B1543F01AFDBCE7E3696269D05429
:10429000E369E1680133B3FBF1F201FB1233E3613F
:1042A000CAE700BF102F002038B5A0F668042379B4
:1042B0006579DB0722D594F84C3803B3D4F8483439
:1042C0001A68D36A5B08536294F8503823B1B4F883
:1042D0005A380133A4F85A38E94301F00101606CFF
:1042E00043F0ECFC012384F84F38002384F84D3868
:1042F00084F84E38A4F8563884F84C3838BD94F811
:104300004F38012B04BF94F84D3884F84E382046BE
:10431000FCF7A2FD94F84F384BB90123E94384F828
:104320004F381940606CBDE8384043F0C7BC0023EB
:1043300084F84F3805F00101606CBDE8384043F067
:10434000BDBC01EB81010D4B70B5A1F1A1051D4470
:104350009C3B06465C1815F8013F717996F90400FC
:1043600040223FF017FFA542F5D1717996F904007C
:1043700000234022BDE870403FF00CBF20E3050859
:1043800038B505464C1E14F8011F01B938BD284642
:10439000FFF7D7FFF7E770B505460C468E1814F8FF
:1043A000013B697995F9040080223FF0F3FE08B1E2
:1043B000A642F4D170BD07B501EB410301EB410109
:1043C000C1F3C301503A10315B008DF8042003F0B3
:1043D0000E038DF80610032201A98DF80530FFF7B2
:1043E000DAFF03B05DF804FB38B504461D464068AB
:1043F000FFF7E1FF60682946FFF7A3FF002038BD03
:1044000038B504461D464068FFF7D5FF6068294669
:10441000FFF7B6FF002038BD0A460021CBE72DE9A3
:10442000F0410F4FDFF84080002407F2245638F99E
:1044300014300C492246304616F09CF9FFF7CCFCAC
:10444000D7F850550134E1B22846FFF7E5FF314671
:104450002846FFF795FF042CE9D1BDE8F08100BFA5
:10446000102F00208B63060864BA00202DE9F04766
:104470002D4DDFF8C080D5F850452DED028B20463C
:104480008EB00121FFF7C8FF204628499FED288AFA
:10449000FFF776FF0024022605F2245704A9E0B2B4
:1044A0000EF0F2F89DF81830ABB3062C33D0DDEDEA
:1044B000087A099B0B98B8EEE77A41F2883EC8EE7D
:1044C000077A42F2107C06F101095FFA89F9FDEEE4
:1044D000E77A17EE902A00FB02E102FB03E2B1FB50
:1044E000FCF1B2FBFCF20291CDE90002414622460A
:1044F000384616F03FF9FFF76FFCD5F850A5314666
:104500005046FFF789FF39465046FFF739FFB9F1AA
:10451000080F03D84E4601341B2CBFD10EB0BDECA2
:10452000028BBDE8F08700BF102F002094630608BF
:1045300000247449AA6306082DE9F743554C564EEA
:10454000D4F8505501212846FFF766FF5349284605
:10455000FFF716FF3368990740F19980504D95EDAC
:10456000140A47F0CFFA95ED150A074647F0CAFA44
:1045700095ED160A804647F0C5FA3B46494A4A4936
:10458000CDE9008004F2245016F0F4F8FFF724FC83
:10459000D4F8505502212846FFF73EFF284604F282
:1045A0002451FFF7EDFE03253368DA0725D53F4F89
:1045B00097ED0F0A47F0A6FA97ED100A804647F0EC
:1045C000A1FA97ED110A814647F09CFA4346384A12
:1045D0003549CDE90090374816F0CCF8FFF7FCFBE1
:1045E000D4F8508529464046FFF716FF314940462A
:1045F0006F1CFFF7C5FEFFB23D4633681B0727D58A
:104600002D4E96ED000A47F07DFA96ED010A074619
:1046100047F078FA96ED020A804647F073FA3B4677
:10462000264A2149CDE90080A6F1300016F0A2F813
:10463000FFF7D2FBD4F8508529464046FFF7ECFE41
:10464000A6F1300140466F1CFFF79AFEFFB23D46CF
:104650001B4A0A20B2F90030B2F9041091FBF0F1C4
:104660000191B2F9022000920F49164A114816F042
:1046700081F8FFF7B1FBD4F8504529462046FFF7F3
:10468000CBFE0C49204603B0BDE8F04378E6022596
:104690008AE700BF102F00200C890020BA630608AB
:1046A0008C110010D0630608D463060820040010A3
:1046B000E36306083434002064340020E76306080E
:1046C000B4930020EB630608804B1B6813F0800F47
:1046D0002DE9F0417E4C07D194F86C3543F002038C
:1046E00084F86C35BDE8F081D4F8C022D4F8743574
:1046F0009A420DD094F87835C4F874250133DBB2B2
:104700000522B3FBF2F202EB82029B1A84F87835A1
:10471000D4F85065DFF8F481012200213046FFF71C
:104720004AFE94F878256B4B1344304693F8A31552
:10473000FFF707FE012202213046FFF73CFE00256D
:10474000362718F80510C1EBC10191FBF7F10629D6
:10475000A8BF06216039C9B230460135FFF7F1FD27
:10476000102DEED15C4B5D4D1B782A7D5C495D4878
:1047700013F0020F0CBF4E23592315F0FBFFFFF778
:104780002BFBD4F8506502213046FFF745FE30463A
:104790005449FFF7F5FD29686B68534A514893FB6C
:1047A000F2F391FBF2F2514915F0E4FFFFF714FB2D
:1047B000D4F8506503213046FFF72EFE30464949B4
:1047C000FFF7DEFDEA894A49464815F0D3FFFFF7B7
:1047D000E9FAD4F8506504213046FFF71DFE304653
:1047E0004049FFF7CDFD2A8A42493E4815F0C2FFF5
:1047F000FFF7D8FAD4F85055042228460A21FFF7CB
:10480000DAFD28463749FFF7BBFDD4F8E0223A49E4
:10481000344815F0AFFFFFF7C5FAD4F8505505211D
:104820002846FFF7F9FD28462E49FFF7A9FDD4F8E1
:104830004C34D4F8482431492A4815F09BFFFFF73F
:10484000B1FAD4F85055052228460A21FFF7B3FDE6
:1048500028462449FFF794FDD4F85434D4F8502462
:1048600027492048D21A15F085FFFFF79BFAD4F8A4
:10487000505506212846FFF7CFFD28461949FFF776
:104880007FFDD4F84C241F49164815F073FFFFF73D
:1048900089FAD4F85045062220460A21FFF78BFDFD
:1048A00020461049FFF76CFD1749152201F51770D6
:1048B00048F0ACFBFFF776FA20460721FFF7ACFD86
:1048C00020460849BDE8F0415AE500BF8CD80020D9
:1048D000102F002020E005086C930020B0D90020A4
:1048E000EF630608343400208096980000640608C0
:1048F0000D640608156406081C640608236406088F
:104900002C64060833640608D8310020B03100203A
:10491000F7B5374B374F5C78374907F224562246B4
:10492000304615F027FFD7F8505501212846FFF7EC
:1049300073FD31462846FFF723FD3049304615F018
:1049400019FFFFF749FAD7F8505502212846FFF71B
:1049500063FD31462846FFF713FD222303FB047451
:10496000304694F8811594F8803594F87F250091AD
:10497000234915F0FFFEFFF72FFAD7F85055032112
:104980002846FFF749FD31462846FFF7F9FC94F821
:10499000871594F8863594F8852500913046194995
:1049A00015F0E8FEFFF718FAD7F85055042128460D
:1049B000FFF732FD31462846FFF7E2FC94F88415F4
:1049C00094F8833594F88225009130460E4915F00D
:1049D000D1FEFFF701FAD7F8504505212046FFF731
:1049E0001BFD3146204603B0BDE8F040C8E400BFDF
:1049F0008CD50020102F00203B6406084C6406086C
:104A00005F64060872640608856406082DE9F347AA
:104A10001D4B1E4C1A781E49DFF87CA0DFF87C90F5
:104A200004F2245015F0A6FED4F850550121284672
:104A3000FFF7F2FC284604F22451FFF7A1FC154BC6
:104A40001E68002504F22458B27A337A0192727AF1
:104A5000009249465AF82520404615F08BFEFFF794
:104A6000BBF9D4F85075A91CC9B23846FFF7D4FC7D
:104A7000013541463846FFF783FC032D06F1060653
:104A8000E2D102B0BDE8F0878CD50020102F0020C5
:104A900098640608BC960020C8E50508A4640608CA
:104AA00038B50E4C0E4B0F4A0F4904F224552846D8
:104AB00015F060FED4F8504501212046FFF7ACFC0C
:104AC00029462046FFF75CFC20460221FFF7A4FCA4
:104AD00020460649BDE8384052E400BF102F0020B0
:104AE000B9640608C3640608C9640608D2640608E7
:104AF00038B5042208490546FFF74DFC4FF48064A1
:104B0000013C00234022697995F90400A4B23FF0EA
:104B100041FB002CF4D138BDD4E5050808B5406848
:104B2000FFF7E6FF002008BD094B03EB40039A891D
:104B3000084B5B7B03F0070313EAD22307D0064B35
:104B40001A68511C1960054B134483F848067047D6
:104B5000181E0020A001002078990020102F0020AE
:104B600030B585B0054601A815F0B2FE044618B967
:104B70002870204605B030BD044A0123B2F98026D2
:104B800001A9284615F0FCFEF3E700BF102F002016
:104B90004068E5E72DE9F04704468AB0C8B1AA4B62
:104BA000D3F82802037A9C422246A8BF1A469C42A8
:104BB000BABF0132012500259C1A022194FBF1F4B1
:104BC000E4B235B12246A14B651C2BF0A1F9EDB240
:104BD0002C469F4FDFF8C88200263D4616F8083065
:104BE000D7F8901001229A400A422DD0172B2BD8CB
:104BF000DFE813F0180031004A007D00A200C80071
:104C0000DD00F20006011601580158006A01A501F5
:104C1000B801D501E801F401B30005022C02380205
:104C20004C021E0202A8FFF79BFF18B9894902A88F
:104C300015F0A0FD844802AB22460221D0F82802DC
:104C40002BF066F90134E4B20136182EC6D12046A5
:104C50000AB0BDE8F087B5F88220002312F00F02F9
:104C6000194618BF012202A8FCF71CFEB5F88230D5
:104C700003F00F02784B03EB8203204602AAD3F81D
:104C8000D015FDF703FCDDE7B5F88420012312F011
:104C90000F0218BF1A46002102A8FCF703FEB5F860
:104CA0008430E5E7684BD3F89C01FBF763FC95F88B
:104CB00081C0BCF1000F4FF00A010CBF4FF00F0C88
:104CC0004FF00C0C90FBF1F3CDF800C093FBF1F228
:104CD00001FB12336149642290FBF2F202A815F045
:104CE00049FD02AA5E492046FDF7D0FBAAE75D4BCD
:104CF0001B681B06A8D5544BB3F9902195F8813059
:104D00008BB942F2107312FB03F2574B92FBF3F292
:104D10009D23564902A815F02DFD02AA54492046AC
:104D2000FDF7B4FB8EE702EBC2024FF47A739200F8
:104D300092FBF3F29E23ECE74A4B1B68180683D5DF
:104D4000414B02A8B3F9A0110022FCF729FC02AAEA
:104D500048492046FDF79AFB74E7424B1B68190649
:104D60007FF572AF384B02A8D3F88011002264237C
:104D7000B1FBF3F1FCF714FC02AA3F492046FDF712
:104D800085FB5FE7304BB3F99211642391FBF3F29B
:104D900003FB1213062100911BB2384902A815F03B
:104DA000E9FC02AA36492046FDF770FB4AE7264B8C
:104DB000B3F894116423B1FBF3F203FB1213062141
:104DC00000919BB22D4902A815F0D4FC02AA2D49EE
:104DD0002046FDF75BFB35E72B4B19886423B1FBBD
:104DE000F3F203FB1213062100919BB2234902A8A0
:104DF00015F0C0FC02AA25492046FDF747FB21E734
:104E0000114B02A993F8980143F0CEFF204902A864
:104E100048F0C6F802AA1F492046FDF737FB11E704
:104E20001D4B9B7A002B3FF40FAF074A0F49B2F995
:104E300096219A2302A815F09DFC02AA1749204644
:104E4000FDF724FBFEE600BF102F0020DC640608FF
:104E5000181E0020EC64060820E0050835620608EC
:104E6000F36406088CD8002040D206003862060899
:104E7000006506080A65060817650608DE97060835
:104E80002765060833650608709300203765060815
:104E9000606506083F650608889300204865060897
:104EA000D8E50508894B9B7A002B3FF4CDAE884AA4
:104EB00088499268072302A815F05CFC02AA86497B
:104EC0002046FDF7E3FABDE6DFF81C9299F8863636
:104ED000002B3FF4B9AE032B3FF4B6AE07F0ECFA6B
:104EE00099F88636012B22D120B342F07BFA814615
:104EF00016F054FF824616F0F3FC6423800A5843F0
:104F0000B9F80220B9F8043074499A1ADAF8043072
:104F100002FB03339B0AB0FBF3F302A89AB215F02D
:104F200029FC02AA6E492046FDF7B0FA8AE600285D
:104F300040F0CB806B4902A815F01CFCF1E76A4BEE
:104F400093F88636002B3FF47FAE032B3FF47CAE04
:104F500002A9002043F028FF02AA64492046FDF779
:104F600095FA6FE6624B1B689A077FF56DAE5E4B54
:104F700093ED690AF2EE047A20EE270A46F0C2FDAC
:104F80000A235C4990FBF3F203FB120302A815F01D
:104F9000F1FB02AA58492046FDF778FA52E6524B37
:104FA000B3F9A801FCF78EFF0246FBF7D9FA49498D
:104FB000034602A815F0DEFB02AA50492046FDF781
:104FC00065FA3FE6484B02A9D3F8AC0143F0ECFE8A
:104FD00002AA4B492046FDF759FA33E6424B4949AC
:104FE000B3F8B02102A815F0C5FB474902A847F065
:104FF000D7FF02AA45492046FDF748FA22E6444B6E
:105000001B689B007FF520AE424BB3F818264AB1CF
:10501000414902A815F0AEFB02AA40492046FDF71F
:1050200035FA0FE63E4A3D492046FDF72FFA09E6DC
:105030002D4B3C4993F8B22102A8524215F09AFB3D
:1050400002AA39492046FDF721FAFBE5264B02A9C1
:10505000D3F88C0643F0A8FE02AA34492046FDF797
:1050600015FAEFE5204B3C21D3F89036B3FBF1F372
:1050700002A893FBF1F201FB12332D4915F07AFBE4
:1050800002AA2C492046FDF701FADBE5164BD3F8BE
:10509000942695F8813073B940F249617E23B2FBC2
:1050A000F1F202A80B4915F065FB02AA224920463D
:1050B000FDF7ECF9C6E54FF47A717D23B2FBF1F20E
:1050C00002A8044915F056FBEFE7FFDE88930020A5
:1050D000A493002038620608546506085D6506083A
:1050E0006865060862650608102F002071650608CD
:1050F0000C890020B46206087C65060888650608ED
:10510000956506084381060860650608A1650608DE
:105110008CD8002020040010AA650608AF65060898
:10512000B865060831620608C1650608CE6506083E
:10513000DC650608E5650608F76506082DE9F04F09
:10514000D04DD14C95F85D328FB0074613B1012395
:1051500084F82032D4F89C360526B3FBF6F606EB2D
:1051600086069E1B40F01C83C84A94F8A01613784C
:1051700003F00103994290463DD0002B00F0FB80E4
:10518000C34BC4F89031632384F898310023C4F8EA
:10519000A43194F87031D4F8280284F8A166012B68
:1051A00014BF63234FF49673A4F8B03184F8A26659
:1051B000C4F89C61A4F8A061C4F88C61C4F894613F
:1051C000A4F8A861C4F8AC6184F8B2612AF0C4FE06
:1051D000B04BD4F8280207220C212AF099FE07F5DB
:1051E000F42303F59073C5F8A03598F8003003F068
:1051F000010384F8A03698F8003013F0010300F0A2
:10520000F88094F87A21A44B002A00F0DB80B3F9EF
:105210000C30B4F990219A42B8BFA4F890319F4B5A
:10522000B4F99221B3F900309A42C8BFA4F8923180
:105230009B4B64221B6893FBF2F3B4F996211BB2DB
:105240009A42B8BFA4F896312EF0DAFF94F898315C
:10525000D4F89C21D4ED6D7A94ED697A8342914B18
:1052600088BF84F898011B68B4EEE77A9A42B8BF09
:10527000C4F89C31F1EE10FA48BFC4ED697A2EF003
:1052800091FFB4F8B02103B29A42874B94F8B2214F
:10529000DB79C8BFA4F8B0019A4238BF84F8B231B4
:1052A000824B1B7803F00303032B07D1804BB4F927
:1052B000A0211B889A42B8BFA4F8A0317D4B1B687F
:1052C00013F0006309D0D4F82422B4F9A81192F99C
:1052D00001209142B8BFA4F8A821774A91791046DD
:1052E000002979D0754BDFF8E4C11A7800210B460C
:1052F00091426ADBB3FBF2F2C8235343827EB3FBD5
:10530000F2F3D4F8AC219A42B8BFC4F8AC31D4F867
:10531000A836D4F88821FB1A1A44C4F88821D4F896
:105320008C211344C4F88C31D5F8A035C4F8A87684
:10533000002B00F0D680FB1A002BD4F8280280F254
:10534000C7805F4AB2F9061040F2D663994203DC87
:10535000B2F902209A4201DDC5F8A0752AF0CAFD13
:10536000002384F82032D4F89C360133C4F89C36EC
:105370000FB0BDE8F08FD5F89030002B3FF435AF7B
:1053800094F8A336002B7FF430AF4E4B1B6813F01C
:10539000600F08D0444BEA8E5B7B03F0070313EAEF
:1053A000D2237FF422AF012384F8A136464B3B443D
:1053B000C5F8A035394B1B88A4F89431002384F834
:1053C000A43612E7B3F90E3023E70CEB810E01315E
:1053D000BEF80CE073448BE7002B92D0D4F8243253
:1053E000927E9B89642113FB01F3520893FBF2F335
:1053F00087E794F8A126002A96D0D4F82892B9F12C
:10540000000F0AD099F90F20002A06DD84F8A13692
:10541000C5F8A035C4F88C3186E70E2039F00AF8BB
:1054200094F8A23648B1002B3FF47EAF00234846E3
:1054300084F8A2362AF090FD76E723B9012284F899
:10544000A226C4F8AC36D4F8AC369F42FFF46CAF59
:1054500007F5742303F510734846C4F8AC362AF0F8
:105460007BFD94F8A40638B9FFF794FB84F8A406F2
:10547000D4F828022AF070FD94F8A406FFF78AFBFE
:1054800052E700BF181E0020102F0020309300208C
:1054900000008813FA610608B0D90020709300203C
:1054A000A4930020AC960020A00100206C93002063
:1054B0006E9300208CD8002078BA00208411001050
:1054C00040DA0020B496002000879303EC1100100E
:1054D0002AF042FD0023C5F8A03584F8A136C4F8AF
:1054E0008C31B24B1A6812F0006F994604D0FF203D
:1054F00025F07AF8C4F82402AD4B00931A6812F034
:10550000020F24D0AB4BB5F860205B7B03F00703A0
:1055100013EAD22303D1D5F89030590417D5A64BFE
:10552000D4ED6D7A93ED006AD3ED016A93ED027AC2
:10553000A24BE6EE067AE6EEA67AE7EE077AB1EE41
:10554000E77AD3ED007A67EE877AC4ED6D7AD4F806
:1055500028A2BAF1000F04D09AF90F30002B3FF7C0
:10556000FFAE974B1868FBF705F883462EF048FE10
:1055700095F88020D4F8B83182428CBF43F0010303
:1055800023F00103C4F8B83101932EF00BFEB5F8F7
:10559000D210D4F8BC21019B81428CBF42F48042DE
:1055A00022F48042C4F8BC2195F85A22002A4AD13C
:1055B00023F4800323F00203824AC4F8B83112783E
:1055C00092070DD5804A127D042A09D994F89C14BB
:1055D00091424BD9019338F0C3FE019B002845D07E
:1055E00043F48043C4F8B831B5F88230019303F036
:1055F0000F00FCF73DF9019B744A1B0A5A4327D15F
:10560000D4F8B83123F02003C4F8B831B5F88430A9
:10561000019303F00F00FCF72BF9019B6B4A1B0A67
:105620005A431CD1D4F8B83123F04003684AB5F886
:105630007C009268D4F8BC1190421ADD23F010224D
:1056400021F0200119E043F4800343F00203B3E7A3
:105650009042D4F8B831D3D343F02003D4E7824248
:10566000D4F8B831DED843F04003DFE723F48043B9
:10567000B8E743F0102241F0200164239BFBF3FBC9
:10568000B5F87E30C4F8BC119B4524DB98F8003097
:10569000D80720D542F40042D9F80030C4F8B82128
:1056A0001B010ED595F9942012F1800F16D0D4F875
:1056B000243293F90130934210DB41F00801C4F821
:1056C000BC1150462AF048FC0E2038F0B3FE50B111
:1056D000D4F8280242E622F40042DDE721F0080176
:1056E000C4F8BC11EDE7009B94F8BC261B68D4F805
:1056F0002882C3F340139A4203D084F8BC3626F0C4
:10570000F9FD2C4B334ADFF8D8A0B7FBF2F707F0CE
:1057100001079F739B46DAF800309E42D8D22E4B89
:10572000F35C590904EB810103F01F000122D1F859
:10573000B81182400A4202D09BF80E2072BB05EBE2
:1057400043020021978900931C220DEB0200069171
:1057500047F01EFC0122009B8DF814201F4A8DF893
:10576000083002EB830206A907F01F09C7F34417AC
:105770000391D2F8E0358DF809908DF80A70CDF8D4
:10578000108002A8009198479DF8143000992BB121
:105790000B463A46494640462AF0BAFB0136BAE77C
:1057A000D4F828020368DB689847DCE58CD8002031
:1057B0000C890020A0010020C03500208C110010B1
:1057C000AC9600206C930020B0D900200087930392
:1057D000A4930020400D03005835002020E0050868
:1057E00078990020074B032883F89C0003D8064AC9
:1057F000012310B9537326F07DBD013803FA00F080
:105800005073F8E7181E0020A0010020044A01236D
:1058100003FA00F0D2F890300343C2F8903070479A
:10582000181E002038B50146831E00F16E02EA20E2
:1058300023F8020F9342FBD143F649134B85304BBB
:105840004B600024CE230B81C1F884400320FFF776
:10585000DDFF0520FFF7DAFF0820FFF7D7FF09205B
:10586000FFF7D4FF0A20FFF7D1FF0C20FFF7CEFF90
:105870000D20FFF7CBFF0220FFF7C8FF01252148CD
:1058800081F87550D0F88820234605FA03F40133D7
:10589000102B42EA0402F8D14FF4206322F4604254
:1058A000C0F88820A1F8763040F60123A1F87830BE
:1058B000154B0B67142381F87430802381F88830EE
:1058C00042F61403A1F880304FF6FF73A1F88A3036
:1058D000A1F88C304623A1F88E3040F20123A1F8C4
:1058E0009030002381F8923081F8A33081F8B430F1
:1058F0005023A1F8C6303C23A1F8C83038BD00BF02
:10590000CD004E00181E00209808640010B5084B0A
:10591000084909480024FF2281F8BD46DA73FBF7E5
:10592000B3FB064BBDE8104093F86202FBF7B0BA38
:10593000A0010020102F002038E00508181E0020CC
:105940000F2A03D8052803D805290CD90020704751
:10595000062812D00728F9D10029F7D10B4B0120D6
:1059600083F8CF217047094B00EB400003EB400068
:105970000144012081F8A02170470A29E6D8034B91
:105980001944012081F8C421704700BF181E00206F
:105990001B4B2DE9F04100F120070C4603EB870873
:1059A00040F267160025204615F024FB03469E4270
:1059B0004FF02C0120461CDB95B1114E06EB8706FB
:1059C0002C2186F8E23047F0FAFA90B1013015F058
:1059D00011FBFF280DDC86F8E3002846BDE8F081C6
:1059E000A8F8E03047F0EBFA18B1441CFF26012577
:1059F000D9E7044B002043F82700BDE8F08100BF41
:105A0000181E0020F81E002078492DE9F0430025DB
:105A100008462E462B460AE0062C03F1010308BF78
:105A20000136940448BF0135202B00F0C68050F8A1
:105A3000042BC2F30324002AEED16D4F6D4A87F880
:105A4000DC30F6B2012087F8DD6087F8DE50C7F859
:105A5000A8359071002B00F0BE8000204FF00F0E93
:105A6000F04605460446894659F8042BC2F3031C48
:105A7000654502F00F02B8BF6546E045A8BFE046A5
:105A8000904204F10104B8BF10469645A8BF96465F
:105A90009C42E9DB454540F38D8045446C10013460
:105AA000013D64B245F34702704587F8562287F8F6
:105AB000554278DD704444100134013864B240F33B
:105AC00047024D4887F85322A0FB0602920802EBDA
:105AD0004202A6EB420212F0FF0F87F8544267D051
:105AE000062E324608D9F00706D401E0D50702D4C5
:105AF0005210062AFADCD6B287F8DF60002B71D08C
:105B0000D7F8E050C5F305356C074FD40C1F04EBF4
:105B100083040A4603E052F8040F400446D494423A
:105B2000F9D10126AC070CD40C1F04EB83040A4600
:105B300003E052F8040F870403D49442F9D146F0ED
:105B400002066A090CD10C1F04EB83040A4603E029
:105B500052F8040F800303D49442F9D146F48076BE
:105B600028070CD40C1F04EB83040A4603E052F808
:105B7000040F070403D4A242F9D146F01006EA0646
:105B80000BD40A1F02EB830303E051F8042FD50363
:105B900003D48B42F9D146F00806B6B2174BA3F8EE
:105BA000BE66BDE8F083062207248AE70026B9E72F
:105BB0000626A1E70622072476E70D4F0D4A87F84F
:105BC000DC30F6B2012087F8DD6087F8DE50C7F8D8
:105BD000A835907141E70622072487F8562287F8F6
:105BE00055426EE740F21B16D8E700BFF81E0020B2
:105BF000181E0020A0010020ABAAAAAA102F002086
:105C00002DE9F04F714ADFF8D0B1002389B042F896
:105C100020300C4602909A46019319461E4699463A
:105C20001F464FF02C0E4FF0010823785FFA8AF5DB
:105C3000A3B173457ED0601C0DF1140C00220CF84A
:105C4000013B044610F8013B013243B1734572D069
:105C50000A2AF4D1002009B0BDE8F08F1A4608AB3B
:105C60001A44002302F80C3CBEF1000FF2D16B1E67
:105C70000134032B03D8DFE803F05439106405A87E
:105C800015F0B8F90135EDB2042D014660D85D4438
:105C90000AF1010A95F8C0E6C7E79DF81420002A2A
:105CA00045D00DF1140E8C464320824248494FF0F6
:105CB000000306D00133072B04D011F8010B8242F8
:105CC000F8D19946542A64D04F2A67D0422A6CD022
:105CD000562A73D0492A57D0572A08BF052354D0D3
:105CE0001EF8012F002ADFD1614620E09DF8143014
:105CF000EBB105AA0EE0452B55D0532B5AD0572BAC
:105D00005AD0552B5FD0442B08BF052305D012F87D
:105D1000013F63B14E2BEED1002308FA03F31F437A
:105D2000F5E705A8039115F065F903990190013590
:105D3000EDB2ACE7002208AB1A44002302F80C3C99
:105D400095E705A8039115F055F90F28039919DD7A
:105D50000022019B03F00F0343EA8753134343EAF6
:105D600009231C4A43EA0636029B0901C9B202EB29
:105D700083090E43C9F8E060FFF746FE012009B031
:105D8000BDE8F08F8204E4E7042308FA03F31E431E
:105D9000A6E7002308FA03F31E43A1E7012308FA4C
:105DA00003F31E439CE70123B7E7022308FA03F33A
:105DB0001E4395E70223B0E70323AEE7032308FA67
:105DC00003F31E438CE70423A7E700BFF81E00205F
:105DD0007D4E0608181E002020E0050810B5FFF7CC
:105DE00013FE074B40F6A84203F2B450002193F88B
:105DF000614247F0CDF8034B83F8C04610BD00BFA9
:105E0000181E0020102F0020F0B5364C364D94F8A7
:105E100074112B68C4F85C342868C4F8500400235B
:105E2000022985B0C4F8CC32C4F8D032C4F8D432D8
:105E3000C4F8D83284F8DC3284F86134C4F84834C9
:105E4000C4F84C34C4F8C83284F86034C4F8583408
:105E500084F862343BD002200EF07CFAA8B30779B4
:105E600094F86134214E02E0CBB2042B35D803EB19
:105E7000430206EB8202591C92F87121BA42F3D117
:105E800084F8613494F86134194A90F902000C21C5
:105E900001FB0366002796F87131029752F8233010
:105EA0000093032101913B463A4602210EF0A6F9E8
:105EB000C4F8680448B12B68C4F85C340123C4F802
:105EC000587484F8627484F8603405B0F0BD2B68AF
:105ED000C4F85C3484F86014F7E7002384F8613474
:105EE000D0E700BF102F002074C5002020E0050877
:105EF000C81B060870B50446CC2582B044306171D9
:105F0000A11D2571CDE90010251D9AB16E461146DF
:105F100030461A4615F0EEFA3046294614F040FC99
:105F2000009A019220680095521B294629F026F913
:105F300002B070BD6E46EFE72DE9F04F9D4DDFF8E2
:105F400088B2AB7887B005F104084FF0640ADBF83B
:105F500000604BB32C780AFB0452144613690434D6
:105F6000002B52D09E4250D9D36D002B00F38A8073
:105F700002274FF000090BE0AB7085F800909BB151
:105F80002B69002B40D0B3423ED2EB6D002B79DC65
:105F9000236984F860702046444603B19847AA7884
:105FA000531EDBB2002AE7D1834C844FA4F2C465B0
:105FB00005F5D96800265FFA86FA0AF118095FFA32
:105FC00089F9484638F036FA00286ED0A35D002BD8
:105FD00040F0D780B9F1190FB5F80E3700F0D68030
:105FE000B9F11A0F40F09F8058077CD53B78DA074B
:105FF00000F18580724B1A6812F0600F40F06681E4
:106000004FF01B0A0221C6E044466369186829F074
:10601000E5F80028C8D06369186829F0D7F8A37894
:1060200053B994F85720012A04D02AB9552803D02F
:10603000AB788CE7CC28FBD16268D054A378627827
:106040000133DBB29A42A370F2D194F85730012B9E
:1060500035D0002B43D162681178552973D023695C
:10606000012284F86020002BE2D02046984794F863
:106070006020AB78002A7FF46AAF002B4ED1DBF8AA
:10608000003091E794F85730012B3BD023B9636976
:1060900021781868FDF7A6FDA268A36D1644013BA0
:1060A0000022E660A365A2707EE70AF1190AA055F6
:1060B0005FFA8AFABAF11B0F1AD001367BE762B198
:1060C0006668013EB718002016F8011F14F0A4FB03
:1060D000BE42F9D1021C18BF012284F86020236956
:1060E000002BC2D1C3E7D5F8183559073FF57EAF6D
:1060F000344B1B781BB9314B1B78DB0766D507B0D7
:10610000BDE8F08F60690368002BC5D094F8563065
:10611000217804F11802FFF7EDFEBDE7013BDBB289
:10612000AB702A7013E70AF1190A9B075FFA8AFA23
:106130007BD53B78D907BDD4214B1B6813F0600396
:10614000B8D1194627E05178012988D19178FF29E3
:1061500085D11179AA2982D1D678D17061680F1DB5
:1061600011F8012B5340082204E05B00DBB2013A36
:1061700000F0B2801806F8D5580080F03100C3B2A4
:10618000F5E70AF1190A5FFA8AFA93E7DA0752D5B6
:106190004FF01A0A012195F80C378DF81610012BD3
:1061A0004ED023B90131D5F8C806FDF71BFD0123F8
:1061B000A3557FE770D20020D43500203093002013
:1061C000B4960020DF96002074C50020794B1B6830
:1061D00013F0600393D1784C94F82125002A3AD02B
:1061E000764A9188A1F24751B1F5957F87D85188B9
:1061F000A1F24751B1F5957F81D81288A2F247529A
:10620000B2F5957F3FF67BAF6D4A029202214FF4C3
:10621000C872CDE9002104F5D9601A46032141F086
:10622000DFFC012384F8203569E7D5F81835980795
:106230007FF540AF7DE7D5F81835DB07A8D43CE7FC
:10624000D5F8C826002AB2D019460DF116024046EC
:10625000FFF750FEABE794F82035002B7FF44FAFEB
:10626000564B94F82215D888A0F2475080B2B0F56A
:10627000957F3AD8B3F90020A2F24755ADB2B5F5F3
:10628000957F68D85D88A5F24755B5F5957F44D8C8
:10629000B3F90450B5F5876F3FDA00293FF42FAF0B
:1062A00006AA022302F8013D454901934FF4C87341
:1062B000029100930421012304F5D96041F090FC80
:1062C000012384F8213584F8203518E73D4A1278F7
:1062D000002A3FF47CAF12E7B9427FF441AFF31AD2
:1062E00018BF012384F86030F9E600293FF407AFB6
:1062F000B3F90020B2F5876F30DA022306AA3048DE
:1063000002F8013D02214FF4C873CDE9011000935A
:106310002D48012341F064FCD2E7F9B95A88A2F272
:106320004752B2F5957F3FF6EAAEB3F90430B3F5C4
:10633000F06F7FF7E4AE06AA0123214902F8013D80
:10634000022002914FF4C871CDE9001004211E48CB
:1063500041F046FCB4E70029CCD1D0E6B3F90210F5
:10636000B1F5F06F1FDCB2F5F06F1EDCB1F5876F91
:106370001DDBB0F5957F3FF6C2AEA2F2475292B256
:10638000B2F5957F3FF6BBAEA1F2475292B2B2F59D
:10639000957F3FF6B4AEB3F90430B3F5F06F7FF7F5
:1063A000AEAE0123AAE70423A8E70323A6E705234B
:1063B000A4E700BFB4960020102F002040DA002090
:1063C000013D0108DF960020D835002030B51B4C78
:1063D00085B000254FF4804084F810570DF0BAFFC7
:1063E00018B34FF4E133032290F902000295CDE98E
:1063F00000324FF480412B462A460DF0FFFE94F800
:106400001C35C4F8C80684F80C3770B10C4994F8F0
:106410001025D4F814350093CDE901212B462A46E6
:10642000294604F5D96041F0DBFB012384F8C4362A
:1064300084F8C53684F8C63605B030BD102F00206C
:106440004F3C01080A4B1B7803B1704710B5094C4B
:1064500004F2147005F0B6FF00B910BD05F088F91C
:10646000054B1B6803F5C873C4F82C3210BD00BF80
:10647000DF960020102F002074C500200A4B30B595
:10648000D3F86815094C0022155D854208BFA11894
:106490001032A02AF8D193F86C25C3F8681542F0A1
:1064A000020283F86C2530BD102F0020E8E60508B5
:1064B000144C08B50646D4F868040DF07FFE30464B
:1064C0000DF07CFED4F8685429798A0711D50E4B5B
:1064D0001B689B0308D50820FFF7D0FF94F86C35A4
:1064E00023F0010384F86C3531462846074A42F010
:1064F00065FD284641F0020128F060FED4F868549A
:10650000E5E700BF102F00208CD800200D7B01088C
:10651000024B0146D3F85005FDF713BF102F0020A2
:10652000F8B5104E104F0024B378A34201DD0E2CB5
:1065300000D1F8BD61100131C9B2D7F85005E5B2FC
:10654000FDF76AFF284643F029FEB378A34206DD33
:106550002020FFF7DDFF681CC0B243F01FFE0234AD
:10656000E2E700BF70D80020102F0020642928BF68
:106570006421F8B511FB00F56424064695FBF4F49C
:106580000027E4B2FBB29C4212D8A6420BD91420D9
:1065900095FBF0F0C4EB84156638C4EB8505284400
:1065A000C0B2FFF7B5FF0134E4B2B44205D3F8BD81
:1065B0009F20FFF7ADFF0137E4E79A20FFF7A8FF20
:1065C000F1E7F7B52F4F7A7A002A57D02E4B2F4D8F
:1065D00019886423B1FBF3F203FB12132C490978E9
:1065E00000919BB22B4905F2245014F0C3F8FDF73B
:1065F000F3FBD5F8504501212046FDF70DFF05F2CC
:1066000024512046FDF7BCFE1EF008FE022105467F
:106610002046FDF701FF29461520FFF7A7FF0326B7
:10662000BB7A6BB31C49194D0868896800916423D3
:106630000A2190FBF3F203FB120305F2245093FBB3
:10664000F1F3164914F096F8FDF7C6FBD5F850455E
:1066500031462046FDF7E0FE05F224512046FDF7C5
:106660008FFE1EF0DBFD711C05462046FDF7D4FEB3
:106670002946152003B0BDE8F04077E70126CFE7B3
:1066800003B0F0BD8893002070930020102F0020ED
:106690007693002006660608A49300201F6606086D
:1066A000072937DCF0B500EB81001B4F83B00D46A6
:1066B00000F1FF0420262A46394601A814F05AF8B2
:1066C0009DF80430E21EABB19DF8052004F8033CB0
:1066D0002346CAB19DF8061004F8022CB9B104F89B
:1066E000011C01350022082D04F104041A70E2D1C6
:1066F00003B0F0BD0220531E111803F8016F994238
:10670000FBD1431C1344ECE7A21E0120F3E704F87D
:10671000016CE6E7704700BF186706082DE9F041F5
:1067200000EB01130024DFF884805C8082B0074610
:106730000E469C80DC801C815C819C81DC811C82FB
:1067400000F1D205013428462246414614F012F8E1
:10675000082C05F10205F5D1721C1349684614F0A6
:1067600009F806EBC602823269463A4411F8013B49
:10677000013C73B102F8013B002CF7D137440023F0
:106780003136137087F8CA6087F8E23002B0BDE88E
:10679000F081531E1019202103F8011F8342FBD101
:1067A00001342244EAE700BF206706084381060857
:1067B00010B411F8013B541E4BB100F8013B2246C6
:1067C000002CF6D1002303705DF8044B7047002ABB
:1067D000F8D0431E0119202203F8012F9942FBD162
:1067E00001342044002303705DF8044B70472DE909
:1067F000F04F3A4F3A493B4B97F8240797F8252733
:1068000008601A6007F2A67607F6440907F2EE75EB
:1068100007F6650807F66F0E07F2247C07F6780B7B
:1068200007F6880A00240CEB04020BEB04030AEBC6
:10683000040032F8021F23F8021B8342F9D115F835
:10684000012B49F8046B1034EB7D08F8012B802CE8
:1068500006F109060EF8013FE5D1234B2348C7F89E
:1068600040089A1C191DC7F800299A1D2D20C7F849
:106870000419C7F8082903F1080103F10A021C4CA6
:10688000C7F80C19C7F8102903F10C0103F10E0227
:1068900087F864081748C7F8FC38C7F81419C7F810
:1068A000182903F11A0103F12A020CF1FC0C03F57B
:1068B0009573C7F8F84831F8024B43F8042B61454B
:1068C00020F8024F02F10402F5D10B4A97F80E1896
:1068D0000A4B1160C7F81C39BDE8F08F102F00205B
:1068E000648800202C8800200637002028670608CE
:1068F000507D06081A880020188800203467060892
:1069000060B151B1064B1B68994206DC0139054B59
:1069100033F811301380012070470020704700BF0A
:10692000188800201C880020A0B1002911DD0A4B26
:106930001B688B420DDB002A0BDD084B1B689A425B
:1069400007DC02EBC102064901EB4202B2F866081D
:1069500070470020704700BF648800202C8800200A
:10696000102F002058B1002909DD064B1B68994201
:1069700005DC054B03EB8101D1F8F80870470348AB
:10698000704700BF2C880020102F00201C6B0608C9
:1069900050B1002908DD054B1B68994204DC044B0B
:1069A000194491F8640870473F20704764880020BC
:1069B000102F002003689B6A184703685B6A18471A
:1069C00003681B6A18472DE9FF41294B294D1C68B4
:1069D000297880462046FFF7DBFF69780646204687
:1069E000FFF7C0FF00230393AB788DF80B30074609
:1069F00054B303A92046FFF7DDFF2B7A23B10DF135
:106A00000B012046FFF7DCFF9DF80B20E2B11A4B8B
:106A10001B689A4218DC194B03EB8203D3F81C491C
:106A2000262037F007FD039A80B912F0010F0CBF42
:106A3000002350239207D8F8040009D5104913F019
:106A400099FE04B0BDE8F0810E4CE9E74423F1E77C
:106A50003BB1CDE9004332463B460B4913F08AFE79
:106A6000EFE700943B463246084913F083FEE8E71F
:106A70002C9300202093002018880020102F002045
:106A8000326606081C6B06083A6606084666060863
:106A900003682DE9F341DB6980460D4616469847A9
:106AA00018B12B7883BB337873BB194B1B785BB35E
:106AB000184A127842B3184C234493F86F781FBBDE
:106AC0000DF106014046FFF778FFE8B1134B2F7038
:106AD0003770134A1B681768BDF806C0013B04F6FF
:106AE000780202EB0312002B0EDB0021B94202DB1D
:106AF000013B103AF7E732F81140644501F101011A
:106B0000F4D101332B70317002B0BDE8F08100BFC9
:106B10006593002066930020102F002064880020D9
:106B20002C8800202DE9F041764B1C6882B0002CA7
:106B30003FD0FF230D468DF803308DF8023000283A
:106B40003AD1714C94F84039002B6DD06F4B93F8CB
:106B5000DC5075B36E4994F846094A6991F810E023
:106B600000284FF0000102F0010803F1E00014BF1B
:106B70004FF00F0C8C460A460F4603F5E87350F8A9
:106B8000044B24040ED5002A4BD0964503D3B8F10C
:106B9000000F00F08580002426460132D2B21E800C
:106BA0009F70DC700131A94203D0062A03F104036F
:106BB000E5D102B0BDE8F081554E0DF102020DF1B4
:106BC00003012046FFF764FF06F110012046FFF79E
:106BD000F7FE06F114012046FFF7ECFE9DF8038056
:106BE0009DF80270204641463A46FFF79DFE7269C5
:106BF000317C454C02F0010303EB410303EB081326
:106C000094F84029A4F8420903EB07239BB2002A19
:106C100049D1B4F844299A425ED0A4F844390F22ED
:106C200043E064467826B8E7394EB4F8423941F279
:106C30002862934219D80123344A716902EB830315
:106C4000D3F860310193CB0740D594F84639002B37
:106C50000CBF00230F2301A94FF400408DF807302B
:106C6000F9F766FE02B0BDE8F08141F24F6293424F
:106C70002ED941F2766293422CD941F29D62934221
:106C800039D941F2C562934237D941F2EB6293425E
:106C900035D941F2127293428CBF0D230B23CBE7FF
:106CA00064461E2679E7A4F84439296894F8460911
:106CB000531E01F54332DBB202F5A07280F00101F0
:106CC00084F840392A6084F846193DE7FF23C2E77B
:106CD0000223B1E70323AFE72B6894F84619A4F821
:106CE000442903F5433303F5A07381F001022B60BF
:106CF00084F8462999E704239EE706239CE70A23A4
:106D00009AE700BF2C930020102F0020181E0020AF
:106D1000A001002003685B691847044A1268914289
:106D200002DC03681B691847704700BF1888002001
:106D300070B50D4604461646FFF7F6FD0146A8B1AC
:106D40000B4B1E700B4B1D700B4B22682B4493F8A2
:106D50006F3833B1D368294632462046BDE87040CB
:106D6000184720469369BDE87040184770BD00BFC2
:106D70006693002065930020102F002010B1036857
:106D80005B681847FF20704710B50C4658B128F0D3
:106D9000C9FA18B1032383710023C3712146BDE8EA
:106DA000104028F057BC10BD10B5044601210079F1
:106DB000FFF7EAFF627920689108838902228A40FE
:106DC00023EA0203838110BD10B504462221007915
:106DD000FFF7DAFF63792268990802238B409BB2A0
:106DE000D94389B2118291890B43938110BD73B548
:106DF00090F85F38032B05460C462AD100231E4E1F
:106E00008DF807309DF8073095F860289A4201D830
:106E100002B070BD9DF8073006EBC3031B797BB150
:106E200084F0010373B19DF8073056F8330028F061
:106E3000E5FC9DF807300133DBB28DF80730E1E760
:106E40002346EFE79DF8073056F8330028F0D0FCD2
:106E5000EFE7436C006CDB79DB0748BF81F001048E
:106E600024B102B0BDE8704028F0C8BC02B0BDE853
:106E7000704028F0BDBC00BF38D9002070B5A0F626
:106E8000640494F8513893B1B4F8583801339BB284
:106E9000082BA4F858381CD9002184F85118A4F8FC
:106EA0005818606C40F00AFF94F851388BB93E4E88
:106EB00096F847391BB901212046FFF798FF94F84F
:106EC000503853BBD4E909239A4203D1002386F8F2
:106ED000473970BD96F84729022A12D802F10102FB
:106EE00014BFFF237F2386F84729A4F854380823CA
:106EF00084F85238012384F85038606CBDE8704043
:106F000052E75A1CA169A262CB5C21698A4228BF60
:106F10000022DBB228BFA262E7E794F95238C3B37C
:106F200094F8541896F8485911F0010123D0012D16
:106F300003D801212046FFF75AFFAB1E012B03D8CF
:106F400000212046FFF753FF0135EDB2032D86F8EF
:106F50004859BED9B4F854385B08A4F8543894F8AA
:106F60005238013B5BB2002284F8523886F8482937
:106F7000002BA7D0ADE715F0FD0304D10121204679
:106F8000FFF735FFE0E7012BDED12046FFF72FFFAB
:106F9000DAE7D4E9091291429BD184F85038606C49
:106FA000BDE8704010E700BF102F002010B5A0F61C
:106FB000640494F851381BBB94F850288ABBD4E978
:106FC000091399421CD0591CA069A162C35C2069B5
:106FD000DBB25B0043F40073A4F854380A2384F84E
:106FE0005238012384F8503894F85F38814228BF22
:106FF000A262012B01D0042B02D1606CFFF7D4FEFA
:1070000094F84C38002B6FD194F84D380133DBB233
:10701000092B84F84D3827D12046BDE81040F9F7F8
:107020001BBF94F952387BB1B4F854184B08A4F83C
:10703000543801F001012046FFF7D9FE94F8523888
:10704000013B84F85238DBE784F85038D4E909234F
:107050009A42D5D194F85F38012B01D0042BCFD1BF
:10706000606CFFF7B1FECBE70A2B3DD194F84F38A7
:107070002BB9B4F8563843F00103A4F856382379F5
:10708000D9070AD5B4F85608820501D4C30718D425
:10709000B4F85C380133A4F85C38012284F84C2839
:1070A00094F84F280023012A84F84D381CD16179C7
:1070B00084F84F38606C01F00101BDE8104040F0E9
:1070C000FDBDE36AC0F3470013B1216B9847E4E7C5
:1070D000E3696269D054E369E1680133B3FBF1F21B
:1070E00001FB1233E361D8E710BD2DE9F043C34E35
:1070F00096F8A49599B0B9F1000F40F07381C04C97
:1071000094F8C086B8F1000F00F06C814A462F2138
:107110004046F3F7DDFE0546002800F06381036872
:10712000C4F8683128F0C8FC002800F05B8143688F
:10713000C4F86431002B00F055818768404628F080
:10714000F1F8C4F84C0918B12F23837180F8079027
:107150002A7A2A2128F0AEF9D4F86801F3F7B2FDB3
:107160003EF0A2FCD4F86801A6490388A64ADFF8DD
:10717000B0C223F001031B041B0C8842038010D013
:10718000DFF888E2136870450BD00EF5804E70452D
:1071900007D00EF5806E704503D00EF5806E7045F9
:1071A0007FD11368634540F2828088420FD0DFF8B8
:1071B0005CC260450BD00CF5804C604507D00CF5E7
:1071C000806C604503D00CF5806C60456CD103F198
:1071D000B77303F55853DFF84CC2B3FBFCF3013B24
:1071E0009BB288420ED0894988420BD001F580417C
:1071F000884207D001F58061884203D001F58061A3
:10720000884257D11268591C4FF0030CB2FBF1F2BF
:107210007F49B2FBF1F291B2B1FBFCF14FEA410CB4
:10722000A6F8B01518A94FF0000821F85C3D0292AD
:10723000A6F8B2C5ADF80C80ADF806808DF80E80CA
:1072400021F0AFFECDE906886023CDF820800493BD
:10725000EB79ADF814809A072FD5DB00042203F0F8
:107260000803ADF81420ADF81E30002306936979A9
:10727000D4F8680104AAF2F747FD6979D4F86831B7
:107280000C292FD8DFE811F026002E002E002E004A
:10729000B1002E002E002E00D0002E002E002E0059
:1072A000D900BCEB530F04D213685B088FE70023AF
:1072B00097E7002312685208A5E701225B00ADF8AA
:1072C000122003F002034FF48072ADF82020ADF8D5
:1072D0001C30CAE71A8B22F008021204120C42F08A
:1072E00008021A83B3F8442042F40042A3F8442071
:1072F0001A8842F080021A80EA7990074CBF042273
:10730000012202FA01F11A8CD4F8640189B222EA4E
:1073100001021A841A8C114319841A8842F001025E
:107320001A803BF04DFA00222F213BF05BFAD4F893
:1073300064013BF045FA6022364900233BF08AFAAB
:10734000D4F8640121F004FFD4F86401036823F049
:107350000103036021F0FCFE09A821F0BDFED4F872
:1073600068316A79D4F864010997343313440A9375
:107370004FF0000840F22A33CDE90D384FF4806316
:107380000F93254B0B9340230C934FF480514FF4F4
:107390008043CDE910134FF4403309A9CDE912839E
:1073A00021F0ABFE6979D4F868210C2904D81B4B75
:1073B00003EB4103B3F86887938948EA0308A2F80E
:1073C0000C80D4F86421136843F01003136009A8FB
:1073D00000230993F9F758FE0120F9F759FD01231D
:1073E00086F8A43519B0BDE8F0831A8B22F4006248
:1073F0001204120C42F400621A8373E7181E002074
:10740000102F00200004014088BC00200000014033
:1074100000350C00F3FA0408CC23002020E0050816
:10742000FF6BDC02006CDC029A8B22F00802120473
:10743000120C42F008029A8354E79A8B22F40062FD
:107440001204120C42F400629A834BE72DE9F04FCC
:10745000C44C94F8A4358DB013B194F8A53513B18C
:107460000DB0BDE8F08FC04D95F8BD7606460C20F6
:1074700036F0E0FF002F73D0002876D1FFF735FEFD
:10748000012385F8BD3694F86372012F74D9022F59
:10749000E6D10023B54FDFF80083DFF800E3DFF823
:1074A0000093B5F8BE064FF0010C1D4640FA03F2FA
:1074B00012F0010F4FEA83010DD157F82320B21AC1
:1074C00002EB080AF2450CFA03FB04D94A4588BFCF
:1074D000CE5145EA0B050133092BE7D1002DBFD072
:1074E00094F8DC00002800F01F81A14E94F8C771C9
:1074F000DFF8B0A236889F4994F8C42194F8C531CA
:107500000596203794F8CF61097804960AEB870630
:1075100020323AF8277002972033B778F67803962E
:107520000AEB800001F001010AEB82020AEB8303FF
:107530000197069109920893D3460AF1F006814615
:1075400007955BF8047BC7F3032307F48055042BEE
:1075500063D8DFE813F07B004A00450142012D01AA
:1075600000288BD00DB0BDE8F08FFEF7CFF995F86D
:10757000BD36002B87D173E70B2036F05BFF002868
:1075800000F037817C4A7D4B126894F86A72A3FB45
:1075900002131B09FA2101FB13237D2B28BF0027AF
:1075A000DFF8048298F80F30BB4204D1D5F8743963
:1075B0009E42FFF455AF724800EB8700F9F764FD77
:1075C00094F86202F9F764FC07EE906A9FED6D7A19
:1075D00088F80F70F8EE677A77EE877AFCEEE77A34
:1075E00017EE903AC5F874393AE70599002240231E
:1075F000194207D10132052A0FD0634B33F82230EC
:10760000002BF5D1C7F38553002143FA01F0C007E1
:1076100000F13E8101310629F7D1DDE902320199FD
:107620004FF4B470002D6AD0049F584D35F91750AF
:107630004FF4B477A5F57A7507FB05F54F4F87FB37
:1076400005C7ED17C5EBA715284458E0C7F38347D6
:1076500007F120030AEB83023AF823309178D278BD
:10766000002D00F0E48007F1110000F00F00203041
:107670000A900AEB800507F10F080498434F37F989
:1076800010C00A9808F00F083AF820000A9008F194
:107690002008A8780B900AEB880E40F2DB50844556
:1076A0003AF82870ED789EF802809EF803E000F327
:1076B000C380ACF57A7C314DA1EB08010CFB01F1E4
:1076C000A2EB0E02DB1B0CFB02F20CFB03F385FBAF
:1076D00001C0C917C1EB6011284885FB02C580FBBA
:1076E00003C0D217DB17C3EB6013C2EB6512414432
:1076F00072443B44C9B2D2B29BB24FF4B47003445B
:107700002348B17080FB03051D44D817C0EB25202A
:107710004FF4B47505FB1030D945F270308006F196
:1077200004067FF40EAF079D104FDFF88080194BE1
:1077300000264FF0010901E058F8043F09FA06F26B
:107740002A4214BF01200020394601369847092EED
:1077500007F10407F0D194F862020DB0BDE8F04FD4
:10776000F9F796BB181E0020102F0020603800206B
:10777000B09300203093002074C50020D34D6210D8
:1077800038E0050800247449A4E7050840DA002021
:10779000B7600BB6910501083F4B4C003E4B4C00C7
:1077A0009F860100F81E0020A0010020B8E7050810
:1077B0002CF026FD00B200EB80004B4BC0EB00101C
:1077C0004000A3FB003040091E3820EAE07000238F
:1077D00000F5B4701946FF2224E71DF01FFDE9E70C
:1077E000069B3BB3089B9978DA781B884FF4B470FA
:1077F00018E73E4BDB78002B7FF4C4AE012F44D159
:1078000094F86932002B59D0394B1B7813F00103DF
:1078100054D11F4694F86032002B3FF4C1AE94F867
:107820005D32002B3FF4BCAE94F86A72B8E64FF4B8
:10783000B47064E7099BD6E70B98471A0A98ACF234
:10784000DC5CC01A0CFB00F0AD1A0A9029480CFB56
:1078500005F50CFB07F780FB07EC80FB058E4FEA74
:10786000E5780A9DFF17C7EB6C1780FB050CE8173E
:10787000C0EB6C10C8EB6E15034439442A44C9B2FE
:10788000D2B29BB24FF4B47039E794F86472C1E796
:10789000194B03EB82024FF4B47092F8863703EB76
:1078A000430304EB4303194491F8A03120330AEB5E
:1078B00083023AF823309178D278B3E60F4AB4F8CD
:1078C000661294F868321068074FB0FBF1F201FBC2
:1078D00003F301FB1202A7FB0313B2EB531F94F84F
:1078E000657228BF002795E71F85EB513493002070
:1078F00030930020D34D621020E0050874C50020AD
:1079000038B541790446AE23802290F904003CF05A
:1079100041FC054688B1162209492046FCF73BFD8B
:10792000042208492046FCF736FD2046FDF7E0F822
:10793000032205492046FCF72EFD284638BD00BF2E
:10794000DCE70508F2E70508F6E70508F8B5684C36
:10795000D4F87839064623B193F90F30002B00F3A1
:10796000C680D4F87C39F31A002BC0F2C08006F52B
:10797000433303F5A073C4F87C395E4B1D7894F84B
:10798000803905F0010584F8805975B3012B00F0AA
:10799000AE800120FEF772FD012384F8643594F86F
:1079A0006435002B59D094F86C3523F0020384F829
:1079B0006C35514B3344D4F85065C4F870353046BB
:1079C000FFF79EFF84F88109002800F09080304680
:1079D000FDF78EF830460021FCF71EFDD4F868351F
:1079E00030465968FCF7CCFC37E02BB194F86C3585
:1079F00043F0020384F86C3594F86C3513F00201FF
:107A00001DD0012284F86425D907C8D594F86D35B6
:107A10003A480A210133DBB2B3FBF1F201FB123326
:107A2000DBB200EB031292F8D426D207F2D4344A28
:107A300084F86D3502EB0313C4F86835AFE7D4F86A
:107A40007025B21A002A02DA84F86415A7E703F059
:107A5000010284F86425002AD6D194F88139002BDC
:107A600045D0D4F868359B689847002D3FD1254B09
:107A7000224F93F82430D4F85065062B96BFDB19BB
:107A80003F2593F8D957002212213046FCF793FC8A
:107A900029463046FCF755FC132100223046FCF7FE
:107AA0008AFC194B93F85232002B94F8823914BF98
:107AB00072212121002B18BF52213046FCF741FCD6
:107AC000002214213046FCF776FC94F883592F44A9
:107AD000304697F8A3150135FCF733FCEDB20523CA
:107AE000B5FBF3F303EB8303ED1A84F88359F8BD78
:107AF000102F002030930020404B4C0020E0050860
:107B0000E8E6050834930020181E002008B5FAF7AF
:107B100013FE054B1B689B0300D408BDF4F7CEF899
:107B2000BDE8084012E700BF8CD800202DE9F041E5
:107B3000124E96F89C20551E05EB05157119074647
:107B400091F89E1029B90E494068BDE8F04112F045
